:020000040800F2
:10000000A8A20020D5020008EF37000841310008FF
:10001000ED370008890C0008AB4100080000000023
:100020000000000000000000000000003D02000889
:10003000130F000800000000810200087B3900084F
:10004000EF020008EF020008EF020008EF020008CC
:10005000EF020008EF020008EF020008EF020008BC
:10006000EF020008EF020008EF020008EF020008AC
:10007000B90E0008C50E0008EF020008EF020008E4
:10008000D10E0008DD0E0008EF020008EF020008A4
:100090008D0C0008990C0008EF020008150F0008ED
:1000A000EF020008EF020008EF020008EF0200086C
:1000B000EF020008EF020008EF020008EF0200085C
:1000C000EF020008EF020008EF020008EF0200084C
:1000D000EF020008EF020008EF020008EF0200083C
:1000E000EF020008EF020008EF0200080000000025
:1000F0000000000000000000000000000000000000
:100100000000000000000000EF020008EF020008FD
:10011000EF020008EF020008013A0008EF020008B1
:10012000EF020008EF020008EF020008EF020008EB
:10013000EF0200080000000000000000EF020008CD
:10014000A50C0008B10C0008EF020008EF0200083F
:1001500000F002F800F063F80AA090E8000C824476
:100160008344AAF10107DA4501D100F058F8AFF253
:10017000090EBAE80F0013F0010F18BFFB1A43F085
:100180000103184784E80100A4E801000A444FF085
:10019000000C10F8013B13F0070408BF10F8014BE6
:1001A0001D1108BF10F8015B641E05D010F8016B2B
:1001B000641E01F8016BF9D113F0080F1EBF10F88F
:1001C000014BAD1C0C1B09D16D1E58BF01F801CBB2
:1001D000FAD505E014F8016B01F8016B6D1EF9D535
:1001E0009142D6D37047000000230024002500264A
:1001F000103A28BF78C1FBD8520728BF30C148BF8A
:100200000B607047642900F0A181002070471FB582
:100210009DE8030000F042FB1FBD10B510BD00F0CB
:1002200019FC1146FFF7F3FF16F059FC00F037FCFC
:1002300003B4FFF7F2FF03BC00F068FC224B19681F
:100240000868B0E8F00F80F30988BFF36F8F4FF0B4
:10025000000080F311884EF00D0E70470000000082
:1002600006480068006880F3088862B661B6BFF38C
:100270004F8FBFF36F8F00DF00BF00BF08ED00E0BE
:10028000EFF30980BFF36F8F0F4B1A6820E9F00F6F
:10029000106008B54FF0500080F31188BFF34F8F06
:1002A000BFF36F8F19F0E6FE4FF0000080F3118866
:1002B000BDE8084019680868B0E8F00F80F30988C5
:1002C000BFF36F8F704700BF1C000020EFF3058065
:1002D000704700000948804709480047FEE7FEE7ED
:1002E000FEE7FEE7FEE7FEE7FEE7FEE7FEE7FEE7E6
:1002F00004480549054A064B70470000FD390008CF
:1003000051010008A8820020A8A20020A892002085
:10031000A892002070B5064600F0A4FA056806F120
:100320000B0020F00704B4429CBF002070BD2B4698
:100330006A68BAB11068A04210D304F1080188427B
:100340003CBF5068586007D351681019416011686C
:10035000091B016058601460101D70BD134652687F
:10036000002AE7D12146284600F084FA0028DED191
:1003700070BD70B50446051F00F074FA0068002CCB
:1003800014BF446870BD002C18BFAC423CBF20466F
:100390006468F8D301680A18AA4218BF456003D1FF
:1003A0002A6805461144016028684119A1421CBF12
:1003B0006C6070BD6168696021680844286070BD28
:1003C00053EA020C00F069802DE9F04B4FF0000673
:1003D000002B1FBFB3FA83F503FA05F424FA05F6E0
:1003E0005E4012BF1643B2FA82F502FA05F4C5F177
:1003F00020051EBF22FA05FC44EA0C04203556EA0B
:10040000044C4FEA144418BF641C4FF000084FF02E
:100410000009904271EB030C39D3002919BFB1FADE
:1004200081F701FA07F6B0FA80F700FA07F6C7F18C
:1004300020071EBF20FA07FC46EA0C062037B6FB51
:10044000F4FCA7EB0507103F07F01F0BCBF12006CC
:100450000CFA0BFB2CFA06F644BFB3460026202FFD
:10046000A4BF5E464FF0000B5BEA060C08BF4FF0DE
:10047000010B19EB0B09ABFB027C48EB0608C01B18
:1004800006FB02CC0BFB03CC71EB0C01C1E70B4666
:10049000024641464846BDE8F08B13B54FF00000D8
:1004A0004FF00001AFF30080BDE81C407047000032
:1004B0000FB41CB50C0007AA009001D02044401EC8
:1004C000074B7B4469460190069800F07CFA002CAB
:1004D00003D06946002000F089FA1CBC5DF814FBCB
:1004E000310500002DE9F0410E460446002020624F
:1004F0002046E168884730B3252805D0D4E901219A
:100500009047206A401CF2E7E168204600278847B0
:10051000050018D0A5F14100192802D820354FF464
:1005200000673246294620462760FFF76BFE40B140
:10053000012804D0F61D26F007060836D8E7361D38
:10054000D6E72846DAE7206ABDE8F0812DE9F041D8
:100550000646002410687529314616A510D0AFF361
:100560000080002802DA404213A507E031688A07BC
:1005700001D512A502E0490704D511A5012401E027
:10058000AFF3008000210A2206F1240709E0B0FB46
:10059000F2FCB0FBF2F302FB1C003030785418463A
:1005A000491C0028F3D123462A463046BDE8F041D5
:1005B00000F0AAB9000000002D0000002B00000090
:1005C0002000000040EA0103024630B59B0710D12D
:1005D0004FF0013400E008C208C91D1B9D4315EA15
:1005E000C41FF8D013F0FF0102F8011B0DD01B0A45
:1005F000F8E711F8013B002B02F8013B05D011F898
:10060000013B002B02F8013BF3D130BD10B5431C78
:1006100002E010F8011B71B18107FAD14FF00132ED
:1006200002C88C1A8C4314EAC211F9D0C01A0A0607
:1006300003D0C01E10BDC01A10BD0A0401D0801E18
:1006400010BD0902FCD0401E10BD032A40F23080CC
:1006500010F0030C00F0158011F8013BBCF1020F03
:10066000624498BF11F801CB00F8013B38BF11F884
:10067000013BA2F1040298BF00F801CB38BF00F89B
:10068000013B11F0030300F02580083AC0F0088018
:1006900051F8043B083A51F804CBA0E80810F5E7FC
:1006A000121D5CBF51F8043B40F8043BAFF30080DF
:1006B000D20724BF11F8013B11F801CB48BF11F854
:1006C000012B24BF00F8013B00F801CB48BF00F824
:1006D000012B704710B5203AC0F00B80B1E81850DC
:1006E000203AA0E81850B1E81850A0E81850BFF41C
:1006F000F5AF5FEA027C24BFB1E81850A0E81850BB
:1007000044BF18C918C0BDE810405FEA827C24BF0E
:1007100051F8043B40F8043B08BF7047D20728BF9C
:1007200031F8023B48BF11F8012B28BF20F8023BEB
:1007300048BF00F8012B704702F0FF0343EA032291
:1007400042EA024200F002B84FF000020429C0F071
:10075000128010F0030C00F01B80CCF1040CBCF1F3
:10076000020F18BF00F8012BA8BF20F8022BA1EB45
:100770000C0100F00DB85FEAC17C24BF00F8012B2A
:1007800000F8012B48BF00F8012B70474FF0000222
:1007900000B5134694469646203922BFA0E80C5077
:1007A000A0E80C50B1F12001BFF4F7AF090728BF52
:1007B000A0E80C5048BF0CC05DF804EB890028BFCE
:1007C00040F8042B08BF704748BF20F8022B11F0F7
:1007D000804F18BF00F8012B704700004FF0013C1C
:1007E00050F8042B51F8043B9A4221D1A2EB0C03A0
:1007F000934313EACC1317D150F8042B51F8043B60
:100800009A4215D1A2EB0C03934313EACC130BD1FC
:1008100050F8042B51F8043B9A4209D1A2EB0C0387
:10082000934313EACC13DBD04FF00000704700BFB6
:10083000D01A01BAB1FA81F101F0180122FA01F0DF
:10084000CB40C1F12001DBB2C0B2C01A2CFA01F3D7
:10085000D11A914311EAC311E6D17047704770472E
:1008600070470000004870474C8200207047704776
:100870007047704738B504460A4600206946AFF312
:100880000080002808BF38BD02460099204600F0CD
:10089000BFF8012038BD012000F0D4B8F8B5AFF39F
:1008A0000080054600200C46102000BF0646A8190F
:1008B000A0420DD9324669460020AFF30080070000
:1008C00008BF00F0BFF80098A04218BF0546C41941
:1008D000FFF7C8FF05600746F01D20F00700461926
:1008E000284600F00AF8B44208BFF8BDA21B314602
:1008F0003868BDE8F84000F08BB800210160C0E91D
:1009000001107047102070472DE9F0470D469946B9
:100910009246044600F124080168880604D5E0697F
:1009200021F01001216000E00120A84201DD471BF9
:1009300000E00027A1697A1902EB0900081AA061FA
:100940002078C00602D42046AFF30080002608E0DD
:10095000D4E901211AF806009047206A401C761C51
:1009600020624E45F4DB2078C0060AD52046AFF35E
:10097000008006E0D4E9012130209047206A401C25
:100980002062381EA7F10107F4DC07E0D4E9012159
:1009900018F805009047206A401C2062281EA5F127
:1009A0000105F3DC2046AFF300802078000602D575
:1009B0000220BDE8F0870120FBE7000001694A1C26
:1009C00002610878704700B58FB0CDE90131002190
:1009D000059105497944CDE9031011466846FFF7B2
:1009E00081FD0FB000BD0000E5FFFFFF0A6802F8BF
:1009F000010B0A607047D1E900239A4202D2531CCE
:100A00000B6010707047000000487047448200205F
:100A1000034640688C46002818BF88423CBF034606
:100A20004068F8D318681844884207D00CF10300D6
:100A300020F00700001D411A521A0146081D0A60E5
:100A4000FFF797BC10B500F039F8BDE8104000F092
:100A50002FB870477546FFF7D7FFAE4605006946C9
:100A6000534620F00700854618B020B5FFF740FC3C
:100A7000BDE820404FF000064FF000074FF000089F
:100A80004FF0000B21F00701AC46ACE8C009ACE820
:100A9000C009ACE8C009ACE8C0098D46704710B584
:100AA0000446AFF300802046BDE81040FFF7C0BB0E
:100AB000002801D000F02AB87047000010B50128C6
:100AC00005D0002103A000F027F8012010BD09A1E6
:100AD000F8E7000053494752544D454D3A204F75B1
:100AE00074206F662068656170206D656D6F727926
:100AF000000000003A2048656170206D656D6F72DE
:100B00007920636F727275707465640001491820F2
:100B1000ABBEFEE72600020070B505460C460A2073
:100B200000E06D1C00F011F835B128780028F8D1EC
:100B300002E0641C00F009F814B120780028F8D114
:100B4000BDE870400A20AFF3008008B569468DF813
:100B500000000320ABBE08BD70B50A460546094932
:100B600010461AF08DF81AF06BF8074C80B2216825
:100B7000086428461AF064F8216880B28862002070
:100B800070BD000000FF7F47C802002010B50C2197
:100B9000034802F011F9002801D04FF0FF3010BDDA
:100BA000C802002010B50C21034802F059F90028B2
:100BB00001D04FF0FF3010BDC802002028B101283D
:100BC00001D000207047024870470248704700007B
:100BD00004020020DC01002052B100EB800303EB93
:100BE000C000054B03EB800040F821200020704737
:100BF0006FF00100704700005C8000202DE9F0419B
:100C000005464FF07E500E464FF0FF37824220DC03
:100C100011461AF001F919491AF032F81AF010F8D1
:100C200082B21748006825B1012D05D0022D10D1E0
:100C300005E00021426304E00421826301E0082111
:100C4000C2630124AC400F4D86B1012E07D0022EA5
:100C500002D03846BDE8F0812868044206D0084832
:100C600002F0FEF82868A043286005E0044802F07E
:100C7000A3F8286804432C600020EBE700FF7F47BF
:100C8000C8020020C8010020FEE70000014800F073
:100C9000DFBA0000DC010020014800F0D9BA0000F2
:100CA000DC010020014800F0D3BA0000040200205B
:100CB000014800F0CDBA00000402002010B5002069
:100CC000FFF77CFF084B0021A3F11C0200F046FA5D
:100CD00006480023044980681A461C39406BBDE869
:100CE000104016F0EBBA0000E0800020CC0100209C
:100CF00010B50120FFF762FF084B0121A3F11C0290
:100D000000F02CFA06480023044980681A461C3972
:100D1000406BBDE8104016F0D1BA000004810020FD
:100D2000CC01002000680649884201D101207047AB
:100D30000449884201D10020704703207047000019
:100D40000068004000640040F0B58BB00E4605001E
:100D50006FF0010754D02B4C207818B16FF00200CF
:100D60000BB0F0BD16F0EFFA6060002848D000220A
:100D70002421202016F076FAEE6268632821684666
:100D8000FFF704FD002001260190CDE9060605903D
:100D90000E270390049000900290CDE90867FFF7BA
:100DA0000DFF694600F03EF90020FFF707FF00F055
:100DB000DFFC154A06210020FFF70EFF0020FFF799
:100DC000FDFE022100F0B3F80120CDE90467FFF732
:100DD000F5FE694600F026F90120FFF7EFFE00F06E
:100DE000C7FC0A4A08210120FFF7F6FE0120FFF7A1
:100DF000E5FE102100F09BF8A56026700020AFE70B
:100E00003846ADE7CC010020BD0C0008F10C00080D
:100E100070B504461249838CC28C008D658D4FF4E9
:100E200088760E6000268E60CE6008260E611E0A4F
:100E30000E764B76130A8B76CA76020A0A774877C3
:100E4000280A8877CD77E06A4078FFF7B7FE044A32
:100E500004F130031832024900F07BF8002070BD25
:100E60000C81002030B56FF0010248B141B10B6830
:100E700043B1012B06D0022B04D0032B19D101E082
:100E8000104630BD8D8B00EBC3026DBA9580CD8BC3
:100E900000EB43046DBAD5800D8C6DBA1581498C79
:100EA00049BA51819188A184012201689A40114375
:100EB0000160002030BD0000014800F01DBD0000B1
:100EC00070040020014800F017BD000084020020DB
:100ED000014800F011BD0000E8030020014800F0C7
:100EE0000BBD00002C04002030B590F840500124C8
:100EF000AC40C56B6C60046863604368102B03688A
:100F000003D099600068C26030BD9A600068C1601B
:100F100030BD704710B54FF4807000F0AFFEBDE8F3
:100F200010404FF4007000F0A9BE72B6FEE790F8D2
:100F30002020012A07D0022A05D0416A41F48021ED
:100F4000416201207047006842690A434261002003
:100F50007047F0B590F820500468A468012D05D0C2
:100F6000022D03D0416A41F4802157E014F0406F14
:100F700001D1E5004FD5C4F301640125A5401D60F2
:100F80008D684FF4C0739DB1CE6835434E6845EA15
:100F9000C605066803EB0417F5514FF4C2750768E0
:100FA00005EB04150E697E51097D012905D009E084
:100FB0000E88CD6845EA4655EBE701684E5946F480
:100FC00080764E511179D579567941EA0561957946
:100FD0002D0445EA062529434FF4C676056806EB3D
:100FE0000416A9511178D57841EA056195785278AF
:100FF0002D0445EA022211434FF4C475026805EB43
:1010000004155151006803EB0411425842F00102EB
:1010100042500020F0BD416A41F4001141620120BC
:10102000F0BD000010B590F82020012A07D0022A58
:1010300005D0416A41F480214162012010BD3B4846
:10104000D0F8002242F00102C0F80022D0F80022BD
:1010500022F47C52C0F80022D0F800224B6A42EA07
:101060000322C0F800220A7D02F01F0301229A40E9
:10107000D0F81C329343C0F81C32CB69B3B9D0F816
:101080000C329343C0F80C328C894B6864F31F43D5
:101090004C6900EBC404C4F840320C890B6864F35B
:1010A0001F434C6900EBC404C4F84432CB69012BE4
:1010B00016D1D0F80C321343C0F80C320C884B68B0
:1010C00064F31F434C6900EBC404C4F840320C893C
:1010D000CB6864F31F434C6900EBC404C4F844328A
:1010E0008B69002BD0F804320ED01343C0F80432C1
:1010F0000B69002BD0F8143208D01343C0F8143217
:10110000096A012904D008E09343EFE79343F5E728
:10111000D0F81C121143C0F81C12D0F8001221F0B4
:101120000101C0F80012002010BD00000064004062
:1011300010B5FFF7F7FD03280CD000EB800101EBA1
:10114000C001054800EB8100006B002802D0BDE81B
:101150001040004710BD00005C80002070B590F882
:101160002040012C05D0022C03D0416A41F480219B
:1011700028E0046809B32469A40720D04FF4D87488
:10118000056804EB01142D5915F0040595600568F8
:101190002D591AD0ED08556005682C5904F0020449
:1011A000D4604FF4DA74056804EB01142E5906F08C
:1011B0000F06082E0CD308250DE0E468DCE7416A31
:1011C00041F400114162012070BD6D0D1560E3E72F
:1011D0002D5905F00F05156105682D59C5F3072533
:1011E000956105682C59240C54614FF4DC72046835
:1011F00002EB0112A4581C700468A458240A5C7005
:101200000468A458240C9C700468A258120EDA706A
:101210004FF4DE72046802EB0112A4581C710468DA
:10122000A458240A5C710468A458240C9C710468B6
:10123000A258120EDA71006829B1016941F020014B
:101240000161002070BDC16841F02001C160F8E774
:101250002DE9F05F0546006800244669D0F8049047
:101260008768D0F80CB0D0F810A0D0F81880F1073B
:1012700048D0F90714D001218160B80703D528466A
:1012800000F0B8FA0CE0780702D54FF4006407E0EC
:10129000380702D54FF4805402E0284600F094FA53
:1012A000F80516D529684FF480708860B80503D515
:1012B000284600F0C9FA0CE0780502D544F4005441
:1012C00007E0380502D544F4804402E0284600F0E7
:1012D000A5FAF80316D529684FF480308860B80362
:1012E00003D5284600F0DCFA0CE0780302D544F47C
:1012F000004407E0380302D544F4803402E0284675
:1013000000F0B8FA300707D55FEACB6004D529684A
:10131000102044F40074C86070074FF0080707D528
:101320005FEA0B7004D52868C760284600F0B2F960
:10133000B00706D52868C068800702D0284600F0AC
:10134000BFF9700607D55FEACA6004D52968102086
:1013500044F480640861B00607D55FEA0A7004D5DA
:1013600028680761284600F0C1F9F00606D528680C
:101370000069800702D0284600F0CEF9B00308D5F6
:101380005FEAC96005D5296810204860284600F04A
:10139000D9F9F00307D55FEA097004D528684760DA
:1013A000284600F093FA300446D55FEA497040D5EC
:1013B000F00504D55FEAC87001D044F00104B0051F
:1013C00004D55FEA887001D544F00204700504D5A5
:1013D0005FEA487001D544F00404300529D518F0BF
:1013E000700F26D008F07000402815D006DC1028B9
:1013F00009D020280AD0302816D10AE050280ED073
:10140000602811D10EE044F008040DE044F010040F
:101410000AE044F0200407E044F0400404E044F013
:10142000800401E044F480742868816921F070012F
:101430008161296804204860002C05D0686A204337
:1014400068622846FFF774FEBDE8F09F70B504009F
:1014500003D094F8200010B104E0012070BD2046B4
:1014600000F082F82068016841F00101016000F09D
:101470000BFD0546052604E000F006FD401B0A288A
:1014800011D820684068C007F6D02068016821F0B4
:101490000201016000F0F8FC05460BE000F0F4FCEE
:1014A000401B0A2806D9606A40F40030606284F864
:1014B0002060D2E7206840688007EFD4207E0128B2
:1014C000206801683DD021F080010160607E012824
:1014D0002068016838D021F040010160A07E012819
:1014E0002068016833D021F020010160E07E0128EE
:1014F000206801682ED041F010010160207F012892
:101500002068016829D021F008010160607F01286E
:101510002068016824D021F004010160D4E90201AF
:101520000843D4E90412114308436168491E084383
:101530002168C86100206062012084F8200000203A
:1015400070BD41F08001C0E741F04001C5E741F0C6
:101550002001CAE721F01001CFE741F00801D4E7EC
:1015600041F00401D9E7000070B586B00021434A7C
:10157000009101910291039111683F4E036802248A
:1015800003253F48491CB34231D11160012907D1DD
:10159000C16941F00071C161C16901F0007104913C
:1015A000816941F0040181618069364E00F00400D8
:1015B00004904FF4006000906946304600F06AFBEA
:1015C000B014CDE9000469460395304600F062FB93
:1015D00000220521142000F0C9FC142000F0B8FC02
:1015E00000220521152000F0C1FC15203FE0264E09
:1015F000B3423ED1C36943F08063C361C36901292B
:1016000003F080630493116007D1C16941F0007158
:10161000C161C16901F000710491816941F0080163
:1016200081618069194E00F008000490202000902C
:101630006946304600F02EFB4020CDE900046946A3
:101640000395304600F026FB1148416841F0E861FF
:10165000416000220521402000F088FC402000F07D
:1016600077FC00220521412000F080FC412000F0A1
:101670006FFC06B070BD0000006400400800002050
:10168000001002400008014000680040000C0140CA
:101690000000014010B5FFF745FB03280CD000EB1C
:1016A000800101EBC001054800EB8100C069002802
:1016B00002D0BDE81040004710BD00005C80002053
:1016C00010B5FFF72FFB03280CD000EB800101EBD6
:1016D000C001054800EB81008069002802D0BDE808
:1016E0001040004710BD00005C80002010B5FFF7DF
:1016F00019FB03280CD000EB800101EBC001054869
:1017000000EB8100406A002802D0BDE8104000478D
:1017100010BD00005C80002010B5FFF703FB03281C
:101720000CD000EB800101EBC001054800EB81000B
:10173000006A002802D0BDE81040004710BD00003C
:101740005C80002010B5FFF7EDFA03280CD000EB09
:10175000800101EBC001054800EB8100806A002890
:1017600002D0BDE81040004710BD00005C800020A2
:1017700070B5044690F82000012804D0606A40F457
:101780000020606218E0022084F8200020680168D0
:1017900021F00101016000F077FB05460EE000BF7B
:1017A00000F072FB401B0A2808D9606A40F4003040
:1017B0006062052084F82000012070BD2068406828
:1017C000C007EDD1606270BD10B5FFF7ABFA03281A
:1017D0000CD000EB800101EBC001054800EB81005B
:1017E000C068002802D0BDE81040004710BD0000CE
:1017F0005C80002010B5FFF795FA03280BD000EBB2
:10180000800101EBC001044850F82100002802D0FB
:10181000BDE81040004710BD5C80002010B5FFF708
:1018200081FA03280CD000EB800101EBC0010548D0
:1018300000EB81000069002802D0BDE8104000479D
:1018400010BD00005C80002010B5FFF76BFA032884
:101850000CD000EB800101EBC001054800EB8100DA
:101860004068002802D0BDE81040004710BD0000CD
:101870005C80002010B5FFF755FA03280CD000EB70
:10188000800101EBC001054800EB810040690028A0
:1018900002D0BDE81040004710BD00005C80002071
:1018A00010B5FFF73FFA03280CD000EB800101EBE5
:1018B000C001054800EB81008068002802D0BDE827
:1018C0001040004710BD00005C80002010B5FFF7FD
:1018D00029FA03280CD000EB800101EBC001054878
:1018E00000EB8100C06A002802D0BDE8104000472C
:1018F00010BD00005C8000202DE9F05FC16B0A681C
:1019000001680B68046C4FF0040808FA04F8844D71
:10191000844E854FDFF814C2DFF81492DFF814A26A
:10192000DFF814B2DFF814E218EA020F65D05FEABC
:10193000437862D50A68920603D40A6822F004024A
:101940000A60DFF8F0814FF48062016808F1140842
:1019500013011402414524D9A9420DD0B1420FD040
:10196000B9421AD0614515D0494515D0514501D12C
:10197000120312E0594501D104220EE0714501D154
:1019800040220AE06D4D1435A94206D06B4A283238
:10199000914201D11A4600E022466749091F0A60B8
:1019A00029E0A94213D0B14215D0B94220D06145F7
:1019B0001BD049451BD0514502D14FF4800217E09E
:1019C000414502D14FF0806212E0594501D1042215
:1019D0000EE0714501D140220AE0584D1435A9426C
:1019E00006D0564A2832914201D11A4600E02246DA
:1019F0004B4908394A60C16A71E04FF0020808FAA1
:101A000004F818EA020F70D05FEA83786DD50A688F
:101A1000920606D40A6822F00A020A60012180F8C0
:101A20002110DFF810814FF40072016808F11408EA
:101A300013011402414524D9A9420DD0B1420FD05F
:101A4000B9421AD0614515D0494515D0514501D14B
:101A5000120312E0594501D102220EE0714501D175
:101A600020220AE0354D1435A94206D0334A2832E7
:101A7000914201D11A4600E022462F49091F0A600F
:101A800029E0A94213D0B14215D0B94220D0614516
:101A90001BD049451BD0514502D14FF4001217E02D
:101AA000414502D14FF0007212E0594501D10222A6
:101AB0000EE0714501D120220AE0204D1435A942E3
:101AC00006D01E4A2832914201D11A4600E0224631
:101AD000134908394A60002180F82010816A0029E2
:101AE0001CD0BDE8F05F0847FFE70825A540154278
:101AF00014D01A0712D50A6822F00E020A6090F874
:101B00004020C36B012101FA02F25A60816380F820
:101B10002110002180F82010016BE0E7BDE8F09F64
:101B2000080002401C000240300002404400024015
:101B3000580002406C000240080402401C040240AD
:101B400030B560B11A4B026814219A4209D2194B80
:101B50001344B3FBF1F18900016417490AE0012045
:101B600030BD134B5B421344B3FBF1F189000164B8
:101B70000F490839C163022180F82110136843F628
:101B8000F0718B43F0E901142143D0E902452C4365
:101B90002143046921434469214384692143194352
:101BA000116000214163012242770177084630BD70
:101BB00008040240F8FFFDBF0000024070B5044673
:101BC00090F82000002501280CD0012084F8200086
:101BD00094F821600020012E06D084F82000022510
:101BE000284670BD022070BD022684F82160A063E3
:101BF0002068066826F0010606602046FFF774F9A3
:101C0000E06A00282068016802D041F00E0106E079
:101C100021F0040101602068016841F00A010160BF
:101C20002068016841F001010160D9E770B5044600
:101C300000F02AF90546601C02D0044800780444EC
:101C400000F022F9401BA042FAD370BD0C00002026
:101C50002DE9F0410024084F0646012505FA04F05D
:101C6000304203D057F8240000B18047641CE4B22E
:101C7000102CF3D3BDE8F0811C800020044910B57E
:101C80000A68024202D00860FFF7E2FF10BD0000C0
:101C9000140401402DE9F84FDFF8B8910024A9F1B0
:101CA000040B23460F2709F1040AABF1040EC9E027
:101CB0000125A5402A40AA427DD1674ED1F804C033
:101CC000ACEB0608B44532D014DCBCF1030F3AD0BB
:101CD00009DCBCF1000F2AD0BCF1010F1CD0BCF113
:101CE000020F31D11DE0BCF1110F17D0BCF1120F62
:101CF0002AD119E0B8F5881F19D006DCB8F5803F65
:101D000015D0B8F5801F1FD111E0B8F5001F0ED017
:101D1000B8F5041F18D10AE0CB6815E0CB681B1D8D
:101D200012E0CB6808330FE0CB680C330CE08B6813
:101D30002BB1012B4FF0080303D0456104E00423CD
:101D400002E0056100E00023FF2A01D8064601E019
:101D500000F104064FEA840501D9A5F12005D6F863
:101D6000008007FA05FC28EA0C0803FA05F548EAA2
:101D70000508C6F800804D68ED0062D5374DAE69A4
:101D800046F00106AE61AD6924F0030605F00105D9
:101D90000095334D06EB050CDCF80850A607360F0E
:101DA00007FA06F825EA0805DFF8B880404503D1B0
:101DB0004FF0000817E044E0DFF8AC80404502D166
:101DC0004FF001080FE0DFF8A480404502D14FF04A
:101DD000020808E0DFF89880404502D14FF0030880
:101DE00001E04FF0040808FA06F848EA0508CCF8C4
:101DF00008804D68D9F80060ED024D4601D51643C4
:101E000000E096432E604D68DAF80060AD0255465A
:101E100001D5164300E096432E604D68DBF8006064
:101E2000AD035D4601D5164300E096432E604D6834
:101E3000DEF80060ED03754601D5164300E09643D9
:101E40002E60641C0D682A46E5407FF431AFBDE882
:101E5000F88F00000804014000001110001002403B
:101E60000000014000080140000C0140001001404A
:101E7000001401408068084000D0012070470AB17A
:101E8000016170470904FBE7014880687047000062
:101E90000C0000200248816802781144816070477C
:101EA0000C000020074810B5016841F010010160E6
:101EB000032000F07BF80F2000F006F800F024F873
:101EC000002010BD0020024070B50D4D04464FF4B7
:101ED0007A712878B1FBF0F00A490968B1FBF0F09B
:101EE00000F026FD48B9102C07D200222146501ED2
:101EF00000F03CF800206C6070BD012070BD000057
:101F00000C000020180000200F4808B5816941F03E
:101F100001018161816901F001010091C16941F014
:101F20008051C161C069002200F0805000900F21F3
:101F3000901E00F01BF80548416821F0E06141F077
:101F40000071416008BD0000001002400000014027
:101F5000002809DB00F01F020121914040098000A8
:101F600000F1E020C0F8001170470000F0B40E4B03
:101F70001B680C46C3F30223C3F10705042D00D9E7
:101F80000425191D072901D2002300E0DB1E0126CC
:101F900006FA05F1491E214099409E40761E1640E2
:101FA0003143F0BC02F002B90CED00E0064900F04C
:101FB000070208684FF6FF03184040EA0220034A70
:101FC00010430860704700000CED00E00000FA05C7
:101FD0002DE9F0470F46050061D0434E306800F010
:101FE0000700B84209D2306820F00700384330605B
:101FF000306800F00700B84251D128683B4C810797
:1020000012D5400703D5606840F4E060606028782E
:10201000000703D5606840F4605060606068A9689C
:1020200020F0F000084360602878C00728D0686876
:10203000012810D02168022810D0890700292EDA43
:10204000616821F0030101436160FFF71DFF8046D5
:1020500041F288390DE021688903EFE78901EDE756
:10206000FFF712FFA0EB0801494502D90320BDE8A4
:10207000F0876068696800F00C00B0EB810FEFD169
:10208000306800F00700B8420BD9306820F0070034
:1020900038433060306800F00700B84201D00120BA
:1020A000E5E72878400705D56068E96820F4E06036
:1020B000084360602878000706D56068296920F425
:1020C000605040EAC100606000F038F86168084A7A
:1020D000C1F30311515CC840064908600648006816
:1020E000FFF7F2FE0020C2E700200240001002408D
:1020F00046AF0108180000201000002004480549E0
:1021000000684968044AC1F30221515CC840704725
:10211000180000200010024056AF0108044805498D
:1021200000684968044AC1F3C221515CC840704745
:10213000180000200010024056AF01082DE9F041C0
:102140001D494A681D4802F00C03042B2ED0082BB1
:102150002CD11B48C2F38343C45CD00328D5C86A82
:10216000174A00F00F000E32105CCA6AD20316D56F
:10217000CA6AC96AC2F30312C1F30321521C891C43
:10218000A2FB0023A1FB04150C4F0026A1FB070CAA
:1021900005FB07C501FB0651FEF712F903E00749ED
:1021A0006143B1FBF0F00D2C00D14008BDE8F08197
:1021B00004486043FAE700000010024000127A0071
:1021C00028AF010800093D002DE9F84F040070D048
:1021D0002078F14DC00749D06868C0F3810001281C
:1021E00007D06868C0F38100022809D16868C0037D
:1021F00006D52868800339D5A0680028E7D035E0E7
:10220000A068B0F5803F0BD010B1B0F5A02F11D071
:10221000286820F480302860286820F4802002E0BC
:10222000286840F480302860A06890B1FFF72CFE49
:1022300006460AE0286840F480202860F0E700BFE6
:10224000FFF722FE801B642876D828688003F7D524
:102250000CE0FFF719FE064605E000BFFFF714FE8D
:10226000801B6428F0D828688003F7D42078CB4EF0
:1022700080074FF001094FF000073AD5686810F069
:102280000C0F07D06868C0F38100022809D1686884
:10229000C00306D42868800715D56069012808D1D5
:1022A00011E06069B8B1C6F80090FFF7EDFD804617
:1022B00006E042E1FFF7E8FDA0EB08000228C3D8E2
:1022C00028688007F6D52868A16920F0F80040EA60
:1022D000C10028600DE03760FFF7D6FD804605E0BD
:1022E000FFF7D2FDA0EB08000228ADD828688007D0
:1022F000F6D4207800072ED5A948E169E9B1C0F8E5
:102300000090FFF7C1FD804606E000BFFFF7BCFD6F
:10231000A0EB0800022897D8686A8007F6D5A14884
:102320004FF4FA510068B0FBF1F0009000BF009844
:10233000411E0091FAD20EE0B0E00760FFF7A4FD65
:10234000804605E0FFF7A0FDA0EB0800022889D831
:10235000686A8007F6D42078400763D5E8694FF0B3
:102360000008C00009D4E86940F08050E861E869DD
:102370004FF0010800F0805000908B480168C905BB
:1023800012D40168834641F480710160FFF77CFD3F
:10239000824605E0FFF778FDA0EB0A0064287DD8AF
:1023A000DBF80000C005F5D5206901280AD008B186
:1023B000052813D0286A20F001002862286A20F03E
:1023C000040002E0286A40F001002862206941F21E
:1023D000883B98B1FFF758FD82460BE0286A40F031
:1023E00004002862EEE700BFFFF74EFDA0EB0A01F4
:1023F000594553D8286A8007F6D50CE0FFF744FD0D
:10240000824605E0FFF740FDA0EB0A01594545D89B
:10241000286A8007F6D4B8F1000F03D0E86920F0ED
:102420008050E861E06AD0B36968C90307D569687C
:10243000C1F38101022902D1E96AC9037DD40228CE
:1024400008D0E86A20F48030E862B766FFF71CFD28
:1024500080463BE02868C00005D5E86A616B00F063
:10246000F000884269D1B766FFF70EFD804605E0AF
:10247000FFF70AFDA0EB0800642874D82868000163
:10248000F6D4E86A616B20F0F0000843E862E86A7D
:10249000216B20F470600843E86201E063E018E01B
:1024A000C6F86890FFF7F0FC804605E0FFF7ECFC0B
:1024B000A0EB0800642856D828680001F6D508E08B
:1024C000FFF7E2FCA0EB080064284CD82868000164
:1024D000F6D4206A90B36968C1F38101022949D01A
:1024E0000228376603D0FFF7CFFC04463EE0FFF733
:1024F000CBFC074605E000BFFFF7C6FCC01B022867
:1025000031D828688001F7D4606AB0F5803F09D1DE
:10251000E86A61680843E862E86AE16820F00F0051
:102520000843E862D4E909010843696821F4741199
:1025300008436860C6F8609001E028E029E0FFF7F2
:10254000A3FC044605E000BFFFF79EFC001B022829
:1025500009D828688001F7D51BE000BFFFF794FC7D
:10256000001B022802D90320BDE8F88F28688001EB
:10257000F4D40EE00128F7D06868626A00F4803174
:10258000914204D1A16A00F47010884201D0012068
:10259000EAE70020E8E700000010024000004242A5
:1025A000800442421800002000700040704790F8FC
:1025B0005100704770B5040009D0606A002540B131
:1025C00025616561A56294F8510040B10CE00120DD
:1025D00070BD6068B0F5827FF4D0E561F2E784F801
:1025E0005050204600F040F8022084F85100206846
:1025F000016821F040010160A088218900F4827007
:1026000001F404410843A18901F400610843217CDD
:1026100001F002010843217D01F001010843218BF3
:1026200001F400710843217F01F03801084394F858
:10263000201001F080010843218D01F4005108436E
:1026400021680860A069042101EA104021684860FF
:102650002068C16921F40061C1616565012084F8C9
:102660005100002070BD000070B586B00025064600
:10267000009501950295039500681A4988422ED16C
:102680001949886940F480508861886900F4805055
:102690000490886940F0040088618869694600F008
:1026A00004000490A02000900220019003200390D9
:1026B0000E48FFF7EFFA0F4C0D4820601020C4E9D8
:1026C00001058020C4E903056561A5612046E56137
:1026D000FFF736FA08B1FEF728FCB464666206B06C
:1026E00070BD0000003001400010024000080140B1
:1026F00030000240840200202DE9F84F984616462B
:102700008A460446FFF7C0FB814694F85100012831
:102710001ED1BAF1000F73D0002E71D094F8500082
:10272000012815D0012784F85070032084F8510047
:1027300000256565C4F830A0A686E686A563A58752
:10274000E58765642564A068B0F5004F03D00CE010
:102750000220BDE8F88F2068016821F04001016087
:102760002068016841F480410160206801684906E1
:1027700003D4016841F040010160E068B0F5006FEA
:10278000606803D048B3012E27D047E008B1012E7E
:102790001FD1206B21680088C86006E0206881682E
:1027A000890709D5216B0988C160206B801C2063D3
:1027B000E08E401EE0860CE0FFF766FBA0EB09010F
:1027C000414503D3B8F1FF3F03D035E0B8F1000F26
:1027D00032D0E08E0028E1D123E0206B2168007820
:1027E000087306E02068816889070AD5216B09789B
:1027F0000173206B401C2063E08E401EE0860DE0DC
:102800002BE0FFF741FBA0EB0901414503D3B8F1F1
:10281000FF3F03D010E0B8F1000F0DD0E08E00288C
:10282000E0D14A464146204601F02AF808B120206E
:102830006065A06830B109E084F8517084F85050A8
:10284000032086E72068C1688068009084F8517092
:1028500004F8505F60680028F3D0012079E7000099
:1028600070B5044690F8510001281CD1C9B1C2B11D
:1028700094F85000012816D0012084F8500003205D
:1028800084F85100002565652163A286E286A56370
:1028900065642564A587E587A068B0F5004F04D07E
:1028A0000DE0012070BD022070BD2068016821F09C
:1028B000400101602068016841F480410160A16C21
:1028C0001748C862A16C17488862A16C1648086353
:1028D000A06C4563E38E2268216B0C32A06CFFF77D
:1028E0006DF930B1606D40F01000606584F85050B3
:1028F000D7E720680168490603D4016841F0400128
:10290000016084F850502068416841F02001416026
:102910002068416841F002014160002070BD000064
:10292000133800081D380008F13700087047704759
:1029300010B5401EB0F1807F01D3012010BD4FF0D3
:10294000E02460610F21601701F030FC0020A061DD
:1029500007202061002010BD7047704770B590F8C7
:102960003C20012A29D0012480F83C40022280F832
:102970003D2003685A689D6822F070060A68324359
:102980005A600F4B02689A420BD0B2F1804F08D0C8
:102990000C4B9A4205D00C4B9A4202D00B4B9A42F8
:1029A00004D1496825F080031943916080F83D40C7
:1029B000002180F83C10084670BD022070BD000068
:1029C000002C01400004004000080040000C0040C2
:1029D00010B5040003D094F83D0010B107E00120C9
:1029E00010BD002084F83C00204600F01FF80220B3
:1029F00084F83D00211D206801F008F8012084F8CA
:102A0000460084F83E0084F83F0084F8400084F8D3
:102A1000410084F8420084F8430084F8440084F8BC
:102A2000450084F83D00002010BD000008B5006896
:102A30000B49884212D10B48C16941F01001C161B4
:102A4000C069002200F01000009005213620FFF739
:102A50008DFABDE808403620FFF77ABA08BD0000BD
:102A6000001000400010024090F83D10012901D0F4
:102A700001207047022180F83D100168CA6842F0C9
:102A80000102CA6000680D4988420BD0B0F1804F46
:102A900008D00B49884205D00A49884202D00A4929
:102AA000884204D1816801F00701062903D001683A
:102AB00041F001010160002070470000002C01403E
:102AC0000004004000080040000C004070472DE961
:102AD000F04104460068C66805694FF00007A90781
:102AE00013D5B10711D5F91E0161012020772068A7
:102AF00080698007204602D0FFF7E8FF04E000F07D
:102B0000B1F8204600F056F92777680716D5700708
:102B100014D521686FF00400086102202077206836
:102B2000806910F4407F204602D0FFF7CFFF04E019
:102B300000F098F8204600F03DF92777280715D5D2
:102B4000300713D521686FF0080008610420207752
:102B50002068C0698007204602D0FFF7B7FF04E075
:102B600000F080F8204600F025F92777E80616D512
:102B7000F00614D521686FF0100008610820207756
:102B80002068C06910F4407F204602D0FFF79EFF06
:102B900004E000F067F8204600F00CF92777E8071A
:102BA00008D0F00706D021686FF0010008612046C8
:102BB00000F08EF9280608D5300606D521686FF09A
:102BC000800008612046FFF7C7FE680608D570063A
:102BD00006D521686FF040000861204600F082F9B8
:102BE000A8060AD5B00608D521686FF02000086154
:102BF0002046BDE8F041FFF7B0BEBDE8F08100001F
:102C000000B585B000210091019102910391006807
:102C1000104988421BD11048816941F0100181613F
:102C20008069694600F0100004904FF470700090C5
:102C30000220019003900948FFF72CF808484168EA
:102C400021F4406141F0E06141F44061416005B030
:102C500000BD0000000400400010024000100140D0
:102C600000000140704770B5044690F83C00002613
:102C70000D4601280FD0012084F83C006AB1042AD7
:102C80001DD0082A2FD00C2A3FD00126002084F81E
:102C90003C00304670BD022070BD206800F008FF87
:102CA0002068816941F0080181612068816921F013
:102CB00004018161206881692A69114311E020685B
:102CC00000F01EFF2068816941F400618161206885
:102CD000816921F480618161206881692A6941EA02
:102CE00002218161D2E7206800F036FF2068C169C7
:102CF00041F00801C1612068C16921F00401C1618E
:102D00002068C1692A69114311E0206800F050FF72
:102D10002068C16941F40061C1612068C16921F482
:102D20008061C1612068C1692A6941EA0221C161EB
:102D3000ACE710B5040003D094F83D0010B107E0F3
:102D4000012010BD002084F83C00204600F01EF851
:102D5000022084F83D00211D206800F057FE01206C
:102D600084F8460084F83E0084F83F0084F8400070
:102D700084F8410084F8420084F8430084F8440059
:102D800084F8450084F83D00002010BD08B50068B7
:102D90000649884208D10648C16941F00201C16173
:102DA000C06900F00200009008BD0000000400406F
:102DB000001002407047000010B50446022249B1DD
:102DC00004290ED0082913D094F84100012816D008
:102DD000012010BD94F83E000128F9D184F83E206E
:102DE0000FE094F83F000128F2D184F83F2008E07A
:102DF00094F840000128EBD184F8402001E084F8E9
:102E000041200122206800F045FE114920688842D7
:102E100003D1426C42F400424264206888420BD0E5
:102E2000B0F1804F08D00B49884205D00A4988424A
:102E300002D00A49884204D1816801F007010629BD
:102E400003D0016841F001010160002010BD0000C5
:102E5000002C01400004004000080040000C00402D
:102E600030B504460D460068002200F013FE174BF3
:102E700041F2111120688A10984209D1036A0B426D
:102E800006D1036A134203D1436C23F40043436425
:102E90002068036A0B4206D1016A114203D101681E
:102EA00021F00101016001203DB1042D08D0082D61
:102EB00009D084F84100002030BD84F83E00FAE7D4
:102EC00084F83F00F7E784F84000F4E7002C014065
:102ED00000680349884202D1012013F0E7B9704726
:102EE00000100040704770B5040004D094F8410011
:102EF000002510B106E0012070BD84F84050204646
:102F000000F024F8242084F841002068C16821F4EE
:102F10000051C160204601F0B3F82068016921F436
:102F2000904101612068416921F02A0141612068D6
:102F3000C16841F40051C1606564202084F84100FB
:102F400084F842006563002070BD00002DE9F04167
:102F500086B0002400940194029403940646484DE0
:102F6000036848480221032280274FF01008AB4233
:102F700045D1C36943F40033C361C36903F400332B
:102F80000493836943F00403836180693E4D00F03C
:102F9000040004900420CDE900010392694628460C
:102FA000FEF778FE0820CDE9000469462846029421
:102FB000FEF770FE364D3548C5E90004C5E9024705
:102FC0002C616C61AC612846EC61FEF7B9FD08B17B
:102FD000FDF7ABFFF5632D486E622D4D143044357F
:102FE000C5E902472C616C61AC61EC61C5E9000880
:102FF00028463EE0B5636E6206B0BDE8F081254D1F
:10300000AB42F9D1C36943F48023C361C36903F4BC
:1030100080230493836943F01003836180690392E2
:1030200000F0100004902815CDE900011A4D694602
:103030002846FEF72FFEE814CDE90004694628462D
:103040000294FEF727FE1548416821F0300141F057
:10305000E06141F0100141600D4D0C488835503859
:10306000C5E902472C616C61AC61EC61C5E90008FF
:103070002846FEF765FD0028BCD0FDF756FFB9E7EE
:103080000044004000100240000801406C00024073
:10309000E80300200048004000100140000001400B
:1030A0002DE9F843044690F84100984616460D462F
:1030B000202802D00220BDE8F88385B17EB100202F
:1030C0006064212084F84100FEF7DEFEA68481467C
:1030D000E684A0682027B0F5805F02D003E00120DD
:1030E000E9E7206910B12E4600250EE000260CE02D
:1030F0008021204601F020F8A8B9C6B116F8010BCE
:1031000021684860E08C401EE084E08C4B464FF024
:103110000002CDF800800028EAD14FF0400120469F
:1031200001F00AF840B184F841700320C3E735F894
:10313000020BC0F30800E3E784F841700020BAE70F
:10314000FEE72DE9F041070AC6B20021F0238722ED
:10315000084600F0CDF84FF487700446FDF7DAF822
:10316000050013D0002029182F54801C4E70A04257
:10317000F9D300262146284600F054F9761CF02E9B
:10318000F8D32846BDE8F041FDF7F3B8BDE8F0817B
:1031900038B5144602460846C2F1EF01012389B250
:1031A0001A4600F0A5F8200A8DF800008DF80140BD
:1031B0000221684600F00EF938BD000010B5414C00
:1031C0008AB0002210212046FEF759FE3220FEF779
:1031D0002DFD012210212046FEF751FE3220FEF780
:1031E00025FD362000F0B6F8602000F0D3F83A2034
:1031F00000F0B0F8052000F0CDF8B22000F0AAF8F9
:1032000031A1D1E90001CDE90801052108A800F0AC
:10321000E1F8B72000F09EF8352000F0BBF8BB20A5
:1032200000F098F8192000F0B5F8C02000F092F8EE
:103230002C2000F0AFF8C22000F08CF8012000F044
:10324000A9F8C32000F086F8122000F0A3F8C420EB
:1032500000F080F8202000F09DF8C62000F07AF8F9
:103260000F2000F097F8D02000F074F8A42000F0B0
:1032700091F8A12000F08EF8E02000F06BF814A087
:103280000FC88DE80F000E21684600F0A3F8E1207A
:1032900000F060F812A104AC0FC984E80F000E2101
:1032A00004A800F097F8212000F054F8112000F055
:1032B00051F87820FEF7BAFC292000F04BF80AB04C
:1032C00010BD0000001001400C0C00333300000062
:1032D000D0040D11132B3F544C180D0B1F2300006D
:1032E000D0040C11132C3F44512F1F1F202300002A
:1032F0002DE9FC4100F1340401F12807A518FE185E
:103300002A206D1E761E00F025F8200A8DF8000098
:103310008DF80140280A8DF802008DF80350042131
:10332000684600F057F82B2000F014F8380A8DF8A2
:1033300004008DF80570300A8DF806008DF80760DE
:10334000042101A800F046F82C2000F003F8BDE8A5
:10335000FC81000031B5002220210B48FEF78FFDD3
:103360000A4C002210212046FEF789FD4FF0FF3362
:10337000012269460648FFF7BFF9012210212046C5
:10338000FEF77DFD38BD000000100140000801403F
:103390002C02002031B5012220210B48FEF76FFDE1
:1033A0000A4C002210212046FEF769FD4FF0FF3342
:1033B000012269460648FFF79FF9012210212046A5
:1033C000FEF75DFD38BD000000100140000801401F
:1033D0002C02002070B50C460546402903D9BDE8F3
:1033E000704000F01FB8012220210B48FEF747FD76
:1033F0000A4E002210213046FEF741FD4FF0FF3308
:10340000224629460648FFF777F93046BDE8704066
:1034100001221021FEF733BD0010014000080140D9
:103420002C02002070B50C460546012220210D48D3
:10343000FEF725FD0C4E002210213046FEF71FFD41
:10344000224629460948FFF70BFA0848FFF7AFF86C
:103450000128FAD13046BDE8704001221021FEF764
:103460000EBD000000100140000801402C020020A9
:103470000E4810B50C4901600921416000214FF44C
:1034800080328160C0E90312416101764176817624
:10349000C17601774177FDF7D9FF002803D0BDE859
:1034A0001040FDF742BD10BD00640040DC0100206B
:1034B0000E4810B50C4901600921416000214FF40C
:1034C00080328160C0E903124161017641768176E4
:1034D000C17601774177FDF7B9FF002803D0BDE839
:1034E0001040FDF722BD10BD00680040040200201E
:1034F000154808B5416941F0010141614069002268
:1035000000F00100009005210C20FEF72FFD0C209B
:10351000FEF71EFD002205210D20FEF727FD0D20E0
:10352000FEF716FD002205211020FEF71FFD1020DA
:10353000FEF70EFD002205211120FEF717FDBDE864
:1035400008401120FEF704BD0010024010B5074AE4
:103550000021074813F0FAFE064C074A002160607C
:10356000064813F0F3FE206010BD000004AF010810
:103570006D390008000000200CE90108B13E000888
:103580002DE9F04186B000242D4800940194029466
:103590000394816941F020018161816901F020017A
:1035A0000491816941F004018161816901F00401A4
:1035B0000491816941F010018161816901F010017C
:1035C0000491816941F0080181618069DFF87480AC
:1035D00000F008000490002250214046FEF74FFC06
:1035E000194F002230213846FEF749FC50200125B2
:1035F0000226CDE90005CDE9024669464046FEF7C0
:1036000049FB3020CDE90005CDE902466946384640
:10361000FEF740FB4FF4407000900C48CDE90104E8
:1036200069464046FEF736FB002205211720FEF7CB
:103630009DFC1720FEF78CFC06B0BDE8F081000071
:10364000001002400008014000100140000031104D
:10365000104810B50E4901604FF48271416000219D
:103660008160C1604FF400720161C0E90512082257
:10367000C0E90721416281620A21C162FEF79AFF17
:10368000002803D0BDE81040FDF74FBC10BD00007E
:10369000003001402C02002010B58AB000240794AD
:1036A0001C2168460894FDF771F822482049C0E9BA
:1036B00000144FF6FF71C0E9024104618461FFF715
:1036C00038FB08B1FDF731FC079407A919480894A5
:1036D000FFF744F908B1FDF728FC6020CDE90004AC
:1036E00002940022694613480494FFF7BCFA08B11B
:1036F000FDF71BFC042269460E48FFF7B4FA08B137
:10370000FDF713FC082269460A48FFF7ACFA08B136
:10371000FDF70BFC0C2269460648FFF7A4FA08B136
:10372000FDF703FC0348FFF76BFA0AB010BD000079
:1037300000040040C80200201CB500240E4800947C
:103740000C49019401604721C0E9011440F2E731BE
:103750008461C160FFF73CF908B1FDF7E6FB009416
:10376000694605480194FFF7F9F8002801D0FDF7F4
:10377000DCFB1CBD00100040100300200C4810B5FD
:103780000A4901604FF4E1314160002181600C225F
:10379000C160C0E904128161C161FFF7A4FB002888
:1037A00003D0BDE81040FDF7C0BB10BD0044004091
:1037B000580300200C4810B50A4901604FF4E1316C
:1037C0004160002181600C22C160C0E90412816166
:1037D000C161FFF788FB002803D0BDE81040FDF76A
:1037E000A4BB10BD00480040A0030020FEE7FEE798
:1037F00010B5406A01684A6822F003024A60416DD0
:1038000041F010014165012180F85110FEF7CEFE14
:1038100010BD10B5406AFFF78AF810BD38B50546EF
:10382000446AFEF731FB024628680068800623D40C
:103830002068416821F0200141602068416821F042
:10384000020141606421204600F01AF818B1606D51
:1038500040F020006065A068002118B92068C268A7
:1038600080680090E186012084F85100606D18B1F5
:103870002046FEF79BFE38BD2046FFF757F838BDBF
:10388000F8B515460E460B46009204460122022169
:1038900000F010F840B93346002280212046009500
:1038A00000F008F8002804D0606D40F0200060654A
:1038B0000320F8BD2DE9F8431E469146884604468C
:1038C000089DFEF7E1FA401B351AFEF7DDFA0746C0
:1038D00025480068C0F3CB30684338E0701C37D00F
:1038E000FEF7D2FAC01BA84203D215B1009860B30C
:1038F0002CE02068416821F0E00141606068B0F58B
:10390000827F0BD1A068B0F5004F02D0B0F5806F78
:1039100004D12068016821F040010160A06AB0F57F
:10392000005F09D12068016821F40051016020681E
:10393000016841F400510160012084F85100002029
:1039400084F850000320BDE8F8830025401E009055
:103950002068816838EA010004D000214945BDD1C2
:103960000020F0E70121F9E71800002010B513F05E
:10397000EAFCBDE8104013F02EBD10B5FEF78AFA40
:1039800016F03EFF012803D0BDE8104016F0F8BB4A
:1039900010BD000070B594B038216846FCF7F6FE03
:1039A00014210EA8FCF7F2FE012500242804CDE91D
:1039B00002040226CDE908600095059501944FF4B4
:1039C000E010CDE90A046846FEF7FEFB08B172B6C6
:1039D000FEE70F20CDE90E064FF48060CDE91040E0
:1039E00002210EA81294FEF7F3FA08B172B6FEE7B0
:1039F0000148056714B070BD0000424270470000E6
:103A00000148FFF764B8000010030020F0B5026819
:103A10001C4B1D4C1D4D1E4E4FF08047984207D049
:103A2000B84205D0A04203D0A84201D0B04204D190
:103A300022F0700C4A6842EA0C02984207D0B84261
:103A400005D0A04203D0A84201D0B04203D122F455
:103A50004074CA6822434C6922F08002224302600B
:103A60008A68C2620A688262984201D10969016368
:103A7000012141610169C90703D0016921F00101F8
:103A80000161F0BD002C014000040040000800402E
:103A9000000C004010B501F01F030121046A994099
:103AA0008C430462016A9A401143016210BD000018
:103AB00030B5036A026A22F0010202624268846938
:103AC00024F073050C682C4323F002058B682B430C
:103AD0000A4DA8420BD123F00805CB6822F44072AE
:103AE0002B434D6923F0040315438A692A4342603E
:103AF000846149684163036230BD0000002C0140CD
:103B000030B5026A036A23F01003036243688469D4
:103B10000D6824F4E64444EA05248D6822F020026E
:103B200042EA05120B4DA8420ED1CD6822F0800268
:103B300042EA05124D6923F4406343EA85038D6927
:103B400022F0400243EA850343608461496881634F
:103B5000026230BD002C014030B5036A026A22F4D3
:103B6000807202624268C46923F4007324F0730512
:103B70000C682C438D6843EA05230C4DA8420ED1F6
:103B8000CD6823F4006343EA05234D6922F44052D3
:103B900042EA05128D6923F4806342EA051242600D
:103BA000C4614968C163036230BD0000002C01405C
:103BB00030B5046A026A22F4805202624268C36924
:103BC0000D6823F4E64343EA05238D6824F400548A
:103BD00044EA0534064DA84204D14D6922F48042DE
:103BE00042EA85124260C36149680164046230BDE3
:103BF000002C014013F09FFA6421B0FBF1F613F0A2
:103C000093FA044617491848FDF79EF8164F3444B6
:103C100004E0154914483831FDF724F9124900230E
:103C20001A463831786B13F0EBFA0028F1D00F4DBB
:103C3000686913F077FB00231A460B49686913F093
:103C40003DFBA86913F06EFB00231A460649A869DC
:103C500013F034FB0448FDF7DBF8204613F04DFA6F
:103C6000D5E70000D80100202C810020C081002071
:103C70001FB513F060FA064613F056FA0446FFF734
:103C80009DFA0DF0B3FC11F07DFE11F09BFE4FF696
:103C9000FF70FFF756FA6248FEF7E6FE11F048FFA4
:103CA00009F0A0FB05465022AA2111F0BEFB142208
:103CB0003C21284611F0D8FB28460DF0F9FC0023E2
:103CC00005461A4609210EF075FC56A128460EF04D
:103CD00071F911F02DFF09F085FB05466E22AA212E
:103CE00011F0A3FB14223C21284611F0BDFB28460D
:103CF0000DF0DEFC002305461A4609210EF05AFCA1
:103D00004AA128460EF056F911F012FF0DF0D0FC32
:103D10000A228346114611F088FB45A158460EF051
:103D200049F911F005FF0DF0C3FC82460A22782103
:103D300011F07BFB41A150460EF03CF911F0F8FE6A
:103D40000DF0B6FC814628220A2111F06EFB3EA13F
:103D500048460EF02FF911F0EBFE0DF0A9FC80465D
:103D60002822782111F061FB3AA140460EF022F999
:103D700011F0DEFE0DF09CFC05465F220A2111F0D9
:103D800054FB37A128460EF015F911F0D1FE0DF0C5
:103D90008FFC054672220A2111F047FB33A1284609
:103DA0000EF008F9344F344412F0BCFA64230022B8
:103DB0003249786913F024FA00282CD113F0D0F995
:103DC0002E4D2FA21021AB8C6846FCF771FB694683
:103DD00058460EF0EFF8EB8C2CA210216846FCF749
:103DE00067FB694650460EF0E5F82B8D2AA210219C
:103DF0006846FCF75DFB694648460EF0DBF86B8DC4
:103E000028A210216846FCF753FB694640460EF095
:103E1000D1F813F0D7F9204613F06FF9C3E700008B
:103E2000100300204E455854000000004F4B000086
:103E30005369636B313A2030000000005369636BB3
:103E4000323A2030000000005369636B333A20306F
:103E5000000000005369636B343A2030000000001A
:103E60004D696E695F63726F650000004279205290
:103E70006F626F6669736800C08100200C82002049
:103E80005369636B313A2025640000005369636B0A
:103E9000323A2025640000005369636B333A2025D1
:103EA000640000005369636B343A2025640000000D
:103EB00010B513F055F9164A0021164813F046FACA
:103EC000154C164A00216060154813F03FFA206037
:103ED000144A0021144813F039FAE060134A002113
:103EE000134813F033FAA06000223821022013F0A7
:103EF000B9F9606100223821022013F0B3F9A06102
:103F000013F060F913F01FFABDE8104013F063BA24
:103F100054E90108713C0008C081002030E9010823
:103F2000F53B000878E90108353F00089CE90108E5
:103F3000D53F000813F0FFF8054613F0F5F800220E
:103F4000044611461046FCF759FE00221146022095
:103F5000FCF754FE19491A48FCF7FEFDFCF716FE63
:103F60004FF496763046FDF761FE4FF07C500146E7
:103F7000FCF7F2FD3046FDF759FE12491248FCF7F6
:103F8000EBFD3046FDF752FEFCF70CFE0F4E2C44C5
:103F9000306B042808D113F0D6F913F01CFA002274
:103FA00011460B4813F0D2F9002202210120FCF740
:103FB00025FE204613F0A1F8E9E700009A99993E02
:103FC000CDCCCC3D3333333F6666663F2C81002039
:103FD000F53B000813F0AFF86421B0FBF1F513F0E6
:103FE000A3F80F4FDFF83C8004464FF0FF360D4931
:103FF00000232C441A462439786913F001F958B982
:104000003346082241460848FFF74AF8334608225B
:1040100041460648FFF744F8204613F06EF8E6E7FD
:10402000C0810020AC810020A003002058030020A4
:1040300001680C3151E8002F22F4907241E800230E
:10404000002BF5D10168143151E8002F22F0010254
:1040500041E80023002BF5D1016B012909D101684A
:104060000C3151E8002F22F0100241E80023002B10
:10407000F5D1202180F84210002101637047000033
:1040800070B5044600680169E26821F440511143AB
:1040900001612169A0680843616908432168CA6811
:1040A00041F20C639A430243CA6020684169A269E5
:1040B00021F44071114341611E492068884202D1B8
:1040C000FEF72CF801E0FEF719F800EBC00101EB58
:1040D0000012606864218000B2FBF0F3B3FBF1F3DF
:1040E0006FF018067343B2FBF0F5B2FBF0F605EB88
:1040F0008305322303EB0515B5FBF1F5B6FBF1F6AD
:1041000005F0F00505EB0615B2FBF0F6B2FBF0F09A
:10411000B0FBF1F06FF01802504306EB800003EBA8
:104120000010B0FBF1F0216800F00F002844886017
:1041300070BD0000003801402DE9F843984617464D
:104140000D460446089E24E0701C22D0FDF79CFE1C
:10415000A0EB0800B0421AD8CEB12068C168490768
:1041600017D5802D15D0402D13D00168C9430907FC
:104170000FD401680025406800902046FFF758FFE3
:104180000820606484F840500120BDE8F8830320D3
:10419000FBE72068006835EA000004D00020B84240
:1041A000D2D00020F1E70120F9E7FEE70907090E68
:1041B000002804DB00F1E02080F80014704700F0D4
:1041C0000F0000F1E02080F8141D704710B5442165
:1041D000074800F082FE00221E21064812F070F807
:1041E000054CA06001F0B6FA0020207010BD000060
:1041F0000453002009580008480100202DE9F04729
:104200000E46814617461146304600F011F9002847
:104210007ED000223946304600F0B6F800284FF034
:10422000000076D1B6F904C0B6F90030F288ACEBE4
:1042300003010FFA81FAB6F90210B7F80280521A98
:10424000A8EB01080FFA88F812B2B8F1000F0EDDE2
:1042500063F30F046CF30F0501EB080061F31F44D7
:1042600060F31F45C9F800400120C9F80450B7F9B0
:1042700006107388CB1AD21A12B2002A13DDB6F9CF
:10428000063099420FDA338863F30F04B38861F381
:104290001F4463F30F05114461F31F4509EBC0018F
:1042A000401C0C604D60B7F90220B6F902108A423A
:1042B00000DD1146B7F90630B6F90620934200DA60
:1042C0001A463B88B6F900C0521AA3EB0C031BB286
:1042D00012B2002B10DD002A0EDD634463F30F05DC
:1042E0008B1863F31F456CF30F0409EBC00361F3F4
:1042F0001F441C605D60401CB7F904703388FE1ACF
:10430000AAEB06031BB2002B11DD67F30F0401E0DB
:104310000FE00CE061F31F443B4463F30F051144CD
:1043200061F31F4509EBC001401C0C604D60BDE806
:10433000F0874FF0FF30FAE770B5B1F90030B2F90D
:104340000040A34200DC23460380B1F90250B2F9D9
:104350000240A54200DD2C464480B1F90460B2F968
:104360000450AE4200DA35468580B1F90610B2F944
:104370000620914200DB1146C1800120AB4201DCE6
:104380008C4200DD002070BDF8B50D460446B0F942
:104390000000B1F900101646884247DBB4F902105C
:1043A000B5F90220914241DBB4F90410B5F90420BB
:1043B00091423BDCB4F90610B5F90620914235DC98
:1043C00096B3ADF800006088ADF802003246694649
:1043D000284600F099F8002827D0A088ADF8000002
:1043E0006088ADF8020032466946284600F08CF835
:1043F00000281AD02088ADF80000E088ADF802004F
:1044000032466946284600F07FF800280DD0A08883
:10441000ADF80000E088ADF8020032466946284653
:1044200000F072F8002800D00120F8BD0020F8BD8F
:10443000B0F90020B1F904309A4213DCB0F904203D
:10444000B1F900309A420DDBB0F90220B1F9063023
:104450009A4207DCB0F90600B1F90210884201DB8C
:104460000120704700207047F8B50D460446B0F9AA
:104470000400B1F900101646884243DBB4F9060087
:10448000B5F9021088423DDBB4F90000B5F904101B
:10449000884237DCB4F90210B5F90620914231DCCC
:1044A00076B3ADF800006088ADF802003246694688
:1044B000284600F029F818BBA088ADF800006088F5
:1044C000ADF8020032466946284600F01DF8B8B93A
:1044D0002088ADF80000E088ADF802003246694659
:1044E000284600F011F858B9A088ADF80000E0881F
:1044F000ADF8020032466946284600F005F808B1DA
:104500000020F8BD0120F8BD2DE9FC4114460E46FF
:10451000B1F90020B0F9001005468A423ADBB5F93E
:104520000400824236DCB6F90270B5F902209742E7
:1045300030DBB5F906309F422CDC002C75DD401ACB
:104540009A1A401C521C00B212B200EBD07002EB5F
:10455000D27240105210904200DB1046844200DDBF
:104560000446ADF80010288800222044ADF804006D
:104570006888ADF80200688831462044ADF806002E
:104580006846FFF7C1FF40B1BDF804002044ADF814
:1045900004003FE00020BDE8FC81E8880022001B09
:1045A000ADF80200E888ADF8060031466846FFF72E
:1045B000ABFF28B1BDF804002044ADF8040011E0C1
:1045C000A8880022001BADF80000A888ADF8040000
:1045D00031466846FFF798FF50B1BDF80000001B58
:1045E000ADF80000BDF80200001BADF8020016E0B7
:1045F0006888ADF80200688800222044ADF8060003
:1046000031466846FFF780FF70B1BDF80000001B1F
:10461000ADF80000BDF806002044ADF806003146B4
:10462000684611F091F9B6E7FFE70120B3E710B54E
:10463000B1F90040B2F900309C4200DA2346038011
:10464000B1F90240B2F902309C4200DA23464380BD
:10465000B1F90440B2F904309C4200DD2346838066
:10466000B1F90610B2F90620914200DC1146C18072
:1046700010BD0000F8B5074611F00EFE0025374CBE
:104680000646009537B1F8686060384611F0E6FEDE
:10469000606802E009F0C0F96060006911F058F844
:1046A0006068406908B111F053F86068C06911F0A2
:1046B0004FF86068006A11F04BF86068016991B1C9
:1046C00011F0D6F913F048FE13F09CFC6068B0F8C6
:1046D0005011D9B30068017CC9071DD0C06840687B
:1046E000D0B1002713E0A0F85051F8BDC11991F8DE
:1046F000301151B900F5AC7000F046FC616801EB77
:10470000C7010A6B0260496B41607F1CBFB26068E1
:10471000B0F85011B942E9D860684FF48071303078
:104720000DF048FE6068202100F598700DF042FE03
:104730006068A0F85051304611F0A7FD0090606805
:104740000068436A13B12268009998470DF0BCFCD9
:1047500000F032F8BDE8F84000F002B8C8000020D0
:1047600070B50A4D002400BFC4EBC40655F82600FE
:1047700008B10DF01DFD05EB86001C210DF01AFEA1
:10478000641CE4B2042CEFD370BD0000E0530020A1
:10479000084949680AE04A68824202D00A688242AF
:1047A00003D10A7E42F001020A7649690029F2D15A
:1047B000704700009C000020704700000421014861
:1047C00000F08BBBF85200202021014800F085BB8F
:1047D000105300202DE9FF410446DDE90A671D0062
:1047E0004FF0000002D1B6F5807F2BD003900190EE
:1047F0000290ADF80C100090ADF80410ADF80A204E
:10480000ADF80E203B4632462946684610F0FCFFC4
:104810003B463246294601A810F0F6FF3B46324699
:10482000294602A810F0F0FF3B463246294603A86D
:1048300010F0EAFFBDF90000BDF90430984209DA32
:10484000054608E02080491E6080A180521EE2805B
:10485000BDE8FF811D46BDF90820BDF90C108A4254
:1048600001DA164600E00E46B54203DA984206DB4E
:10487000184604E08A4201DA104600E00846801E2D
:104880002080BDF90030BDF90420934201DD1D46B2
:1048900000E01546BDF90800BDF90C10884201DDA5
:1048A000064600E00E46B54205DD934201DD19469D
:1048B00004E0114602E0884200DD0146891CA18027
:1048C000BDF90230BDF90620934201DA1D4600E031
:1048D0001546BDF90A00BDF90E10884201DA0646F8
:1048E00000E00E46B54205DA934201DA194604E0CB
:1048F000114602E0884200DA0146891E6180BDF956
:104900000230BDF90620934201DD1D4600E0154648
:10491000BDF90A00BDF90E10884201DD064600E02F
:104920000E46B54205DD934201DD194604E011460D
:1049300002E0884200DD0146891CE18088E7000032
:104940002DE9F04115460E460746114C11F0A4FC26
:1049500080462B463246394620460CF0C1FC20B139
:104960000020A062E06950B110E02C2120460DF03B
:1049700021FD4FF00040A0620020BDE8F0814046DC
:1049800011F083FCE06108B90120E0612046F4E702
:104990003453002010B51421074800F09EFA0CF0A3
:1049A00065FC40B1054901600549416005498160E8
:1049B0000549C16010BDFEE71C530020450C0108ED
:1049C000C10F01088D110108130C010870B50D46C7
:1049D0000446102128460DF0EDFC206800780128DF
:1049E00004D0022807D0042807D008E0A08A288035
:1049F000E08A688003E0E06800E00A2068602068E0
:104A00004268002A03D02946BDE87040104770BDB7
:104A10002DE9FE430446808A10B9E08A002873D04D
:104A2000D4F82C805FEA080010D1204605F085FFFD
:104A30005FEA000868D0204607F05CFE00220921EA
:104A400040460BF08DFB607880075DD44FF4807991
:104A500000274E464546002128460FF0AEFA38445E
:104A600007B2002128460FF0BAFAC11700EB116017
:104A70000012704306B228460EF05AFC0500EAD137
:104A80000FB94E450CD0784201B24FF4803090FB04
:104A9000F6F002B26B4604F11400009510F0B4FE7B
:104AA000ADF80450ADF8085094F8400000F00F0045
:104AB0000328404616D00EF06DFD064640460EF027
:104AC00043FC03460C200090B4F9161032464046D1
:104AD00005F02AFBADF8080040460EF087FCC10740
:104AE00013D018E00EF0EAFC064640460EF086FCB5
:104AF000024603200090B4F914103346404605F0F6
:104B000013FBADF80400E7E736E0BDF90410002917
:104B100001DDADF80450810705D4BDF9041000296A
:104B200001DAADF80450410705D4BDF90810002999
:104B300001DDADF80850000705D4BDF908000028D4
:104B400001DAADF8085002AA01A9204613F094FE3C
:104B5000BDF90820BDF90410404600F07CFA6078E9
:104B6000800709D4208BBDF8041008442083608B93
:104B7000BDF8081008446083BDE8FE832DE9FC5FA2
:104B80000446C06A5FEA000B71D094F84000000749
:104B90006DD00CF05FFC019000684021457E5846C6
:104BA0000FF000FB4FF0000818B9A4F81E80A4F81D
:104BB0001C8058460EF0E0FC824658460EF0E3FC9E
:104BC000064694F840004FF0640900F00F000C28EE
:104BD00002D003284CD09AE0A4F81C8056B1B4F956
:104BE0001E5000270CF036FC0068407EC0F16401C6
:104BF000484622E0B4F91E00C5F16401484390FB29
:104C0000F9F0E08358460EF09FFB054658460EF03B
:104C1000C1FC02460C200090B4F91E102B465846E9
:104C200005F082FAE083024600231EE07A1917B2EB
:104C300001FB05F292FBF0F215B2002DF6D1ADF8B2
:104C40000070A4F81E806A460021204613F014FE6E
:104C500041F6FF72BDF900305142584606F004F8A3
:104C6000BDF800100123084402B200214CE09AE094
:104C7000A4F81E80BAF1000F0AD0B4F91C50002726
:104C80000CF0E8FB00684946407EC0F1640022E079
:104C9000B4F91C00C5F16401484390FBF9F0A0830E
:104CA00058460EF0ABFB054658460EF007FC03468F
:104CB00003200090B4F91C102A46584605F034FA37
:104CC000A083014600231EE07A1917B200FB05F20B
:104CD00092FBF1F215B2002DF6D1ADF80070A4F8F8
:104CE0001C8000226946204613F0C6FD41F6FF7283
:104CF000BDF900305142584605F02EFFBDF80010B6
:104D00000123084401B20022584610F0EBF9A08BB1
:104D1000002848D1E08B002845D1C6B958460EF08E
:104D200039FC054658460EF00FFB002D06DC002826
:104D30000DDD002D02DA01232A4604E0002806DA00
:104D40000123404202B20021584610F0CBF9BAF1DB
:104D5000000F19D158460EF051FB054658460EF08B
:104D6000ADFB002D07DC00280EDD002D03DA01234A
:104D70000022294605E0002806DA012300224042ED
:104D800001B2584610F0AEF90A215846019A0BF0CC
:104D9000E7F96078800706D414F8400F20F00F0080
:104DA000207044F8148CBDE8FC9F7FB50E460400CB
:104DB00003D108F031FE04002CD008F0A1FE002839
:104DC00028D094F82800400724D4002506B3ADF875
:104DD0000050ADF80250204608F036FE401EADF8F7
:104DE0000400204608F076FE401EADF806006A4634
:104DF000314602A8FFF7A0FA00280BD02068017CFA
:104E0000890708D5DDE90001C4E90C01012029E08A
:104E1000A4F850517FBD82690AB102A990470026CB
:104E20000AE004EBC601002202A83031FFF7ACFA19
:104E30000028EFD1761CB6B2B4F85001B042F0D8D9
:104E400080B2202804D204EBC00002A9303004E074
:104E5000A4F8505104F13000694608F005FAB4F89E
:104E60005001401CA4F8500160680028D2D011F015
:104E700001FB7FBD70B5054600F012F804460CE05A
:104E80002146284600F01EF806462146284600F036
:104E9000A2F820460DF08CF93446002CF0D170BDFC
:104EA000002800D04068704700B503460022FFF795
:104EB000F7FF03E01846521C00F004F80100F9D196
:104EC000104600BD0068091D4058704700684058F2
:104ED0007047002800D08068704700224260C91CDB
:104EE00021F0030182600160704770B504460068DC
:104EF00008300DF0D1F8050013D0014600222046FD
:104F000012F0F6F829462046626812F0EBF8616864
:104F100019B12A46204612F0EBF86560A06800B986
:104F2000A560284670BD2DE9F0410C4606000AD068
:104F30004CB1FFF7B5FFA04208D13046FFF7D5FFCF
:104F4000051E01D01EE00020BDE8F0813068083069
:104F50000DF0A2F8051EF7D030682A4607593046F2
:104F6000394612F0BFF83A462946304612F0C0F8EA
:104F70002A462146304612F0BBF8224629463046E2
:104F800012F0B0F82846DFE770B504460068083034
:104F90000DF082F8050013D001460022204612F0E1
:104FA000A1F829462046A26812F0A2F8A16819B11A
:104FB0002A46204612F096F8A560606800B9656040
:104FC000284670BD28B1416809B9806808B1002041
:104FD00070470120704770B504000DD0FFF760FFE7
:104FE00000228842204608D1FFF76CFF6060011E56
:104FF00001D000221EE0A26070BDFFF76AFF884268
:10500000206808440AD10168A16029B12046BDE8A2
:105010007040002212F066B8626070BD05682046DC
:10502000FFF750FF064602462946204612F05AF87E
:105030002A4631462046BDE8704012F059B88068D3
:10504000002801D0B0F9160070478068002801D010
:10505000807E8009704770B5164605460C4651EAB9
:1050600006001AD028460DF0B3FAA868012332468C
:10507000018A21440182A868418A31444182214643
:1050800028460FF0F9FA00220B2128460BF068F8A9
:10509000012803D128460FF06BFA012070BD77B5C7
:1050A00081B00E46050017D062220EF0F9FE040012
:1050B00012D0206880B12846314663220EF0F0FEFF
:1050C00010F0FF0208D0236820460399984700900B
:1050D000BDF80000ADF80C00039804B070BD0000EE
:1050E0002DE9F047074692B0408C1A9E40F0080028
:1050F000788490463A8499468A46328938460EF03A
:10510000CFFE0546A7F820903289514638460EF06A
:10511000C7FE0446788CA54220F00800788403D1AD
:105120002904B1EB044F68D0A7F82080328951469A
:1051300038460EF0B5FE05468046A7F82090514649
:10514000384606F0C5FB318900682A4610F03EFF5C
:1051500030890B2823D147F6FF794D4501D04C45C6
:105160001DD138460FF018F800EBD07045103846C6
:105170000EF0B7F800EBD0704010C84506D1691C9E
:10518000431C994200DA00E0194688464C4506D196
:10519000691C421C914201DA6C1C00E0144619485B
:1051A000FFF7A3FE05002BD02F60C5E903843089EB
:1051B000A8806846C5F808A007F0B2FF1248FF2192
:1051C000CDE900501148029011480390002008904A
:1051D000CDE9090130880B9070889DF8421040425B
:1051E0000C90F0680790002060F300018DF84210E9
:1051F00030690690684607F0E7FF12B0BDE8F08717
:10520000FEE7000028530020799701086199010802
:10521000BD98010814210148FFF75FBE2853002004
:105220002DE9F84F00259046894606462C4604276E
:10523000E6E000BFF06807EBC401405881017CD470
:1052400080B230EA090112D05FF0000230EA0800B3
:105250000FD00020824270D0F0686A46102150F8CA
:105260003400824610F06BFC002871D103E001226B
:10527000ECE70120EEE76A461121504610F05FFC92
:10528000002865D16A461221504610F058FC0028CB
:105290005ED16A461321504610F051FC002857D1C8
:1052A0006A461521504610F04AFC002850D16A4643
:1052B0001421504610F043FCF0BB6A460A215046C8
:1052C00010F03DFCC0BB6A466B21504610F037FC25
:1052D00090BB6A466C21504610F031FC60BB6A46B8
:1052E0000121504610F02BFC30BB6A460421504689
:1052F00010F025FC00BB6A460221504610F01FFC4E
:10530000D0B96A460321504610F019FCA0B96A468C
:105310000521504610F013FC70B96A46062150462C
:1053200010F00DFC40B96A463221504610F007FCDF
:1053300010B96A466E2101E00AE060E0504610F0C4
:10534000FEFB28B96A466D21504610F0F8FB10B1FB
:105350000320BDE8F88F6A466921504610F0EFFB44
:10536000F0BB6A466A21504610F0E9FBC0BB6A46B2
:105370006E21504610F0E3FB90BB6A466D2150460B
:1053800010F0DDFB60BB6A463721504610F0D7FBBA
:1053900030BB6A463821504610F0D1FB00BB6A464C
:1053A0003521504610F0CBFBD0B96A46402150461B
:1053B00010F0C5FBA0B96A464521504610F0BFFB6E
:1053C00070B96A464121504610F0B9FB40B96A46AF
:1053D0004221504610F0B3FB10B96A46432100E069
:1053E00009E0504610F0ABFB28B96A464921504607
:1053F00010F0A5FB08B1022501E005B90125641CE8
:10540000708CC0F30510A0423FF614AF2846A0E709
:105410000148406870470000C80000207047C0F392
:105420000410072800D9072070470000A0F57F412D
:10543000FF3905D0002804D0712803D208490AE0BA
:105440001F2070470749713880B2096829B1064AA0
:105450005268904201D2085C7047002070470000FB
:1054600058E80108740100208801002010B51821B7
:105470000348FFF732FD03490120087010BD00000A
:10548000D4520020900100202DE9F041094D9046B2
:105490000E466A681C46074619469047306020B1A0
:1054A00020686A68384400219047C8F80000BDE8C9
:1054B000F0810000A40100202DE9F04F87B08A465A
:1054C000DDE910581F4693460446002105B12980A6
:1054D0005CB12078002809D0BAF1000F05D0002671
:1054E00018F0060F15D0002004E0002007B0BDE83A
:1054F000F08F401C215C0A2904D00D2902D000291C
:10550000F7D100E0401C002DF0D04FF0FF31298092
:10551000ECE75FEA887001D541F6FF7789460846D7
:105520008DF81410049127E00498CDF8189068B312
:105530004FF0000C05AA06ABCDF80CC0CDF80080EA
:10554000CDE9013220443B465A46514611F0CCF891
:1055500006997A1A314417B20EB288B104990144FF
:10556000049120780A280BD00D2809D0605C0A2805
:105570000FD00D280DD00846205C08B1002FD3DCD9
:10558000049848B105B12E800498AFE74FF0010CA4
:10559000D0E7481C0490F3E7064A04A92046526865
:1055A0009047002DF0D00146002250460AF0ECFE54
:1055B00006B2E8E7A401002000230278232902D0E4
:1055C000012A0DD00FE02AB10021012A04D0022ABD
:1055D00004D008E0012101E0017004E0017001E065
:1055E000202902D00123184670470221F6E7000067
:1055F0002DE9F0471E4614460D468246DDF8209000
:1056000015E000BF4FEA540808FB065739465046DC
:105610004A469047002808DD44F30000C0EB5404DC
:1056200007EB0605A4F1010401E005DA4446002C6D
:10563000E8D12046BDE8F0873846FBE710B5020008
:105640004FF000000CD04B1E194200D0FEE70A4478
:10565000521E9A43B2F5005F02D20C2A01D91046BD
:1056600010BD0C2010BD08444A1E401E904311423C
:1056700000D0FEE7704700002DE9F84F8146407AE0
:105680000F4600F00700022819D0104680469742C6
:1056900000DD3A46164603202A4C2B4A00EB460012
:1056A00020F00305A06811681035411A636805EB06
:1056B000010C9C4505D2416821F0004124E00846D8
:1056C000E4E79D4219D892464FF0FF3B48196168C4
:1056D000884210D9002269461C48CDF800B007F076
:1056E00019FA002269461A4807F014FAA168DAF894
:1056F0000000091AEAE7A068DDE728460CF0CCFCB8
:10570000C0B1416841F0004188EA6702416089EA1E
:1057100002010160416801F04041491C31F08041C3
:1057200041608681A0F80E8005D500F110018160EE
:10573000BDE8F88FFEE7A16801F1100229448260FC
:10574000A160F5E7D00000207001002029A9000821
:1057500075CB000810B5084C012020700748FFF7F2
:105760009FFB0028A06803D0BDE8104010F082BE67
:10577000BDE8104010F072BE480100200453002024
:1057800010B5044690F84200A16B820709D4B4F822
:1057900040204AB1A2F57F43FF3B1BD0521EA4F824
:1057A0004020B4F84020AAB909B1820712D5214699
:1057B0001448FFF710FCFFF7CDFFE16809B1204660
:1057C0008847216909B1204688472046BDE8104036
:1057D0000CF0EEBCE26B52422263002911D082072A
:1057E00002D4626B524222634210521C62F34100A7
:1057F00084F84200A26A206A2262A062E06AE16242
:10580000A06310BD0453002070B5304D686810F0DF
:105810003CFD0646687880F00100687047E0002093
:10582000287094F842006978C0F380028A4242D01E
:1058300061F3820084F84200216B8A19030719D4AE
:10584000002917DC002A15DBC00709D1616939B1CD
:1058500020468847216A01442162A16A0844A06267
:10586000A16809B12046884794F8420040F008003A
:1058700084F84200206B8019206316D4E16A8842C4
:1058800000DD2163E169204688470146606A88425D
:1058900004D0616262680AB120689047D4E90B01C4
:1058A000814202DB2046FFF76BFF287818B10848D9
:1058B000FFF7F6FA03E021460548FFF703FB040073
:1058C000ADD110F0E9FC686070BD00004801002017
:1058D0000453002070B5044640680D4608B1FFF738
:1058E000F9FF2268002A04D029462046BDE870400E
:1058F000104770BD2DE9FF4F99B09846DDE926B1FC
:105900002D9816468A464FF00009042811D0052824
:1059100011D0062812D0142873D10127022508FBC4
:1059200006F00E901A980024401E0D90701E0690EE
:105930004AE10027F2E701270325F0E701270225C6
:10594000FFF766FD0068D0F83890E8E728986043D4
:105950000BEB2022299860430AEB202110124FEA1A
:10596000212E7DD41A9B98427ADABEF1000F77DBA4
:10597000B645F9DAD3B201F0FF0C802B05DAC3F19A
:105980007F014FF0FF32490003E001225900A1F5E9
:1059900080710991BCF1800F05DACCF17F034FF0E3
:1059A000FF315B0004E04FEA4C030121A3F5807353
:1059B0000A930EFB080C199B0CFB05330793831805
:1059C00011937BD4DDF834C0634577DC1EEB010313
:1059D0000F9373D4DDF818C063456FDC079B01FBA0
:1059E00008F102FB053201FB053116929C460C9131
:1059F000BFB32D99052905D014290AD006294CD00A
:105A000059E0E5E00C989CF802208178169880789F
:105A100010E0199A0E9902EB41010B180EFB0811C8
:105A2000119817930EFB08F2085C0F99D25C01FBEA
:105A300008F1C95C914207D00A9B5943C3F58073B2
:105A400002FB0311C1F30721904207D0099B584381
:105A5000C3F5807302FB0300C0F30720084401E094
:105A60009AE02CE02C99400808555FD09CF8001073
:105A70009CF8010001EB0020ADF80C000C980178B7
:105A8000407801EB0020ADF81000169801784078BE
:105A900001EB0020ADF808001FE0BCF800101FFA71
:105AA00089F0814278D00C990988814274D0169986
:105AB0000988814270D0FF210846CFE737E0BCF863
:105AC0000000ADF80C0016980088ADF808000888B2
:105AD000ADF810002C98FF210155BDF80C00BDF861
:105AE0001010884209D1BDF80810884205D12B98C2
:105AF000BDF80C1000EB440017E00A98C2B2DDE9D3
:105B0000031007F0F3FD04900998C2B2DDE9020129
:105B100007F0ECFD7F220290049907F0E7FD00906A
:105B20002B98BDF8001000EB440001804AE0079B71
:105B300093F800C05B780CEB0323DDF8ACC09BB29C
:105B40002CF81430DDF8B4C0BCF1050F06D0BCF160
:105B5000060F06D0BCF1140F09D10AE0079B9B7811
:105B60000FE01FFA89FC634501D1002309E0FF2300
:105B700007E0199B0EFB083C0E9B00EB43031CF84F
:105B8000033008B9002A05DBDDF834C0604504D1D4
:105B9000002A02DD09980BE011E0BEF1000F01D1EF
:105BA000002904DB069A964509D1002907DD0A98E9
:105BB000C0F1FF005843010A2C98015502E02C99CE
:105BC00000200855641C24B22A988442FFF6BEAE19
:105BD0001DB0BDE8F08F10B50446406882080AD0B9
:105BE000496821F00301091D08446060204600F067
:105BF00042F8204610BDFEE74068103120F0030057
:105C0000884201D301207047002070472DE9FC47EE
:105C1000054648680C4620F0030001AA694611F0C9
:105C200025FADDE9007005EBC71101EB800980461C
:105C3000D9F8300060B164B1C4E9020504F1080686
:105C4000C46030460421FFF70EFD864202D0FEE715
:105C5000FEE7FEE7C9F830400120296900FA07F2A3
:105C60001143296105EB870100FA08F04A690243F4
:105C70004A61BDE8FC8710B5044600F087F804606F
:105C800010BD2DE9FC4706464FF000000D000090C6
:105C90000746019042D00C46E9460DF104088029E0
:105CA00007D3084613F060FD411F01208840401EC5
:105CB000044442464946204611F0D8F9009C072C7E
:105CC0002CDA06EB8400019A40694FF0FF3101FAAB
:105CD00002F210400CD1641C3069A14008401DD074
:105CE00013F03AFD0446009006EB8000406978B15D
:105CF00013F032FD034606EBC411019001EB800066
:105D0000076B5FB1786820F00300A84201D2FEE77C
:105D1000FEE739463046009A12F0CFFB3846BDE820
:105D2000FC8710B50446FFF7A6FF416841F0020169
:105D30004160606840F00100606010BD10B504462D
:105D400000F024F8416821F002014160606820F011
:105D50000100606010BD70B506460D46084600F0B3
:105D600015F8040010D02079C0070BD068688008AF
:105D70000BD02146304600F03CF821462846FFF77C
:105D80002AFF0546284670BDFEE7FEE7426800F19F
:105D9000080122F00300001F0844910800D1FEE72B
:105DA000704770B506460C004FF000001ED0F2B1EF
:105DB00020791546C0071BD011462046FFF71CFF6F
:105DC00078B12946204600F025F805462046FFF721
:105DD00052FF6868294640F0020068603046FFF7CD
:105DE00015FF2046FFF7AAFF04F1080070BDFEE78B
:105DF000FEE77CB5054648680C4620F0030001AA82
:105E0000694611F033F9DDE900232146284612F0F6
:105E100054FB7CBD2DE9F0410D46044600F108011C
:105E2000281F0E18606806F1080720F00300401BC9
:105E3000A0F1040838460421FFF715FC874200D082
:105E4000FEE7606820F0030108EB0500001D8142B9
:105E500000D0FEE7307900F0030040EA08007060EF
:105E600020F003000C2800D2FEE7207900F00300A8
:105E7000284360603046FFF754FF3046BDE8F081AC
:105E80002DE9F05F00240D46134F4FF0010A134E29
:105E90004FF4807B4FF40078A14603E014B1012C4D
:105EA00007D101E0594600E041463846FBF7E2FFE2
:105EB00020B1641CE4B2022CF0D306E060B20028EA
:105EC00003DB85F80EA0307001E085F80E90307885
:105ED000A860BDE8F09F000000080140C00100205C
:105EE0002DE9F04F0D4687B0044600210DF028F94A
:105EF00060B32946204600F061FA2946204600F0AA
:105F00006FF8002120460DF083FF05900021204608
:105F10000DF0AEFF0490002120460DF0BCFE0128DC
:105F200000D000208046002120460EF06AF8074687
:105F3000002120460DF000FF42F2D17906464F4580
:105F40000BD1608C000508D4012707E007B0284674
:105F5000BDE8F04F1C210CF02DBA002720460DF0B3
:105F60006DF9DFF878A0834620460021BAF80420B6
:105F70000DF096FFD5F810C0AB682968CDF800C0C9
:105F8000CDF80C80CDE90131C2B239465846059BA7
:105F900005F010FD28834E4504D1608C400501D4E6
:105FA000012600E0002620460DF02EF90746204687
:105FB0000021BAF808200DF073FFC2B2686900240E
:105FC0006B68E9688DE81B0031463846049B05F094
:105FD000F1FC688307B0BDE8F08F0000F0000020FE
:105FE0002DE9F34F81B00C46019805F0CDF9064636
:105FF00001980DF023F98246304600F083FF2061BE
:1060000040000CF077F82060206940000CF072F836
:10601000002541F69A79A0603AE036F91510DFF8CC
:106020002081494533D10027DFF818B11FE03946F8
:1060300001980DF085F8594600900EF0BAF8A8B90D
:10604000009805F0B3F9012810D1009805F0A4F9E3
:10605000A8420BD100980EF09FF84146404501DA66
:10606000084602E000980EF097F880467F1C0198E1
:106070000DF078F8B842DAD8B8F1000F03DBA16868
:1060800021F8158003E0A168002021F815006D1C9F
:106090002069A842C1D800252F46284641F69B78A2
:1060A0004A4615E036F91010414504DB0D44A5F5CC
:1060B000F8559B3D0BE0914204D1A16831F81010D6
:1060C000394403E0A36823F8101039440FB2401C90
:1060D00021698142E6D8002101980DF099FE2169DD
:1060E000C1F1010200FB02A0C01B00B2002800DACF
:1060F000002000224FF0FF331146C44611E000BFDC
:1061000036F9117067450BDBA7F5F8579B3F3AB29C
:1061100000FB02F3B3FBF5F3A76827F811300B4639
:10612000491C27698F42EBD8002B07DBA91A414392
:10613000B1FBF5F1401AA16821F81300BDE8FE8F0C
:1061400001E0FFFF010006002DE9F14F002211469A
:1061500000980FF009F9002100980DF0C3FD0446E6
:10616000002100980DF090FE20440FFA80F90021E4
:1061700000980DF03BFE20440FFA80F800980DF0D7
:106180004BFD00EB090101EB0800DFF898A006B217
:10619000544600980CF0E6FF074600252AE00098D8
:1061A00021498068006850F8250083460EF001F808
:1061B000F8B958460EF034FA40BB002158460DF0AD
:1061C0004FFD18B3012821D002281FD003281DD06D
:1061D000002158460DF027FF58B9BBF81A10BBF83C
:1061E0001600081A401C00B24844A04200DB0446D6
:1061F00024B26D1CBD42D2D3544504D004EB080038
:1062000000B2B04200DC3046BDE8F88F0098BBF920
:106210001A10B0F91600081A411CA142E8DB0C461E
:10622000E6E7000001E0FFFF010004002DE9F84F60
:106230000022804611460FF081F8002140460DF003
:1062400051FD0446002140460DF000FE20440FFAA7
:1062500080FA002140460DF0E7FD20440FFA80F956
:1062600040460DF0E7FC00EB090101EB0A00DFF806
:1062700044B105B25C4640460CF074FF074600216D
:1062800040460DF0F6FC01284FF0000644D078E0BF
:10629000D8F808004849006850F8260000900DF032
:1062A00088FFC0BB00980EF0BBF950B10098B8F958
:1062B0001810B0F91400091A481CA0422ADB4C1C23
:1062C00028E0002100980DF0CBFC58B1032809D03C
:1062D000062807D0082805D0002100980DF09DFE63
:1062E00058B118E00098B8F91810B0F91400081A5D
:1062F000411CA1420EDB0C460CE0009814300090CB
:1063000006F0F9FF5044A04204DB009806F0F3FFCA
:1063100000EB0A0424B2761CBE42B9D35C453BD0E4
:1063200004EB090033E000BFD8F8080022490068F8
:1063300050F8260000900DF03CFF08BB00980EF0CE
:106340006FF960BB002100980DF08AFC38B301287A
:1063500025D0042823D0072821D0002100980DF053
:1063600062FE68B900981430009006F0C4FF4844FB
:10637000A04204DB009806F0BEFF00EB090424B243
:10638000761CBE42D0D35C4506D004EB0A0000B2B6
:10639000584501D0A84200DC2846BDE8F88F009897
:1063A000B0F91810B8F91400091A481CA042E6DB2D
:1063B0004C1CE4E701E0FFFF010004002DE9F84F69
:1063C0000C46834605F068FA064600F09BFD6061C6
:1063D00040000BF08FFE6060606940000BF08AFEA9
:1063E000002541F69A79E0603AE036F91500DFF8C9
:1063F0002881484533D10027DFF820A11FE0394626
:1064000058460CF09DFE514600900DF0D2FEA8B902
:10641000009805F053FA012810D1009805F044FACD
:10642000A8420BD100980CF05CFF4146404501DAD0
:10643000084602E000980CF054FF80467F1C584646
:106440000CF090FEB842DAD8B8F1000F03DBE16837
:1064500021F8158003E0E168002021F815006D1C8B
:106460006069A842C1D800252F46284641F69B788E
:106470004A4615E036F91010414504DB0D44A5F5F8
:10648000F8559B3D0BE0914204D1E16831F81010C2
:10649000394403E0E36823F8101039440FB2401C7C
:1064A00061698142E6D8002158460DF0E1FC814641
:1064B00058460CF0A9FE01466069C0F1010209FBD3
:1064C0000210C01B00B2002800DA002000224FF0AA
:1064D000FF331146C44610E036F9117067450BDBF7
:1064E000A7F5F8579B3F3AB200FB02F3B3FBF5F375
:1064F000E76827F811300B46491C67698F42EBD8D3
:10650000002B07DBA91A4143B1FBF5F1401AE16802
:1065100021F81300BDE8F88F01E0FFFF010006003D
:106520001CB50B8804892344ADF800304B8844899E
:106530002344ADF802308B8804892344ADF804303D
:10654000C98843891944ADF80610436969469847DC
:106550001CBD00002DE9FF4F89B0C8781A9CC00708
:106560000D46002801D0F84800E0F848069001D018
:10657000F74800E0F748049001D1F54800E0F548FD
:106580004FF010034FF00C0E4FF0080BCDF8140035
:106590006188A2884FF0000AA1EB0201504609B2BF
:1065A0005246D4F810C00FE002EB8207E66803EB16
:1065B000870816F808805FEAC87809D00BEB8707D0
:1065C000F65B891B09B2521C9445EDD8002254E0B9
:1065D0000EEB8707F65B304400B2F4E7E66802EBA7
:1065E000820703EB870CB146CDF820C016F80C608B
:1065F000F60741D1002872D091FBF0F80EEB870628
:10660000079639F8066006FB08F60FFA86FCCDF807
:1066100000C04FF0060C0CEB870C042639F90C80F7
:1066200006EB8706DDF800C039F90660E04500DCBE
:10663000C446664504DC009EC446B04500DC6646A0
:10664000DDF800C00196664506D0DDF820C04FF0A9
:106650000108C24649F80C80D4F80C80019E0BEB6F
:10666000870728F80760D4F80CC0079F3CF807702C
:10667000C01B891B00B209B2521C26699642ADD8D4
:10668000BAF1000F84D1002109980DF0FEFA01281B
:1066900026D000270020ADF80800ADF80C0003A9B3
:1066A00002A8CDE900012089B4F9022003B22878BC
:1066B000189910F0AAFEE878384207D009980CF033
:1066C000BDFDBDF808100844ADF808000B99099805
:1066D0000CF036FD06464FF4FA682AE1FFE7FEE7C4
:1066E0000127D7E79C4930460DF063FD00286FD1A4
:1066F000002130460DF00AFBF0B34FF00009484688
:1067000021690FE0E26800EB800352F82320B242D7
:1067100007D1E16800EB80020BEB820031F90090B9
:1067200002E0401C8142EDD8E878C007708C04D0AC
:1067300020F4806040F4006003E020F4006040F446
:106740008060708406F114000499824688474845A9
:1067500028D030460DF00CFFB08AADF80000F08A6A
:10676000ADF80200308BADF80400708BADF8060078
:1067700049465046069A00E010E090476A462921B3
:10678000304609F0EDFC30460CF0D2FD32462221B5
:1067900009F0E6FC30460DF0EBFE03E0708C20F4CF
:1067A00040607084002000906878012811D0022891
:1067B00017D1059906F114008847B4F90010491C57
:1067C00021F00101081A00EBD07040F34F0007E000
:1067D000A7E0059906F1140088472188081A00B23D
:1067E0000090E878384208D0049906F114008847F0
:1067F000BDF80810081AADF80800304600216B22D9
:106800000DF04EFB0FFA80F9304600216C220DF09E
:1068100047FB0FFA80FA30460DF0BEFC019030467F
:106820000CF05FFD0146C9F3413001280FD129F476
:10683000C04040450BDCB0F57A7F01DDC0F57A70D1
:10684000019A5043642290FBF2F00FFA80F9CAF3E8
:10685000413001280ED12AF4C04040450ADCB0F591
:106860007A7F01DDC0F57A704843642190FBF1F036
:106870000FFA80FAB18A1698F28A411A01EB0900E0
:10688000179900B28A1A02EB0A01EA7809B2D20714
:10689000002A02D0BDF9082000E0009A10440FFA47
:1068A00080FA01D0009801E0BDF9080008440FFA11
:1068B00080F95AEA09011BD030460DF059FEB18A21
:1068C00001EB0A00B082318B01EB0A003083F18AC0
:1068D00001EB0900F082718B01EB090070833046F7
:1068E0000DF046FE00234A46514630460DF0C4FEE8
:1068F000E87838420CD1049906F1140088471999B8
:106900000844BDF80C100844BDF80810084406E01F
:10691000BDF80C1019980844BDF80810081AADF815
:106920000800E8780BAAC0F38001099804F0EAFE99
:106930000646002E04D0DDE90B0188427FF4D2AE7A
:106940000DB0BDE8F08F000073D3000869D30008D4
:106950001BD30008CFD20008010006002DE9F04F3C
:1069600091B00E0005463FD02E83286808B10BF089
:106970001FFC06EB4600062101EB40000BF08CFBF0
:10698000286040B3022101EB46010144E960042183
:1069900001EB86010144C5E9010101210024012E1A
:1069A0001AD0F00008300BF0A5FB814600EB860002
:1069B00000F10408B00000B2A346ADF81000C0F129
:1069C00001028010ADF812B00FFA82FA5C46CDF8E1
:1069D00028B00690ABE0FEE7B4220270E8680480BD
:1069E000E8684180A868048011B0BDE8F08F0027F6
:1069F000BDF81220BAF1000F07DC032101EB4201C0
:106A00000AEB01000FFA80FA0CE0BDF81010052324
:106A1000521A03EB420202EB0A00491E0FFA80FAF7
:106A2000ADF81010BDF81200401CADF8120004A81B
:106A300000F0E7F868B1BDF9100006AA811042F82D
:106A400027100AA900F0030041F827007F1C042F3B
:106A5000CEDB042F71D109990698884212D129F80A
:106A6000140028F814B0DDE90A010144DDE90C2026
:106A70001044084469680855696800010855641C99
:106A800024B252E00799884219D029F8140028F856
:106A900014B06A680A9810556A6800011055641CA1
:106AA000069A20B2521E29F8102028F810B0DDE90D
:106AB0000B120A440D99091D11446A682FE00899C8
:106AC00029F81400884228F814B0DDE90A02594672
:106AD000104412D06A6810556A6800011055641C91
:106AE000069A20B2521E29F8102028F81010DDE96D
:106AF0000C12114408316A6811E00C9A10446A685B
:106B000010556A6800011055641C069A20B2521E86
:106B100029F8102028F810100D996A680C311154CA
:106B20006A6809011154401C04B20BF1010B04A85E
:106B300000F067F800287FF45AAF09EB440140F2F7
:106B4000D320464331F9021CB012814205D108EB33
:106B5000440131F9021C81421AD0A6EB8021B1F523
:106B6000007F03DC494341F3CF3106E0C1F580618A
:106B7000494341F3CF31C1F10F0129F8140028F83E
:106B8000140068680155686809010155641C24B245
:106B9000A01E0DE038F8102029F8142039F8102034
:106BA00028F8142069680A5C0A55641C24B2401E47
:106BB0000028EFDAEB680021084619801BE0EA683C
:106BC00022F81100AB6839F8102023F811200AE0F0
:106BD000AE6839F9102036F81130934200DA1A46BF
:106BE00026F81120401C38F910208A4201D1A04219
:106BF000EEDB491C09B2A042E1DB48460BF0C6FAC5
:106C0000F2E6B0F90210B0F90000814201DC012087
:106C100070470020704717B581B0022A03D8BDF82D
:106C2000080004B010BDBDF80830BDF80400D90A52
:106C300001EBD0211F2900D31F2161F3CF20C3F323
:106C40004511C0F345142144ADF804003F2900D399
:106C50003F2161F34A1003F01F0100F01F031944A4
:106C6000ADF804001F2900D31F2161F30400ADF823
:106C70000400FF2A07D0DDE9010106F01DFD0090A8
:106C8000BDF80000CDE780B2CBE717B581B0022A8E
:106C900003D8BDF8080004B010BDBDF80400BDF86D
:106CA0000810C30ACC0A63435B0963F3CF2001F0E9
:106CB0001F0400F01F0363435B0963F30400C0F388
:106CC0004513C1F345114B43990961F34A10ADF8DF
:106CD0000400FF2A07D0DDE9010106F0EDFC009079
:106CE000BDF80000D7E780B2D5E717B581B0022A1A
:106CF00003D8BDF8080004B010BDBDF80830BDF8D9
:106D00000400D90AA1EBD021002900DC002161F3A5
:106D1000CF20C3F34511C0F34514091BADF804009F
:106D2000002900DC002161F34A1003F01F0100F08C
:106D30001F03C91AADF80400002900DC002161F32B
:106D40000400ADF80400FF2A07D0DDE9010106F0D8
:106D5000B3FC0090BDF80000CDE780B2CBE72DE991
:106D6000FF4F89B00446169EDDE919577000DDF823
:106D70006090DDF828A00FFA80FBB9F1040F22D053
:106D8000B9F1060F1FD0B9F1050F5CD0B9F1140F9E
:106D900056D1B4F90000B4F90210CDF80CB006FBDE
:106DA00001030AEB43020092E2884FF00008511AF7
:106DB000491C0FFA81F9A188081A401C0FFA80FAC1
:106DC0004FEA4A0B81E0204606F087FA014603901D
:106DD00038460BF01DFBB4F90000B4F90280A1881D
:106DE00006FB0802081A401C00B2069040000AEB9D
:106DF000420A2E4602900CE051463046029A0BF0B1
:106E000013FA069808F10108DA4406EB40060FFA77
:106E100088F8B4F906004045EEDAB9F1060F0FD153
:106E200000224FF4FC60ADF80000114605E035F893
:106E30001130834200D17A54491C039B9942F6D306
:106E40000DB0BDE8F08FB4F90010B4F9023006FBC4
:106E5000031000EB400202EB0A00A288511A491C01
:106E60000AB2B11A01EB41010EB2E188C91A491CFC
:106E70000CB2002317E000210DE090F802C007F8E3
:106E800001C010F801CB10F8028B0CEB082C25F890
:106E900011C0491C09B29142EFDB5B1C05EB4205B6
:106EA000174430441BB2A342E5DBC9E75A462846E3
:106EB00000990BF0B9F90099039805EB4A050844CD
:106EC000009008F101000FFA80F8C845EEDBDDE91B
:106ED0000A014A000C9902FB0100B4F90010B4F950
:106EE000022006FB02110D18002408E05246294634
:106EF00038460BF099F9641C5744354424B24C458C
:106F0000F4DB9DE70146002041F6FF7200E0401CE3
:106F100031F910309342FAD1704708B5084611464E
:106F200006F0F4FA0090BDF8000008BD2DE9F04F1E
:106F30000746C87A89B015460E46022803D80120B4
:106F400009B0BDE8F08F18463269B168FDF7F8FC6A
:106F5000041EF5D0207D00F01F0009F052FE4FF412
:106F6000807808B1062011E0207D00F01F000E2877
:106F700006D014280AD009F034FE30B1052005E00F
:106F800030884FF00E0930B902E00420814606E057
:106F90007088404503D000204FF00509A061226AA7
:106FA00022B12946384611F08EFEB7E0A069E0B361
:106FB000294602A806F061F9B6F9003013B97088C5
:106FC000404529D0A88829886A88401A401C01B207
:106FD000E88806F1040C801A401C02B27088CDE9E2
:106FE000000C02A8FDF7F6FBBDF80800298808444C
:106FF000ADF80800BDF80A1068880844ADF80A002A
:10700000BDF80C0029880844ADF80C00BDF80E103E
:1070100068880844ADF80E0002AA04A8B968FDF714
:107020008BF900287AD004A800E00DE0D7F808809A
:10703000B860CDF800902A4631463846A36906F07C
:1070400099FDC7F8088069E02A4604A8B968FDF7E9
:1070500073F9E0B3BDF81400BDF81010401A401CDD
:107060000FFA80FB0BEB4B000BF044F8039004A9E4
:1070700001A8D7F808A006F000F9012101A806F040
:1070800073F9BDF91000B5F90010BDF91280401A6E
:107090000690B5F90200A8EB000536E001AA5146BA
:1070A00007A8FDF749F970B30398009006985B466E
:1070B00001B22AB220460AF071F901280ED020460A
:1070C0000AF0C1F803980BF061F8204600E025E0D3
:1070D0000AF0B9F80020C7F808A031E707A8B8609F
:1070E000CDF8009001AA31463846039B06F042FDD8
:1070F000BDF80600401CADF80600BDF80A00401CB3
:10710000ADF80A006D1C08F10108BDF916004045F4
:10711000C4DAC7F808A003980BF038F820460AF044
:1071200092F80CE72DE9F0418046104817460D46CD
:107130000078B0B1B5F902600FE000BFB5F90040CA
:1071400006E03A88B1B2A0B2FCF722F8641CBF1C7A
:10715000B5F90400A042F4DA761CB5F90600B04295
:10716000ECDA4046BDE8F04106F050BCBC0100201E
:107170002DE9F74FC878A0B00C4602287DD91146FA
:1071800001A806F095F8B4F92000012829DD94F84B
:107190002200FD2825D3208818B394F82300BDF8D9
:1071A00004104008C0F380021144ADF80410BDF88B
:1071B0000610C0F340000844ADF8060094F8231010
:1071C000BDF808004908C1F3C001401AADF8080035
:1071D00094F82310BDF80A00C1F34001401AADF83D
:1071E0000A00209801A9826805A8FDF7A5F80028E3
:1071F00043D0E07B10F0070619D0E088ADF800001E
:10720000BDF800006189884200D1002601A807F07E
:1072100003FA07461C210EA8F9F7B8FAA0788DF8F2
:107220005100BDF80000ADF840001FB105E06068F6
:107230000090E5E7208800B9EEB3E078FD2800D3A0
:10724000FF208346BDF80800BDF80410401A401C1A
:107250000FFA80FABDF80A00BDF80610401A401C6B
:1072600001B289465046CA4500DB0846B4F90050D1
:10727000B5EB600F00DB451000E043E0BDF81810EF
:10728000BDF81400081A401C0FFA80F84FF0FF30C8
:107290001D9000200790002D00DC87B140460AF0C9
:1072A00029FF079000232A4601A916A807F020FC11
:1072B000002116A800E01CE006F0CEFF1D90BDF8EE
:1072C0001400ADF80C00BDF81800ADF810000798D8
:1072D000119003A80E901390FF208DF850004A469D
:1072E0005146A01D09F070FA040018D0022E0CD0EF
:1072F00015E001A80E90E0788DF850000EA92098B6
:1073000007F0BCFE23B0BDE8F08FBDF91410A068F3
:1073100000EB4100BDF90410A0EB41000F90002FDD
:107320007DD0BDF9165027E02FB2ADF80E70ADF844
:1073300012704246594607980BF00AF8BDF914102E
:1073400043463A46079807F029F98DF84800012886
:1073500002D102208DF84800012E08D1BDF9061097
:10736000A068691A00EB41000088ADF840000EA942
:10737000209807F083FE6D1CBDF91A00A842D3DAED
:10738000B7E000BFBDF80600BDF9161038440FFA8B
:1073900080F9BDF80A00C01B0FFA80FA494503DDE9
:1073A000BDF91A10514544DB4246594607980AF088
:1073B000CFFFBDF90C1043464A46079807F0EEF898
:1073C0008DF84800012802D102208DF84800BDF94F
:1073D0001610494513DCADF80E90ADF81290012E51
:1073E00009D1BDF90620A168A9EB020001EB40001C
:1073F0000088ADF840000EA9209807F03FFEBDF9C7
:107400001A10514515DBADF80EA0ADF812A0012EF3
:107410000BD1BDF90600A268AAEB000000E009E06C
:1074200002EB40000088ADF840000EA9209807F05C
:1074300025FE7F1CAF42A5DBBDF80400ADF8780047
:10744000BDF80800ADF87C00BDF806002844ADF892
:107450007A00BDF80A00401BADF87E001EA807F0B8
:10746000DBF8074630430CD001208DF84800BDF909
:107470000A008DF850B0A0EB0509BDF906000544DF
:1074800035E0BDF806008DF850B02844ADF80E0088
:10749000BDF80A000EA9401BADF8120000201190A3
:1074A000209807F0EBFD24E06FB14246594607985B
:1074B0000AF04EFFBDF9141043462AB2079807F0B0
:1074C0006DF88DF84800ADF80E50ADF81250012E51
:1074D00008D1BDF90600A168281A01EB4000008818
:1074E000ADF840000EA9209807F0C8FD6D1C4D4571
:1074F000DADD079808B10AF049FE1D98401C05D056
:107500001D9807F0A1FB16A807F06AF8002C3FF4BD
:10751000F9AE204609F052F9F4E62DE9F0410646AD
:10752000086992B015460C4600287DD0A07E02283E
:107530007AD929460EA8B268FCF7FEFE002873D05F
:107540000EA8D6F80880B060206909F03AFF02283A
:1075500006D06946206909F097FE012849D0C9E0A4
:10756000002741F6FF70CDE900700297D4E90412BC
:107570003B4610A80FF052F9284605F0C8FE014618
:107580002A88BDF9400001EBD17102EB610100EBEB
:10759000D072A1EB62010844401EADF81000ADF8B6
:1075A0000C10284605F08DFE01466A88BDF94200A0
:1075B00001EBD17102EB610100EBD072A1EB620132
:1075C0000844401EADF81200ADF80E1005A806F0F4
:1075D00093FD60690590208BADF82000A07E8DF8AA
:1075E0002E00009703AA05A93046236906F0E4FAA5
:1075F00080E005A806F0C6FAA0788DF82000208B60
:10760000ADF81C00E07E8DF81E00A07E8DF81F00F6
:10761000207F4FF0FF3740B100996888ADF8060031
:1076200007EB515108445DE066E0284605F06FFE27
:10763000298800EBD07001EB60000099C1F38A212A
:10764000A0EB5100ADF80400284605F03AFE698829
:1076500000EBD07001EB60010098A1EB9051C0F3FA
:107660008A22ADF80610BDF80430521E1A4407EB0A
:107670005050ADF808200844ADF80A0001AA05A949
:107680003046236906F04AFA34E000992888C1F3AD
:107690008A21ADF80400491E084410E001AA05A99A
:1076A0003046236906F03AFA0098BDF80410C0F39A
:1076B0008A200144ADF80410BDF808100844ADF864
:1076C0000800BDF90400B5F904108842E6DDBDF8F4
:1076D0000610009801EB5051ADF80610BDF80A10E5
:1076E00001EB5050ADF80A00BDF90600B5F90610DF
:1076F0008842CADDC6F8088012B0BDE8F081F0B556
:10770000074691F8220087B016460C4602286BD92E
:10771000208C002868D094F8230010F03E0F63D02E
:10772000C00761D1B08831887288401A401C01B20C
:10773000F088B4F90050801A401C00B2814200DA8F
:107740000846B5EB600F00DD4510314604A805F092
:10775000AFFD94F82300BDF91020C0F344014807A1
:10776000B4F9200001D4284440421044ADF8100080
:107770000807BDF91420B4F9200001D42844404280
:10778000101AADF8140094F82300BDF91210400847
:107790008007B4F9200001D4284440420844ADF8E1
:1077A000120094F82300BDF916104008C007B4F980
:1077B000200001D128444042081AADF81600208C60
:1077C000281A00B2002800DA0020A27894F82210CB
:1077D000CDE90212E18BADF8041000902B4604AA0B
:1077E0003146384600F002F807B0F0BD2DE9FF4FF2
:1077F000A9B01D46DDE93879DDF8D88016460C467B
:10780000FF2F00D3FF27084606F006FF26902843E7
:1078100050EA080074D029982146826808A8FCF72D
:107820008BFD002873D0BDF82400BDF82010401A4D
:10783000401C00B204901C210AA80AF0BBFD049869
:107840000AF058FC0D904FF0FF302490002D0ADD17
:1078500000232A46214615A807F04AF9002115A859
:1078600006F0FAFC24900123424631461BA807F09B
:107870003FF900211BA806F0EFFC259001A80A9013
:107880000F90BDF8DC008DF84070ADF830008DF839
:107890004190B4F900002290B6F9003041199942A4
:1078A00000DC1946B4F904000FFA81F92190B6F909
:1078B0000410421B8A4200DB0A460FFA82F8B4F930
:1078C00002E0B6F902200EEB05009246504500DCBE
:1078D0001046B4F906B007B2B6F90620ABEB0500C6
:1078E000904200DB104600B20590A8EB0900401C56
:1078F00000B22790D6450DDC01200CE000E006E048
:10790000009732462146379B299800F0B8F92DB0F0
:10791000BDE8F08F00208246934501DB012000E0A6
:10792000002083462698D8B3BDF82000ADF80400A7
:10793000BDF82400ADF80800BDF9224022E000BFE8
:10794000BAF1000F01D1A7421BDCBBF1000F02D13D
:107950000598A0421ADB25B2ADF80650ADF80A50E2
:1079600004990D980AF054FDBDF920102A46049B95
:107970000D9806F013FE8DF838000AA9299807F033
:107980007DFB641CBDF92600A042D9DA1BA806F0D5
:1079900027FE259807F058F92498401C07D000E0EE
:1079A00009E015A806F01CFE249807F04DF90D9883
:1079B0000AF0ECFBABE72298984201DC012000E0E2
:1079C000002013902198884201DB012100E0002172
:1079D0000120009013981291084000EA0A0010EA72
:1079E0000B0F04D02798322801DA002000900120E4
:1079F00000998DF838001AEA010F0ED0ADF8049006
:107A0000ADF808806088ADF8060070880AA9401EAD
:107A1000ADF80A00299807F031FB00991BEA010F25
:107A20000ED0ADF80490ADF80880F0880AA9401C8B
:107A3000ADF80600E088ADF80A00299807F01EFBB3
:107A4000139878B12088ADF804003088ADF806703E
:107A5000401EADF808000598ADF80A000AA929985B
:107A600007F00CFB129878B1B0880AA9401CADF859
:107A70000400A088ADF808000598ADF80670ADF8D0
:107A80000A00299807F0FAFA0098C0B1BDF924005D
:107A9000BDF92010A9F10102ADF80410904200DBFD
:107AA0001046ADF80800401A401C05B2002D70DDEC
:107AB000139850EA0A0066D0BDF9224061E0BDF893
:107AC0002000ADF80400BDF82400ADF80800B6F9B8
:107AD0000200B4F90210401AA84200DB05460FFA72
:107AE00085F8002533E06088284406B2E088401B12
:107AF00007B2BDF92200B04203DDBDF92600B8424D
:107B000024DB04990D980AF083FCBDF90410324679
:107B1000049B0D9806F042FD8DF83800BDF9220057
:107B2000B04207DCADF80660ADF80A600AA92998F2
:107B300007F0A4FABDF92600B84207DBADF80670DD
:107B4000ADF80A700AA9299807F098FA6D1C454506
:107B5000C9DB8DE026B2ADF80660ADF80A602946B3
:107B60000D980AF055FCBDF904102B4632460D98CD
:107B700006F014FD8DF838000AA9299807F07EFA5E
:107B8000641CA742E6DC139850EA0B001DD0059C4C
:107B900016E01AE026B2ADF80660ADF80A60294694
:107BA0000D980AF035FCBDF904102B4632460D98AD
:107BB00006F0F4FC8DF838000AA9299807F05EFA5F
:107BC000BDF92600641CA042E4DABDF9200008F1EA
:107BD0000101884200DC0846BDF82410ADF804001D
:107BE000081A401C05B2ADF80810002D40DD1298AF
:107BF00050EA0A001BD0BDF9224016E026B2ADF8CB
:107C00000660ADF80A6029460D980AF001FCBDF93E
:107C100004102B4632460D9806F0C0FC8DF8380053
:107C20000AA9299807F02AFA641CA742E6DC1298F0
:107C300050EA0B001CD0059C15E026B2ADF806609A
:107C4000ADF80A6029460D980AF0E2FBBDF9041070
:107C50002B4632460D9806F0A1FC8DF838000AA993
:107C6000299807F00BFABDF92600641CA042E4DA5B
:107C70001BA806F0B5FC259806F0E6FF8FE62DE977
:107C8000FF478EB00C46824615461C2102A81A9E5C
:107C90000AF090FBCDF808D0BDF84400ADF8100014
:107CA0008DF82060B4F90200B5F90210884201DCB9
:107CB000012700E00027B4F90600B5F90610884254
:107CC00001DB012600E00026B4F90000B5F9001040
:107CD000884201DC012100E000218946B4F904104A
:107CE000B5F90420914201DB012100E00021ADF84B
:107CF0000000A088ADF804006088ADF80200688834
:107D00008846401EADF806001FB102A9504607F094
:107D1000B5F9E888401CADF80200E088ADF806002F
:107D20001EB102A9504607F0A9F92088ADF800005D
:107D30002888401EADF8040017B1B5F9020001E033
:107D4000B4F90200ADF8020016B1B5F9060001E081
:107D5000B4F90600ADF80600B9F1000F03D002A98E
:107D6000504607F08BF9A888401CADF80000A088A9
:107D7000ADF80400B8F1000F03D002A9504607F097
:107D80007DF912B0BDE8F0872DE9F0412E4D074690
:107D9000686805F055FE04463868C66B716B09B11A
:107DA0003046884768680068B0F90010B0F90200F2
:107DB0004143E068814201D1012000E000202168B8
:107DC00059B1616849B128B107E068680068816A03
:107DD00001B1884720690028F7D101202061696836
:107DE0000968C9688A69D20702D08969890700D4FD
:107DF00000206061606908B1012500E00025386855
:107E0000416971B1016911F0300F06D0490704D5FD
:107E1000D6E9001000F01AF803E0D6E90021FEF7D9
:107E20007FFB206800280BD06168002908D03A68E1
:107E3000127CAA43D20703D1A268824202D1A16078
:107E4000BDE8F081A060FBE7C80000202DE9F34FFA
:107E500005468A4893B041680E683069820701D5AB
:107E600042076ED4C0F3011002281ED0012801D0B1
:107E7000032866D100200F90084605F0E1FD8346F7
:107E8000A988B5F90000EA88091A491C0CB2B5F9AD
:107E90000210521A521C17B24FF42052B2FBF4F3E4
:107EA000BB420FDAB2FBF4F20DE029463046149AD9
:107EB00000F0F0F8149A15B029463046BDE8F04FAE
:107EC000FEF72EBB3A460C920791317CC1F30111AB
:107ED000012905D06880611E0844E8800020BDE0CB
:107EE0007188081A401EE880001B401C6880F5E776
:107EF0000C99A7EB0A00884200DD084600B2019009
:107F00000120CBF81000BAF1000F20D1A7421EDBF0
:107F10000194307CC0F30110032810D000202146CA
:107F2000149A00F0ECF8307CC0F30110012809D05D
:107F300031880798081A401EA880001B56E00120CF
:107F4000EDE797E0079828800798204466E00F98AF
:107F500020B94FF4A0400AF0CDF80F90307CC0F368
:107F6000011003281BD000208646DDF850C001997F
:107F70000F980A9004FB01F0401E0D90601E4843CC
:107F80000E9000208146884222DA0E9ABEF1000F40
:107F900002EB090001D00D9A101A002212E0012014
:107FA000E2E70A9BBEF1000F03EB400863460CF1C9
:107FB000020C1B88A8F8003001D0084400E0401AE9
:107FC000521C12B2A242ECDB09F1010000B2D9E767
:107FD000307CC0F3011001281BD031880798091AA2
:107FE000A1EB0A00401EA8800199401A401C28807D
:107FF00001990AEB0108B84513DBDBF81800C0074C
:108000000FD0DBF8180080070BD50120CBF8140047
:108010000AE007985044288001990844401EA8802F
:10802000E6E70021CBF814100F9828B10246294644
:108030003046FEF775FA05E0149AF8E7B16A09B11F
:1080400030468847DBF810000028F7D101981499D2
:10805000604301EB400014900FFA88F08246B8426A
:10806000FFF646AF0F98002804D015B0BDE8F04FDA
:108070000AF08CB815B0BDE8F08F0000C8000020F1
:1080800030B504880D880580108808801888108015
:108090001C8030BDF8B58B880C884D881B1BCC88A4
:1080A0005B1C641B641C1BB224B2634300245B1E74
:1080B0000EE000BF02EB430602EB44073588ADF843
:1080C0000050B7F800C0A6F800C05B1E3D80641CDD
:1080D000A342EFD843884C88CA881B1B5B1ECB8009
:1080E00043889A1A521E4A8003880C888A881B1B70
:1080F0005B1E8B800088801A401E0880F8BD2DE929
:10810000F0470C4617468246002601EBD47931E051
:108110000025601C00EBD07827E0A01B401E01B2B8
:10812000601B401E00B2BAF1000F0AD005FB04121A
:1081300001FB040107EB420300FB046007EB410273
:1081400009E000FB046201FB040007EB420307EBBC
:10815000400205FB041007EB400106FB045007EB4F
:108160004000FFF78DFF6D1C2DB2B5EB680FD4DB1F
:10817000761C36B2B6EB690FCADBBDE8F0870000AB
:108180002DE9FF4F9FB0987B8A7E00F00F04DDF849
:10819000B0E00E46032C18D0012C1DD0022C21D0AB
:1081A000042C13D0082C7DD1A34D4FF0FF0A6101A0
:1081B000FD2A2FD2A14F3878904202D17868A04290
:1081C00025D00020DFF878821FE004249A4D4FF07C
:1081D000F00A103D1021EBE7974D4FF0800A163D55
:1081E0000221E5E7944D4FF0C00A143D0421DFE77A
:1081F00015F800C0BCF1FF0F1DD00CFB02FC4FEACC
:108200001C2C00BF08F800C0401C8842F0D38C4DE5
:108210003A707C602199B3F8068018890790B1F90B
:1082200000201F9908FB04F08968B1F900309A42D8
:1082300003DB002302E09446E4E79B1A9B46B1F976
:10824000043002EB08079F4201DC424601E09A1A23
:10825000521C9146219AB1F90230B2F902209A4299
:1082600001DB002300E09B1A1193079BB1F9061074
:1082700013448B4201DC079901E0891A491C0A91D9
:10828000119941430BFB04100EEBD00100F00707DE
:108290002C911C2115A80AF08DF8B089ADF85C006E
:1082A000B07E00E0C4E08DF86C00B07FC0F3C20087
:1082B0008DF86D00FDF7ACF805F0C6FB079A08FBDA
:1082C00002F1814200DC08461C9009F013FF079080
:1082D000189021980026008800EB0B02ADF80C20C6
:1082E00021980188A9F1010001442198ADF81010EE
:1082F0004388119818448B1AADF81200ADF80E009F
:10830000ADF83810ADF834200A99ADF836005B1C92
:1083100008441BB2ADF83A000B930DA806F07CF9A7
:108320001D9003A815901A90C4F1080008EB0B01EA
:108330000F90A1EB090060431290119860E0334662
:108340002AFA07F059464FF0000C1FE02C9ADDF88E
:108350003C801278A8EB0708024032FA08F205D0F8
:1083600015F80280079A02F8068002E0079A02F8E0
:1083700006C00F9A974202D22744E04004E02C9AAC
:108380000027521C50462C92491C761C4945DDDBC7
:108390001D9880B10798BDF912201844BDF90C1042
:1083A00080460B9B06F0FAF88DF8640018B9404639
:1083B0000B9909F0FFFFA9EB0B0081191C98814272
:1083C00005D2BDF81200401CADF812000EE00220EC
:1083D0008DF8640015A91F9806F050FEBDF8120034
:1083E000401CADF80E00ADF81200002612982C9932
:1083F000384401EBD00100F0070701982C91401C94
:10840000014601900A98814299DBBDF90E10BDF931
:108410001200814209D0401EADF8120002208DF8F2
:10842000640015A91F9806F029FE079809F0AEFE12
:1084300023B0BDE8F08F00009AAF0108DC000020F7
:10844000885100202DE9F04F8346B1F902000C4617
:10845000401E411000F001004618B2F90050B3F977
:10846000000089B0854200DA2846ADF80000B2F974
:108470000000B3F90030984200DC1846401EADF809
:1084800004005088801BADF8020050880844ADF805
:10849000060069460846DBF80820FBF74DFF002878
:1084A0001FD0E08818B1A08808B1012700E000279C
:1084B0000125684606F0B0F800B907B100251C2177
:1084C00002A809F077FFCDF808D02088ADF8100099
:1084D000207A6E468DF8200035B102A9584606F084
:1084E000CDFD09B0BDE8F08FBDF80410BDF9000066
:1084F000BDF90680091A491C0DB2BDF80210ADF88D
:1085000006104FF0000A47B1B4F90610B4F9042080
:10851000114490FBF1F201FB120A284609F0EAFD32
:10852000079605908146BDF902603EE0294648461F
:1085300009F06EFFBDF900102B4632B2484606F036
:108540002DF88DF818000FB300B3002150460B46EC
:1085500017E000BFB4F90420824205DB121A11446F
:10856000104409B200B208E0B4F906C06244824285
:1085700001DC002001E009F80130491C401C09B26F
:1085800000B2A942E6DB02208DF8180002A9584685
:1085900006F074FDBDF80200401CADF80200BDF805
:1085A0000600401CADF80600761C4645BEDD484678
:1085B00009F0ECFD95E700002DE9FF4FB2F90250FC
:1085C000B3F90240C5B0A54208DA128865F31F402E
:1085D00062F30F0064F31F411A8807E01B8864F3FD
:1085E0001F40128865F31F4163F30F0062F30F0110
:1085F0000FFA81F904B20514A9EB04064FEA214AE7
:10860000AAEB05070391002E01DD314600E071421F
:10861000002F01DD384600E07842814201DD012073
:1086200000E0002015904698B0F90210159858B156
:10863000002F01DD384600E078424201002E01DDC6
:1086400030460CE070420AE0002E01DD304600E0CA
:1086500070424201002F01DD384600E0784292FB73
:10866000F0F0AA4A105C48433F30C0114FEA60085E
:1086700000F0010202EB080B49464C4500DA2146A6
:10868000A1EB0001ADF8581001DD214600E049469C
:108690000144ADF85C105146554500DA2946A1EB7E
:1086A0000001ADF85A1001DD294600E051460844AA
:1086B000ADF85E00459816A982680846FBF73CFEB7
:1086C00000287DD01598002100287AD0002E16DDD4
:1086D000AAEB080000B2CDE90001A5EB080002B248
:1086E0004B46214620A806F03BF80AEB0B0001217F
:1086F00000B2CDE900014B4605EB0B0015E00AEB9B
:108700000B0000B2CDE9000105EB0B0002B24B46B5
:10871000214620A806F024F8AAEB0800012100B2A7
:10872000CDE900014B46A5EB080002B221460AA89C
:1087300006F016F8002120A805F08EFD1890002103
:108740000AA805F089FD159046984FF0FF39C846F4
:10875000407AC00623D4A819032100B2CDE9000154
:10876000E01B03B22A4621462BA805F0F9FF039926
:1087700002200A14911909B2CDE90010039801B240
:10878000C81B03B236A805F0EBFF00212BA805F0AB
:1087900063FD8146002136A805F05EFD8046BDF8E8
:1087A0005C00BDF85810401A401C04B2FCF730FEC3
:1087B00005F04AF9054616A804F08FFDA84201E02D
:1087C000A1E004E01AD216A804F087FD17E009EB37
:1087D0000B00CDE900A103B204EB0B0001B22A4665
:1087E00020A805F0BDFF0121A9EB0800CDE900A1FB
:1087F00003B2A4EB080001B22A4698E72846824655
:1088000009F078FC8346BDF95E70BDF85A00ADF8FA
:108810005E0000255146584609F0FAFD1C2119A8B2
:1088200009F0C8FD16A9199146980088ADF86C00AA
:108830004698BDF95A60007A8DF87C00CDF870B08A
:108840001E912DE0BDF958100BEB0500234632B206
:10885000079005F0A3FE8DF8740018B9214607981B
:1088600009F0A8FD25442919514505D2BDF85E003F
:10887000401CADF85E0012E002208DF8740019A9CA
:10888000459806F0FBFBBDF85E000025401CADF8E6
:108890005A00ADF85E005146584609F0B9FD761C05
:1088A000BE42CFDDBDF95A10BDF95E00814209D04C
:1088B000401EADF85E0002208DF8740019A945989D
:1088C00006F0DCFB584609F061FC20A805F088FEA4
:1088D0000AA805F085FEB9F1FF3F02D02BA805F0EC
:1088E0007FFEB8F1FF3F02D036A805F079FE189858
:1088F00006F0AAF9159806F0A7F9484606F0A4F97B
:10890000404606F0A1F949B0BDE8F08F9AB00108E1
:108910002DE9F04F8346B1F902000C46401E41108C
:1089200000F00100158889B00844281AADF800004D
:1089300010880844ADF80400B2F90210B3F902003F
:10894000814200DA0846ADF80200B2F90200B3F93C
:108950000210884200DC0846401EADF80600694659
:108960000846DBF80820FBF7E7FC00281FD0E0886A
:1089700018B1A08808B1012600E00026012768464A
:1089800005F04AFE00B906B100271C2102A809F033
:1089900011FDCDF808D02088ADF81000207A6D4682
:1089A0008DF8200037B102A9584606F067FB09B0E0
:1089B000BDE8F08FBDF80400BDF80010BDF90670E9
:1089C000401A401C0FFA80F9BDF80200ADF806000D
:1089D000484609F08FFB824605900795002056B166
:1089E000B4F90600B4F904100844BDF9021091FB73
:1089F000F0F200FB12108046BDF9025031E049460A
:108A0000504609F005FDBDF900104B462AB250460C
:108A100005F0C4FD8DF81800A6B178B1B4F90410C2
:108A2000414502DA00208DF81800B4F90600B4F9C7
:108A300004100144414501DC4FF0000808F1010039
:108A40000FFA80F802A9584606F018FBBDF802009C
:108A5000401CADF80200BDF80600401CADF8060051
:108A60006D1CBD42CBDD504609F090FB9FE72DE920
:108A7000F04798B0054607F071FB0446284607F01A
:108A800035FB064609A920460AF090FB94F84800F9
:108A90000025C10600D50125800601D545F0020557
:108AA000002120460BF0B3FAA0F51C51D13904D1B6
:108AB000608C000501D445F004050BA805F01CFBF3
:108AC000B4F84400ADF84200B4F84600ADF84400F4
:108AD0008DF849500BAA002120460BF0A3FB9DF80E
:108AE00048004FF0010808B98DF84880E06B0C9001
:108AF000206C0D900C994FF6FF7081421ED00D999D
:108B000081421BD04FF480292746552249462046F2
:108B10000BF0C6F9024649463846FCF7C0FA009009
:108B2000BDF80000ADF83A002046202249460BF07F
:108B3000B7F90090BDF80000ADF83C0094F848008B
:108B400041F6FF7A00F00700022801D003281ED169
:108B50009DF84800022801D0032818D1BDF93E1025
:108B6000CDE9001A0295BDF940300B9A16A8616A4A
:108B70000DF054FEBDF82800BDF82410401A401C2A
:108B8000BDF9581000B2884201DA8DF8488094F897
:108B9000480004F1300700F00700032809D0BDF8B1
:108BA0002A00BDF82610401A401C00B2B0F5806FB4
:108BB00000DA002709A914A8B268FBF7BDFB00285A
:108BC0007DD094F8480040070BD120460AF0E2FC23
:108BD000404202B2002109A804F0B2FB608BADF85C
:108BE0002A0094F848000DF1500900F0070002280F
:108BF00013D0032811D0009709AA0BA93046636A45
:108C000004F0DAFFB068C6F80890804694F848008F
:108C100000F0070003280FD05FE0D6F80880C6F800
:108C20000890009709AA0BA93046636A04F0C4FFB4
:108C30004046C6F80880E6E7BDF93E10CDE9001AC7
:108C40000295BDF940300B9A06A8616A0DF0E6FD69
:108C5000BDF82800BDF82410401A401CBDF91810BA
:108C600000B2884219DA202211460B9807F08CFBDB
:108C7000B4F84410BDF8182000EB4000114408443B
:108C8000ADF84200B4F84600ADF84400009709AAD8
:108C90000BA93046636A04F08FFFBDF82A00BDF8C7
:108CA0002610401A401C01B2BDF91A00814214DAA4
:108CB000B4F84410ADF842100B99098900E00EE0B9
:108CC000B4F84620009710440844ADF8440009AABF
:108CD0000BA93046636A04F06FFFC6F8088018B02D
:108CE000BDE8F08730B5054691F82A0089B00C46FA
:108CF00002285FD9E08C00285CD0114604A804F05B
:108D0000D7FA208DBDF81010401E091AADF81010CA
:108D1000BDF81210091AADF81210BDF81410014474
:108D2000ADF81410BDF816100844ADF8160004A9EB
:108D300006A804F0BDFABDF81810E08CBDF81220AA
:108D4000091AADF81810BDF81C100844ADF81C0045
:108D5000BDF81A00E18C401AADF81A00BDF81E00EB
:108D6000E18C0844ADF81E00BDF81400BDF81010E9
:108D7000401ABDF81610401C891A491C00B209B2ED
:108D8000B4F90020884200DA0146B2EB610F00DD41
:108D90004A10E08CA178104403B294F82A00CDE97F
:108DA0000201A08CADF80400009204AA06A928468E
:108DB000FEF71CFD09B030BD7CB5044680696189B1
:108DC0006D468668A08961B1002865D0814203D1D3
:108DD0002289E3889A427CD302297BD003297AD066
:108DE000AFE010BBE088218988421ED2B4F90600AA
:108DF0000DF050FCB4F90410B4F90E20891A484360
:108E00002168498801EBE030ADF80200E0885A3073
:108E100000B20DF03FFCB4F9041048432168098802
:108E200001EBE030ADF8040040E020680088ADF8C8
:108E300000002068A18840880844ADF80600B4F915
:108E400006000DF027FCB4F90410B4F90E20891ABD
:108E500048432168498801EBE030ADF80200E08822
:108E60005A3000B20DF016FCB4F9041032464843F3
:108E70002168098801EBE030ADF804006946084636
:108E8000FBF75AFA30B1A0698560D4E90520216961
:108E900005F0EAFEA08970BB2068A188008808441C
:108EA000ADF8040020684088ADF80200B4F908006D
:108EB0000DF0F0FBB4F9041048432168498801EB38
:108EC000E030ADF8060020895A3000B20DF0E2FB28
:108ED00002E015E012E00FE0B4F90410B4F90E203E
:108EE000891A484321683246098801EBE030ADF821
:108EF000000069461AE024E0022801D0012820D1B0
:108F0000206832460088ADF8000020684088ADF83F
:108F100002002068A18800880844ADF80400206899
:108F2000A18840880844ADF8060029460846FBF7AA
:108F300003FA30B1A0698560D4E90520216905F004
:108F400093FEA06986607CBD7CB50446806961891A
:108F50006D468668A08901290CD0012867D081421E
:108F600003D12289E3889A427ED300297DD0032948
:108F70007CD0B5E0012822D1E088218988421ED228
:108F8000B4F906000DF086FBB4F9041048432168DB
:108F9000498801EBE030ADF80600E0885A3000B2B5
:108FA0000DF078FBB4F90410B4F90E20891A484387
:108FB0002168098801EBE030ADF8040042E0206848
:108FC000A1880088401AADF8000020684088ADF8FC
:108FD0000200B4F906000DF05DFBB4F9041048433B
:108FE0002168498801EBE030ADF80600E0885A308E
:108FF00000B20DF04FFBB4F90410B4F90E20891A39
:10900000484321683246098801EBE030ADF804009E
:1090100069460846FBF790F930B1A0698560D4E94C
:109020000520216905F020FEA089012858D120687B
:109030000088401EADF804002068A18840880844DC
:10904000ADF80600B4F908000DF024FBB4F90410E3
:10905000B4F90E20891A48432168498801EBE030B1
:10906000ADF80200208902E018E010E014E05A3068
:1090700000B20DF00FFBB4F90410324648432168EA
:10908000098801EBE030ADF8000069461DE00228D8
:1090900004D0032802D023E0022821D12068A1882F
:1090A00032460088401AADF8000020684088ADF8CC
:1090B000020020680088401EADF804002068A188E6
:1090C00040880844ADF8060029460846FBF734F905
:1090D00030B1A0698560D4E90520216905F0C4FD9F
:1090E000A06986607CBD7CB50446806961896D4657
:1090F0008668A08902290CD002287ED0814203D143
:109100002289E3889A4279D3002978D0012977D03F
:10911000D4E002283FD1E088218988423BD25A30EE
:1091200000B20DF0B7FAB4F9041048432168098879
:1091300001EBE030ADF80000B4F906000DF0AAFA3A
:10914000B4F90410B4F90E20891A484321684988FB
:1091500001EBE030ADF80600B4F908000DF09AFA22
:10916000B4F9041048432168498801EBE030ADF8B8
:10917000020020895A3000B20DF08CFAB4F90410C4
:10918000B4F90E20891A48432168098801EBE030C0
:10919000ADF8040066E020680088401EADF80400C9
:1091A0002068A1884088401AADF80200E0885A3053
:1091B00000B20DF06FFAB4F9041048432168098831
:1091C00001EBE030ADF80000B4F906000DF062FAF2
:1091D000B4F90410B4F90E20891A484321683246C4
:1091E000498801EBE030ADF8060069460846FBF718
:1091F000A3F858B1A069856003E00AE03BE034E0E1
:1092000036E0D4E90520216905F02EFDA089022869
:1092100054D12068A1880088401AADF80000206869
:109220004088401EADF8060020895A3000B20DF08B
:1092300031FAB4F90410B4F90E20891A48432168B0
:10924000098801EBE030ADF80400B4F908000DF036
:1092500021FAB4F9041048432168498801EBE03051
:10926000ADF80200324669461DE0032803D025E030
:10927000032800D010BB2068A18832460088401A1D
:10928000ADF800002068A1884088401AADF80200BF
:10929000206829460088401EADF8040020684088F8
:1092A000401EADF806000846FBF746F830B1A0694D
:1092B0008560D4E90520216905F0D6FCA0698660A7
:1092C0007CBD7CB50446806961896D468668A0894D
:1092D00003290ED0032867D0814203D12289E38875
:1092E0009A427ED302297DD001297CD002297BD0ED
:1092F000B1E003281FD1E088218988421BD25A306F
:1093000000B20DF0C7F9B4F90410B4F90E20891AAF
:1093100048432168098801EBE030ADF80000B4F95A
:1093200006000DF0B7F9B4F90410484321684988E4
:1093300001EBE03040E02068A18800880844ADF8E7
:10934000040020684088401EADF80600E0885A30CE
:1093500000B20DF09FF9B4F90410B4F90E20891A87
:1093600048432168098801EBE030ADF80000B4F90A
:1093700006000DF08FF9B4F9041032464843216815
:10938000498801EBE030ADF8020069460846FAF77B
:10939000D3FF30B1A0698560D4E90520216905F0CB
:1093A00063FCA089032856D120680088ADF800002E
:1093B0002068A1884088401AADF8020020895A3000
:1093C00000B20DF067F9B4F9041048432168098828
:1093D00001EBE030ADF80400B4F908000DF05AF9E3
:1093E00003E016E010E013E00FE0B4F90410B4F964
:1093F0000E20891A484321683246498801EBE03043
:10940000ADF8060069461BE018B1012801D022E042
:1094100008BB206832460088ADF800002068A188AB
:109420004088401AADF802002068A18800880844EE
:10943000ADF80400206829464088401EADF80600BB
:109440000846FAF779FF30B1A0698560D4E90520B4
:10945000216905F009FCA06986607CBD70B5A4B0E7
:109460000C46054620AA22A90AF0A9F822A803F072
:1094700034FF20B920A803F030FF00283ED012A905
:1094800028460FF042FA012838D12146684609F0F3
:1094900095FC1B4801900220029012A804904FF402
:1094A00080300D9022A803F018FF80B122A803900D
:1094B0006A461A21284606F053FE22AA12A920461F
:1094C00005F0D2FB6A461B21284606F049FE20A87B
:1094D00003F003FF002811D020AE6A461A21284667
:1094E000039606F03DFE20AA12A92046039605F039
:1094F000BBFB6A461B21284606F032FE24B070BD35
:1095000060AF01082DE9F74FB1F92E00AAB014465B
:109510000E46002872D096F8361002296ED901281E
:1095200008D1B6F93400002804DC308E10B9708EF2
:109530000028EFD02088318E4218B08E121AADF874
:109540002820A38819440144ADF82C106088738E3C
:109550001844B38EC01AADF82A00E388758E2B44E8
:10956000B58E2B44ADF82E30B6F92E5005EBD575DF
:10957000A2EB6502521EADF84C20012202EB6505FC
:109580002944ADF85010B6F92E1001EBD171A0EBC3
:109590006100401EADF84E00B6F92E0000EBD07011
:1095A00002EB60001844ADF8520096F8360029909E
:1095B000FD2801D9FF2029902A9813A9826827A89D
:1095C000FAF7BAFE0028A5D021461DA803F070FEC8
:1095D0004FF0FF38414642461DA803F0A4FEB6F9FD
:1095E00000901DA803F093FE04461DA803F069FE39
:1095F00084421DA803DA03F08AFE02E0FEE303F0D2
:1096000060FEB9EB600F01DD4FEA6009B6F900407A
:109610000AA803F07CFE05460AA803F052FE854224
:109620000AA802DA03F073FE01E003F04AFEB4EB8D
:10963000600F00DD4410B6F92E00051905FB05F09A
:10964000400008F057FD10900146B6F92E20234641
:109650000AA80FF079FA13A804F0DEFF012720B959
:10966000F078FF2801D3B07860B1002701234A4683
:109670001DA920A805F03CFA002120A804F0ECFD6B
:10968000269001E0CDF8988013A803F040FE08F082
:1096900031FD83461C2115A808F08CFECDF854D06E
:1096A000CDF860B0CDF868D0B08DADF85C0096F81C
:1096B00036008DF86C00B0788DF86D00BDF8500064
:1096C000BDF84C10ADF80400421A521C12B202EB65
:1096D000D27201EB62010FFA81FABDF85220BDF897
:1096E0004E10401B521A521C12B202EBD27201EB06
:1096F0006202401C14B200B26A1EADF80000ADF860
:109700000210114409B20992ADF8061052465045B4
:1097100000DC1046ADF80000A14200DB21462A988B
:10972000ADF806106946826806A8FAF705FED0B3C0
:109730004A461DA906A8FAF727FEA0BBBDF81C00E3
:10974000BDF91810BDF91A20401A401C00B208904B
:10975000BDF94E301098D21A02FB0500BDF9502019
:10976000521B891A0844401E059047B14A461DA95C
:1097700006A8FAF779FE10B101200F9000E00F97CC
:109780000898002827DDBDF81800ADF80000BDF8E6
:109790001C00ADF804000220CDF860B08DF8640024
:1097A000BDF91A8013E016E0ADF802800F98ADF80D
:1097B000068070B30598189015A92A9805F05EFCEC
:1097C00005982844059008F101000FFA80F8BDF9CA
:1097D0001E104145E8DABDF85000ADF80400401B0A
:1097E000401C00B2ADF80000BDF85220ADF80620D4
:1097F000511B491C09B2ADF802105246504500DC1D
:109800001046ADF80000601C1190814216DD08463C
:1098100015E0FFE72A465846059908F005FDBDF911
:10982000181042465846089B04F0B8FE8DF86400B4
:109830000128C1D102208DF86400BDE7601CADF89D
:1098400002002A986946826806A8FAF775FDD0B327
:109850004A461DA906A8FAF797FDA0BBBDF81C0053
:10986000BDF91810BDF90620401A401C00B208903E
:10987000BDF91E301098D21A02FB0500BDF9502028
:10988000521B891A0844401E059047B14A461DA93B
:1098900006A8FAF7E9FD10B101200F9000E00F973C
:1098A0000898002827DDBDF81800ADF80000BDF8C5
:1098B0001C00ADF804000220CDF860B08DF8640003
:1098C000BDF91E8013E016E0ADF802800F98ADF8E8
:1098D0000680B0B30598189015A92A9805F0CEFB1C
:1098E000059828440590A8F101000FFA80F8BDF909
:1098F0001A104145E8DDBDF84C0009992844ADF83F
:109900000000BDF85000401BADF80400BDF84E004B
:10991000ADF80200084400B2ADF80600A04200DB3A
:109920002046ADF806002A986946826806A8FAF72C
:1099300003FDB0B34A461DA906A8FAF725FDA8B154
:109940007BE0FFE72A465846059908F06DFCBDF913
:10995000181042465846089B04F020FE8DF864001B
:109960000128B9D102208DF86400B5E7BDF81C00CC
:10997000BDF81810BDF90220401A401C00B2089032
:10998000BDF91A101098891A01FB050005904FB116
:109990004A461DA906A8FAF767FD18B101200F90E5
:1099A00001E04AE00F970898002846DD0F9860B163
:1099B00000201890BDF81800ADF80000BDF81C009C
:1099C000ADF80400BDF91A0032E0CDF860B0F1E75F
:1099D000ADF802800F98ADF8068058B12998FF289D
:1099E0000598007803D096F836104843000A8DF8A1
:1099F0006C0013E00598089A0178584608F0A8FC16
:109A0000BDF9181042465846089B04F0C7FD8DF872
:109A10006400012802D102208DF8640015A92A985B
:109A200005F02CFB05982844059008F1010000B2D0
:109A3000BDF91E1080464145CADA96F836008DF809
:109A40006C00BDF84C002844ADF80000BDF8500093
:109A5000BDF85210401BADF80400481B401CADF887
:109A6000061000B21199ADF80200884200DC601CBB
:109A7000ADF802002A986946826806A8FAF75CFCED
:109A800078B34A461DA906A8FAF77EFC48BBBDF884
:109A90001C00BDF81810BDF91E20401A401C00B271
:109AA0000890BDF906101098891A01FB0500059071
:109AB000089800284FDD3FB14A461DA906A8FAF7CD
:109AC000D3FC0020189001E0CDF860B0BDF818007C
:109AD000ADF80000BDF81C00ADF80400BDF91E0093
:109AE00034E038E0ADF80280ADF8068087B14A4630
:109AF0001DA906A8FAF7B8FC2998FF280598007850
:109B000003D096F836104843000A8DF86C0013E035
:109B10000598089A0178584608F01AFCBDF9181003
:109B200042465846089B04F039FD8DF86400012830
:109B300002D102208DF8640015A92A9805F09EFA3A
:109B4000059828440590A8F1010000B2BDF91A104B
:109B500080464145C6DD96F836008DF86C00BDF8AC
:109B60005000ADF80400411BBDF84E00491C0AB27C
:109B70002844ADF8002000B2ADF80200BDF8521044
:109B8000119B491B09B2ADF80610984200DB601C1E
:109B9000ADF80200A14200DC2146ADF806105046A7
:109BA000524500DC02462A98ADF8002069468268DA
:109BB00006A8FAF7C1FBB8B34A464E461DA906A847
:109BC000FAF7E2FB80BBBDF81C00BDF91810099A3A
:109BD000401A401C00B20890109802FB0500BDF925
:109BE0005020521B891A0844401E0590EFB132469E
:109BF0001DA906A8FAF738FC10B14FF0010800E0E3
:109C0000B846059818900898002835DDBDF818006A
:109C1000ADF80000BDF81C00ADF8040002208DF87E
:109C20006400BDF91A6023E026E0B8465846E9E72B
:109C3000ADF80260ADF80660B8F1000F12D15846D9
:109C4000089A059908F0F0FABDF9181032465846FE
:109C5000089B04F0A3FC8DF86400012802D10220C7
:109C60008DF8640015A92A9805F008FA761C36B21A
:109C7000BDF91E00B042DBDA0020109A17E000BFE9
:109C800002EB050EAEF10101002305EBD57608E0ED
:109C900092F800C091F8008002F8018B01F801C928
:109CA0005B1CB3EB660FF3DB401C724600B2A842AC
:109CB000E6DBBDF84C000999ADF800000844BDF89A
:109CC0004E1000B2294409B2ADF80210BDF852207E
:109CD000119B521BADF8040012B2ADF80620994258
:109CE00000DB611CADF80210A24200DC2246AAF1A2
:109CF0000101ADF806200C91884200DB0846ADF862
:109D000004002A986946826806A8FAF715FBA8B3EA
:109D10004A464E461DA906A8FAF736FB70BBBDF8A9
:109D20001C00BDF91810099A401A401C00B2089096
:109D3000109802FB0500BDF90020891A084405901F
:109D4000EFB132461DA906A8FAF78EFB10B14FF00D
:109D5000010800E0B846059818900898002835DDFD
:109D6000BDF81800ADF80000BDF81C00ADF8040007
:109D700002208DF86400BDF91A6023E026E0B846A1
:109D80005846E9E7ADF80260ADF80660B8F1000F9B
:109D900012D15846089A059908F046FABDF91810EC
:109DA00032465846089B04F0F9FB8DF86400012800
:109DB00002D102208DF8640015A92A9805F05EF9F9
:109DC000761C36B2BDF91E00B042DBDABDF84C009D
:109DD0000999ADF800000844BDF84E10099AADF895
:109DE0000210114400B20C9AADF8040009B2ADF8AB
:109DF0000610904201DBAAF1010000E056E1ADF847
:109E00000400A14200DB21462A98ADF806106946FD
:109E1000826806A8FAF790FAC0B34A461DA906A8B8
:109E2000FAF7B2FA90BBBDF81C00BDF91810BDF9E5
:109E30001A20401A401C00B20890BDF90230109858
:109E4000D21A02FB0500BDF90020891A01EB0008B7
:109E500047B14A461DA906A8FAF706FB10B1012032
:109E60000F9000E00F970898CDF860B0002822DD31
:109E7000BDF81800ADF80000BDF81C00ADF80400F6
:109E800002208DF86400BDF91A6010E013E000BFF5
:109E9000ADF802600F98ADF80660C8B3CDF86080E9
:109EA00015A92A9805F0EAF8761CA84436B2BDF93F
:109EB0001E00B042ECDABDF84C00ADF80000099984
:109EC000BDF85220084401B2501BADF80410401CEC
:109ED000ADF8062000B2119AADF80200904200DC05
:109EE000601CADF802000C98814201DBAAF101016F
:109EF0002A98ADF804106946826806A8FAF71CFA99
:109F0000C8B34A461DA906A8FAF73EFAA8B15AE016
:109F1000FFE72A464146584608F086F9BDF9181071
:109F200032465846089B04F039FB8DF8640001283E
:109F3000B6D102208DF86400B2E7BDF81C00BDF96F
:109F40001810BDF90620401A401C0FFA80FABDF91E
:109F50001E301098D21A02FB0500BDF90020891AA4
:109F60000E184FB14A461DA906A8FAF77DFA18B196
:109F70004FF0010801E026E0B846CDF860B0BAF134
:109F8000000F20DDBDF81800ADF80000BDF81C0082
:109F9000ADF8040002208DF86400BDF91E400EE00B
:109FA000ADF80240ADF80640B8F1000F2FD018967A
:109FB00015A92A9805F062F8641E2E4424B2BDF952
:109FC0001A00A042ECDDBDF84C0069462844ADF80B
:109FD0000000BDF85000401BADF80400BDF84E0075
:109FE000CDF860B02844ADF80200BDF85200401B27
:109FF000ADF806002A98826806A8FAF79DF9E8B33A
:10A000004A461DA906A8FAF7BFF9A0B141E02A46C1
:10A010003146584608F008F9BDF918105346224653
:10A02000584604F0BBFA8DF864000128C0D1022024
:10A030008DF86400BCE7BDF91C10BDF918000A1AC0
:10A04000521C15B2002D24DDADF80410ADF800004F
:10A05000BDF91A4019E000BFADF80240ADF8064066
:10A060002946584608F0D4F9BDF918102B46224667
:10A07000584604F093FA8DF8640000E009E015A951
:10A080002A9804F0FBFF641C24B2BDF91E00A04214
:10A09000E2DA2FB920A804F0A3FA269804F0D4FD40
:10A0A000109808F073F8584608F070F82DB0BDE825
:10A0B000F08F00002DE9F041040006D0184E306802
:10A0C00084420AD10020BDE8F081502080F311883D
:10A0D000BFF34F8FBFF36F8FFEE70FF0D7FD6569BA
:10A0E000776BB66B0FF0F2FDBD4201D0B54201D1E6
:10A0F0000220E8E70B48854208D1A06A0028F7D182
:10A1000094F858000128F3D00320DCE70548143800
:10A11000854202D00DB10120D5E70420D3E700002D
:10A120001C000020A40900202DE9FF5F0C46934687
:10A1300080462021DDF838A00AF034F8002878D0D5
:10A14000BAF1030F40461DD009F01DFA814607F011
:10A1500091F9002705463E46BAF1030F39464046BD
:10A1600013D009F08BFE82460021404609F038FEEC
:10A170004946B9F1010F5DD0022963D0B9F1030F4F
:10A1800066D13BE009F0F8F9E0E709F047FE8246C6
:10A190000021404609F054FE4946B9F1010F1ED096
:10A1A000022924D0B9F1030F52D1B8F81820B8F819
:10A1B0001410521A521C13B2A3EB0A02101A00EB2D
:10A1C000D0720AEB6200084407B2298BA88A091AE8
:10A1D000491C09B201EBD17100EB610027E0B8F82E
:10A1E0001410B5F9146001EB0A0007B230E0B8F8BA
:10A1F0001810B5F91860081A07B229E0B8F81A2043
:10A20000B8F81610521A521C13B2A3EB0A02101A15
:10A2100000EBD0720AEB6200084407B2688BE98A4F
:10A22000401A401C00B200EBD07001EB600006B297
:10A230000EE02FE0B8F81610B5F9166001EB0A0031
:10A2400007B205E0B8F81A10B5F91A60081A07B293
:10A25000A01E039900B2002910DAB9F1000F15D041
:10A26000BE4221DC12E0002C01DDA41C24B2E01768
:10A2700004EB9070801004B0BDE8F09FBBF1000FBC
:10A2800012DAB9F1000F01D0BE420DDB002CEADA80
:10A290000446E8E70398E04202D50398404204B23E
:10A2A000BBEB040000D55C462046E4E770B50446ED
:10A2B00007F0D0F848B1006882680AB1217A904767
:10A2C000207E810742D4C0077BD10021606808F05E
:10A2D000F3FF002518E0017A0A0610D5802904D082
:10A2E000227A21F08001914209D14168E160016840
:10A2F00020468847207E810728D4C00761D16D1C85
:10A300002946606808F0D8FF18B101680029F6D026
:10A31000E1E72146002008F0FDFE050053D00021B2
:10A32000606808F0C9FF002619E0016891B1017A60
:10A330000A060FD411B1227A91420BD14168E16033
:10A34000016820468847207E810701D5012070BD25
:10A35000C00736D1761C3146606808F0ADFF10B1F9
:10A36000012DE2D02FE0012D2DD16068416851B35D
:10A37000217E490727D4217A232919D0242917D0EF
:10A38000A90309F00FFFF0B1207A11381C280FD271
:10A39000DFE800F019191919191919191919190EE5
:10A3A0000E190E0E191919190E0E0E0E19190E1975
:10A3B0006068406860602046FFF778FF0546012826
:10A3C00001D0002070BD284670BD00002DE9FF4F70
:10A3D0008A880B8889B0D21A521C17B2CA88498859
:10A3E0000446511ADDE916B8491C19980FFA81F98B
:10A3F000012813D0022813D0032843D1434E00BFB5
:10A400005FEA08000ED0002006902088ADF8140006
:10A4100098F80000FD2838D35A4639E03C4EEFE763
:10A420003C4EEDE72088ADF80000ADF808005A4634
:10A4300000990C98B0470590002020E0002517E017
:10A44000BDF8080034F8151088420BD004EB450025
:10A450005A460088ADF81400ADF8080005990C982C
:10A46000B047059004EB4500BDF8141001806D1C49
:10A47000BD42E5DB0B9804EB400408F10100804687
:10A480004845DBDB0DB0BDE8F08F00FB0BF0020AA6
:10A4900005990C98B0470890002033E0002528E08B
:10A4A00018F8050020B30699884205D1BDF81410AC
:10A4B00034F81520914216D0FD2801D35A4602E007
:10A4C00000FB0BF0020A04EB45000088ADF8180011
:10A4D00006990C98B047089018F80500069034F8D3
:10A4E0001500ADF8140004EB4500BDF82010018004
:10A4F0006D1CBD42D4DB0B98189904EB40048844D2
:10A500000AF1010082464845C8DBBBE78B6C0008B6
:10A51000176C0008EB6C00082DE9FF4F0446888893
:10A520000A8883B0801A401C05B2C8884988DDE9D2
:10A5300010A6401A401C0FFA80F976B1BDF8180039
:10A54000BAF1FD0F00EB004000907CD3A5F10408A8
:10A550004FF0000BBDF818A033E1BAF1FD0F0FD397
:10A56000002608E02A462046069902F0DDFF0598FD
:10A57000761C04EB40044E45F4DB07B0BDE8F08FD9
:10A58000BDF80010002060F3040189B260F34A11A5
:10A5900089B260F3CF21ADF8001088B20090BDF809
:10A5A0000000009001465246069803F085F801909D
:10A5B0000AF104000699C008C00689B2000ECA0A52
:10A5C000424362F30F06C1F34512424301F01F01FB
:10A5D000414361F30F0762F31F46BA46C0F1FF0122
:10A5E00000224CE0002044E0BDF8007034F8103048
:10A5F0009F4238D004EB4003B7B21B88ADF800305F
:10A60000ADF808309BB24FEAD32C0CFB017707EB77
:10A61000C71C0CEBC737BDF80480C7F3C45767F3FA
:10A62000CF28C3F3451C370C0CFB017707EBC71C85
:10A630000CEBC737C7F3C55767F34A181FFA8AF7F9
:10A6400003F01F0300E0C3E003FB017303EBC31738
:10A6500007EBC333C3F3C45363F30408ADF80480BA
:10A660001FFA88F3019304EB4003BDF804701F80C8
:10A67000401CA842B8DB0598521C04EB40044A4534
:10A68000B0DB7AE7002710E03278FF2A12D020886A
:10A69000ADF804000199069803F00EF80190BDF89A
:10A6A00004002080A41C761C7F1CAF425EDAB00739
:10A6B000EAD15BE0A4F800A0F4E73068411C44D084
:10A6C000F0B33278FF2A54D02088ADF80400019905
:10A6D000069802F0F1FF0190BDF80400A4F8000014
:10A6E00016F8012FA41CFF2A46D02088ADF80400DC
:10A6F0000199069802F0E0FF0190BDF80400208067
:10A7000016F8012FA41CFF2A39D02088ADF80400C8
:10A710000199069802F0D0FF0190BDF80400208056
:10A7200016F8012FA41CFF2A2CD02088ADF80400B5
:10A730000199069802F0C0FF0190BDF8040000E006
:10A7400011E02080A41C761C0FE0A00707D0A4F81D
:10A7500000A0022000990151A4F806A003E000988F
:10A760002060009860600834361D3F1D4745A4DD19
:10A770001CE0A4F800A0B3E7A4F800A0C0E7A4F888
:10A7800000A0CDE7A4F800A0DCE73278FF2A1CD0B7
:10A790002088ADF804000199069802F08DFF019021
:10A7A000BDF804002080A41C761C7F1CAF42ECDBAB
:10A7B00005980BF1010B401B04EB40041298401B61
:10A7C0000644CB45FFF65EAFD7E6A4F800A0EAE763
:10A7D00000222188ADF800109346104633E0002790
:10A7E00027E0307818B3904205D0FF282FD000FB27
:10A7F0000AF31B0A9B46904203D134F817008142AA
:10A8000010D0BBF1FF0F24D004EB47005A4600885C
:10A81000ADF800000099069802F04EFF00903278E3
:10A8200034F8171004EB4700BDF800300380761CA5
:10A830007F1CAF42D5DB059804EB40041298401B07
:10A84000064408F1010080464845C8DB95E65346BA
:10A85000D0E70698E2E700002DE9FF4F83B00C46F1
:10A86000DDF84480FAF7D4FDBDF818A08146B8F1B0
:10A87000000F0CD0A0882188401A401C07B2E08845
:10A880006188401A401C0FFA80FB002641E0B4F9B1
:10A89000026017E0B4F900500FFA86F80DE0109846
:10A8A0000290ADF804A0CDF80080D9F800002BB2DA
:10A8B000059AC7690399B8476D1CB4F90400A8420A
:10A8C000EDDA761CB4F90600B042E3DA07B0BDE871
:10A8D000F08F002518E000BF18F8050098B1109916
:10A8E000ADF804A04843000A029060880399304400
:10A8F00000B200902088059A284403B2D9F80000DD
:10A90000D0F81CC0E0476D1CBD42E5DB1298761CF8
:10A9100080445E45DDDBD9E700680968884201D1E3
:10A92000012070470020704740680A6820F04040CE
:10A93000904200D20860002070472DE9F04F4FF0A0
:10A94000000991B00446CB4606F084FD0068CA4673
:10A95000007E0290D4F82480CDF81CA0208BA18A20
:10A9600008442083608BE18A08446083DDE000278F
:10A970004FF4807546460A970FE00021304609F0F3
:10A980001CFB384407B20021304609F028FB454340
:10A990002D12304608F0CCFC0646002EEDD1A06901
:10A9A000019017B9B5F5807F09D0784201B24FF414
:10A9B000803090FBF5F20AAB01A80AF025FFBDF943
:10A9C0000410002900DC4942BDF90600002800DC23
:10A9D000404281424FF0010001DD824600E00790D5
:10A9E0001021404609F0DEFB00287ED0079D574627
:10A9F0002E464046CDF800A008F0F8FCC10700D173
:10AA00000027810701D400210091410700D40025CF
:10AA1000000700D40026404608F0BCFD0F904046D9
:10AA200008F092FC0E90404608F0E8FC0D9040467D
:10AA300008F044FD0F99002902DC0E9900290FDD72
:10AA400025B1BDF9062002998A4206DA46B102997B
:10AA5000BDF9062049428A4202DCC1464FF00C0B88
:10AA60000D99002901DC002810DD27B1BDF9042073
:10AA700002998A4207DA009941B10299BDF904208E
:10AA800049428A4202DCC1464FF0030B0F9900296C
:10AA900000DC00250E99002900DC00260D99002914
:10AAA00000DC0027002801DC0020009027B1BDF960
:10AAB00004100298814214DA009828B10298BDF976
:10AAC0000410404281420CDD25B1BDF90610029808
:10AAD000814206DA4EB10298BDF906104042814229
:10AAE0000EDCBAF1000F03D000E009E0032100E022
:10AAF0000C2194F8400061F3030084F8400018E052
:10AB00004FF48071404609F04DFB3AEA000010D145
:10AB10004FF40071404609F045FB01460798884311
:10AB200007D1404608F004FC8046B8F1000F7FF4DE
:10AB30001EAFB9F1000F0AD094F8401000206BF35B
:10AB4000030184F84010C4F82C902083608311B076
:10AB50004846BDE8F08F00002DE9FF4F83B08B46DB
:10AB6000824608F009FD060012D041F6FF784446FF
:10AB70000021504609F052F900900021504609F09A
:10AB80005FF90190504608F0EDFA074600255FE0B6
:10AB9000002007B0BDE8F08FDAF8080031490068FE
:10ABA00050F82500814609F004FBE8BB4FF48051C2
:10ABB000484609F0F7FAB8B3012E04D0022E08D0A7
:10ABC000032E44D11AE0B9F91400BAF81420009900
:10ABD00032E0BAF818200199B9F91800511A069A0A
:10ABE00009B2104400B2584531DB059A90422EDC80
:10ABF000401A00B2002821DD014620E0B9F81820F3
:10AC0000B9F81410BAF81830501A401C00B200EB12
:10AC1000D070BAF8142001EB6000991A491C0BB2ED
:10AC2000009900B25B1A00E011E00199591A01EB9A
:10AC3000D173009901EB63011144D0E74142002C2C
:10AC400001DD224600E06242914200DA04466D1CBA
:10AC5000BD42A1D3444501D1002000E0604200B2D2
:10AC600097E70000010004002DE9FF4F83B08B46F9
:10AC7000824608F088FC060012D041F6FF78444670
:10AC80000021504609F0FAF800900021504609F0E2
:10AC9000A7F80190504608F065FA074600255FE0E6
:10ACA000002007B0BDE8F08FDAF8080031490068ED
:10ACB00050F82500814609F07CFAE8BB4FF480513A
:10ACC000484609F06FFAB8B3012E04D0022E08D01E
:10ACD000032E44D11AE0B9F91600BAF816200099EB
:10ACE00032E0BAF81A200199B9F91A00511A069AF5
:10ACF00009B2104400B2584531DB059A90422EDC6F
:10AD0000401A00B2002821DD014620E0B9F81A20DF
:10AD1000B9F81610BAF81A30501A401C00B200EBFD
:10AD2000D070BAF8162001EB6000991A491C0BB2DA
:10AD3000009900B25B1A00E011E00199591A01EB89
:10AD4000D173009901EB63011144D0E74142002C1B
:10AD500001DD224600E06242914200DA04466D1CA9
:10AD6000BD42A1D3444501D1002000E0604200B2C1
:10AD700097E70000010004002DE9FF4F83B00E4665
:10AD8000DDE910B417460021039809F034F90546AF
:10AD90000021039808F0CAFF0146F07882070BD51E
:10ADA000C30742F2D17202D0954202D006E091422E
:10ADB00006D120F00200F070C00701D07B4800E00F
:10ADC0007B488146F078C00712D079484FF0000ADE
:10ADD000A4F802A0A4F804A0C4F810A0A4F800A04D
:10ADE000C4F808A0C4F80CA0804639460197A9E031
:10ADF0006E48EBE70198B84206D04FF400012846B0
:10AE000009F0D0F900286FD16A49284609F0D1F934
:10AE100000286AD10021284608F078FF029070B31C
:10AE20002069401C2061A28802EB0B01A180217DDA
:10AE3000C9076DD000EB8000800007F05BF900903F
:10AE4000E0B1E16851B12069401E00EB8000820052
:10AE5000009807F0E9F9E06807F098F9206900EB3D
:10AE60008001009800EB81004FF0000140F8145C75
:10AE7000F078C007284603D0022202E0FEE735E062
:10AE8000052209F00DF8216900B201EB8102009959
:10AE900001EB820121F8100CF0784FF00001C0079F
:10AEA000284601D0032200E0062208F0F9FF2169BC
:10AEB00000B201EB8102009901EB820121F80E0C36
:10AEC0002069029900EB8002009800EB820040F8B4
:10AED000081C206900EB8002009800EB820040F81B
:10AEE00004AC0098E06013E032E020E028464946D8
:10AEF00088470146F078800705D5B4F90400421868
:10AF00000698824224DCA28801EB0B001044A0804A
:10AF10002846414688470146B4F90000814202DDD7
:10AF20002846414688472080A068401CA060F078F1
:10AF3000400702D54FF0FF3000E001200199411891
:10AF4000019105D4039808F0FBF8051E7FF452AF79
:10AF5000B4F90400002802DDA0EB0B00A0802069FA
:10AF600008B1069801E0B4F904006080CDB1019801
:10AF7000B84216D1039901AA8968096851F820508E
:10AF8000F078C0F38001039800F0BCFB4DB1284677
:10AF900041468847208028464946884760800120EE
:10AFA000A060019807B0BDE8F08F0000994101084A
:10AFB000E3320108010006002DE9F04FB14D93B0D6
:10AFC000044600216A8808F06BFF9DF81710421CA8
:10AFD00062F30001820862F34101C00860F382015C
:10AFE0008DF8171020460021AA8808F059FF8DF827
:10AFF000140020460021EA8808F052FF8DF8150061
:10B00000204600212A8908F04BFF8DF81600002108
:10B01000204608F03AFE012800D0002081469DF825
:10B0200017004FF00001C00720460CD008F01AFFAF
:10B0300082469DF817004FF00001C007204605D05A
:10B0400008F0E0FE04E008F0DDFEF1E708F00AFF9A
:10B0500007909DF81700C007204602D008F0EEF8D0
:10B0600001E008F0D1F8069020460021322208F0D5
:10B0700017FF054620460021102208F011FFE18A43
:10B0800028444618204608F093FA301AADF82000FC
:10B0900020460021122208F003FFA18A2844451807
:10B0A000204608F07EFA281AADF840009DF81700F7
:10B0B0009DF81660C00701D008AD00E010AD00217A
:10B0C000204608F098FF11900021204608F02EFE3F
:10B0D00083469DF81700C10708D0ABF51C52D13A42
:10B0E00002D1618C490509D5C10708D1119AA2F591
:10B0F0001C51D13903D1618C090500D40026B9F166
:10B10000000F08D0C00706D116B1012E02D002E010
:10B11000012600E000260027ADF83C70B8468EB34B
:10B120009DF81700400703D5A0684268521E15E03D
:10B13000002213E000200E9009A90798CDE9000134
:10B1400005A92046069BFFF717FE0246BDF824100E
:10B1500007EB0A00084407B208F10108A06840683C
:10B16000904201DD002AE5DAB8F1000F02D0A7EB2A
:10B170000A0007B29DF81700C007204603D008F068
:10B1800043F802E00BE008F059F80FA9CDE90051AF
:10B1900001460FFA88F33A4630460CF036F99DF82E
:10B1A0001700410703D5A1684E68761E00E000260F
:10B1B000B9F1000F04D0C00702D128883844288094
:10B1C00009AFA0684068B04249DD002E47DB01208E
:10B1D0000E900798CDE90007324605A92046069B48
:10B1E000FFF7CAFD8046B9F1000F08D09DF817009F
:10B1F000C00704D12888BDF82410401A2880DDE952
:10B200000601BDF9202002AB019283E88300BDF95D
:10B21000400000904346324605A92046FBF79AF9C4
:10B2200046460C9806F0B2FF00200C90B9F1000FD2
:10B2300003D09DF81700C0070AD02888BDF8241055
:10B24000BDF83C20014402EB0A0008442880B8E71E
:10B25000BDF83C20298802EB0A00081AF6E711998C
:10B2600042F2D170814201D0834502D1204609F0DB
:10B270005DFC00222B21204604F072FF13B0BDE8D4
:10B28000F08F0000E40000202DE9F74F0546007F15
:10B2900093464FF0000AC00760D14FF00108EC68F8
:10B2A0000026C1467CB9287FC0F3C000401E304252
:10B2B00054D1B9F1000F51D00199284688474FF079
:10B2C00000080446C1460EB9261E47D0B8F1000F4B
:10B2D00006D0214628465A4690470446B0423DD003
:10B2E0004FF00108002CDED0206808F0B1FC000609
:10B2F000D8D427681FE00121384608F053FFB0B1C9
:10B300002FB10121384608F04DFF0028CAD1E86866
:10B31000A04223D0B0B1284600F0E4F80246E86825
:10B320000F21006804F01CFF012817D106E0384601
:10B3300007F0FEFF0746002FDDD1E8E7E868006868
:10B3400009F016F92846EC6000F0CCF80246E868EF
:10B350000E21006804F004FF012802D05046BDE829
:10B36000FE8FE868006809F003F9296909B12846E9
:10B3700088470120F3E7B0F90C00032101EB4000FE
:10B3800020F0030010307047024A0021528808F074
:10B3900087BD0000F0000020034A10B5002152894B
:10B3A00008F07EFDC0B210BDF0000020034A10B5C9
:10B3B0000021928908F074FDC0B210BDF000002099
:10B3C0002DE9FC470F0023D0046962692AB1106897
:10B3D000B84202D15068BDE8FC87608A00214FF076
:10B3E000040CC0F308030CE0A66801EB810556F8D5
:10B3F00025000CEB8505755B381A85420AD2491C7D
:10B4000089B28B42F0D81AB1176061690020486098
:10B410000020E0E701EB81051221A26801EB850124
:10B420000026515C4FF0060802290BD04FF00C0AA1
:10B4300061B1DFF8ACC01022082303290FD0012925
:10B4400027D045E008EB8501515A40E00AEB850121
:10B4500008EB85035158D25A085C161838E0ADF84D
:10B460000400CDF800C0A06802EB850103EB85095C
:10B47000425A50F80910022301A8FAF7B9F838B374
:10B48000A16851F80920801A08EB85024010895AFA
:10B490001DE0ADF80400CDF800C0A06802EB850106
:10B4A00003EB8509425A50F80910022301A8FAF764
:10B4B0009FF868B1A16808EB850351F80920801A4C
:10B4C0000AEB850240108A58C95A32F810000E184B
:10B4D000606910B107606069466030467BE7000034
:10B4E000CD9B01082DE9F041002607463546304640
:10B4F00010E000BF05F0DFFF616DB94209D10228FD
:10B5000002D0042803D003E02046BDE8F08126469F
:10B510002546204605F0A4FF0400EBD10EB13046CD
:10B52000F3E70DB12846F0E7BDE8F041002005F053
:10B5300097BF00007CB50369006900255B8AC46879
:10B540009E04A3682BD4980F17D00120B0EB937FF3
:10B5500031D101EB02402668019018480090A068A4
:10B56000042320F04042314601A8FAF741F810B315
:10B57000801B801061680D561DE001EB02202668DB
:10B58000ADF804000E4823F04042009002233146FB
:10B5900001A8FAF72DF870B1801B4010EAE7606847
:10B5A000405C995C38B131B1637B2268401E00FB7E
:10B5B0000320491E455628467CBD00004BCB0008A1
:10B5C0005FCB00082DE9F04105460F46698C00204D
:10B5D0000426C1F30513EA680FE000BF06EBC004C0
:10B5E00014595FEAC41C07D524F07F44BC4203D140
:10B5F00052F83000BDE8F081401C8342EED84FF095
:10B60000806000EBB1204FEAB0506884C0F30510B1
:10B61000C100104606F0F0FDE860C0B3688CC0F3CE
:10B620000514641E16D06FF003025300E86802EBA5
:10B63000C40141585FEAC11C0CD489010AD403EB50
:10B64000C40C00EBC4018444641EDCE9000CC1E9B5
:10B65000000CEBD1E868082100EBC40006F0AAFE5C
:10B66000082006F019FDE96841F834000AF00DFBE6
:10B67000EA6806EBC400115841F080711150EA6885
:10B6800067F317011150E86850F83400B2E7FFE79C
:10B69000FEE700002DE9FC410068C068C068B0FB0F
:10B6A000F1F4944200DD1446154F78680068806913
:10B6B00020B30020ADF80000ADF80400ADF80200A2
:10B6C00025B2681E06B2ADF8066078686946006863
:10B6D00082699047BDF80600BDF80210401A401C70
:10B6E00000B2A04202DD351EEBDC01E0002D02DCE1
:10B6F0000020BDE8FC81BDF90640641C2046F8E747
:10B70000C8000020136821B15B1E13600BD4806851
:10B7100005E05B1C1360806841688B4203DA0068B7
:10B7200050F823007047002070472DE9FF4F83B089
:10B7300005461F460598F9F772FE0146012088402C
:10B74000B5F8209000F0FF086FEA090080B2019080
:10B7500095F822004FF0FF36C0F3C00A00244FF0E6
:10B76000040B1FE0E96801EBC4004268920140D578
:10B77000BAF1000F15D10BEBC4028958049AC1F33A
:10B780000741090491420CD10068817911EA080F40
:10B7900007D06A4605990AF0D2F9012830D002286C
:10B7A00031D0641C688CC0F30510A042DAD820E0C8
:10B7B000E96851F83400827912EA080F18D00BEBCF
:10B7C000C4028A58C2F307411FFA82FA049A090494
:10B7D00091420DD1019A1AEA020F09D1B24507DD53
:10B7E0006A4605990AF0ABF901280FD002280AD061
:10B7F000641C688CC0F30510A042D9D8002E0EDB63
:10B8000000983860012007B0BDE8F08F5046CA4567
:10B81000F6D05645ECDA064600983860E8E7002096
:10B82000F1E72DE9F047814642F30006C0F15A00E6
:10B830001D460F46540800B2761C0AF02BFFA7EBFA
:10B84000040800FB08F0C71148460AF023FF00FB7C
:10B8500008F0C011002F06DD7F3F39120A1B324469
:10B860002A80214405E07F3739120A1B21442A80AF
:10B87000891BA980002806DD7F380012011B314496
:10B880006980204405E07F300012011B204469805C
:10B89000801BE880BDE8F087024A0021D28808F0CA
:10B8A000FFBA0000F0000020034A10B50021128A00
:10B8B00008F0F6FAC0B210BDF0000020034A10B53F
:10B8C0000021528A08F0ECFAC0B210BDF00000204E
:10B8D0002DE9F04104460D46668C00200423C6F392
:10B8E0000511E2680BE000BF03EBC007D7595FEA20
:10B8F000871C03D527F07F47AF4202D0401C81420E
:10B90000F2D8814203D002EBC000BDE8F0814FF0D5
:10B91000806000EBB6204FEAB0506084C0F30510A1
:10B92000C100104606F068FCE060608CC0F30510B2
:10B93000401E0DD06FF00702E16802EBC00601EB7C
:10B94000C0030E44401ED6E90016C3E90016F3D129
:10B950000821E06806F02EFD082006F09DFBE16856
:10B9600008600AF092F9E168486840F000704860A9
:10B97000E16865F317004860E068C6E738B50C4831
:10B980000D46144690F820004FF00201C0074FF01A
:10B99000120002D009F0F6FE01E009F00BFF22468A
:10B9A000294601F0BDFE0090BDF8000038BD000042
:10B9B000B05200202DE9F0474FF0000CDDE909649A
:10B9C000089DDDF82CA0E1466F1E09BB052A03D0B7
:10B9D000062A01D0042A02D10023012D01D0002122
:10B9E00009E001225FF000019C4436F81180491CF7
:10B9F000C4440FFA8CFCA942F6D3ACEB030109B2A4
:10BA0000072A2AD2DFE802F004070B2921160D00CD
:10BA1000A4F8009021E0411A01EBD17112E0411A23
:10BA200011E0411A09B23AB291FBF2F1A4F8009088
:10BA30000BB212E0411A09B22AB291FBF2F10BB239
:10BA400003EBD3714910218007E0411A0AB2691C47
:10BA500009B292FBF1F10BB2238000210BE000BF91
:10BA600034F8112036F811C0624404EB410C1A443A
:10BA7000ACF80220491CB942F2D304EB450106EBB5
:10BA8000450231F8021C32F8022C11442288891A2E
:10BA90000AB2BAF1000F0CD0002108E034F81130DE
:10BAA00036F81170C31ADB1B24F81130491CA94267
:10BAB000F4D31046BDE8F08770B58AB00446FFF7AE
:10BAC00063FC05462046FFF7E7FE002D5CD000280A
:10BAD0005AD069462046FAF703FA0C2107A806F067
:10BAE00069FC20460021322208F0DAF9054620469A
:10BAF0000021122208F0D4F9461920460021102214
:10BB000008F0CEF90544204607F04BFDA18A3144E8
:10BB1000081AADF82400204607F04AFDE18A2944BE
:10BB2000081AADF82600002507E0006807AA694654
:10BB300050F8250000F084FE6D1CA0684168A94201
:10BB4000F3D8009806F022FB019806F01FFB02983C
:10BB500006F01CFB039806F019FB0021204608F0B4
:10BB600050FA05460021204608F0E6F842F2D1716D
:10BB70008D4201D0884202D1204608F0D7FF002232
:10BB80002B21204604F0ECFA0AB070BD0021A0F190
:10BB90003002092A01D8D1B216E0612801D3203839
:10BBA000C0B2413806280FD2DFE800F003050709CC
:10BBB0000B0D0A2108E00B2106E00C2104E00D2109
:10BBC00002E00E2100E00F21084670472DE9F04108
:10BBD0000446806D0D4600282BD0A968022230F95A
:10BBE000217002EB8101465EA87B01280AD1B4F9DD
:10BBF0001000B84203D1B4F91200B04202D0201DA7
:10BC000000F0BEFC201D00F069FD002811D1278145
:10BC10006681A87B012804F104000CD000F0B0FC80
:10BC2000201D00F05BFD002803D12089208260895F
:10BC30006082BDE8F08100F0B1FBF1E770B5254C02
:10BC400005460421606808F0ADFA002828D0296B69
:10BC50006068814224D007F03FFB0646286B08B19C
:10BC600007F03AFB86421CD11EB1606804F098FED2
:10BC70000FE0286B40B10F21A26804F071FA28464A
:10BC800000F02CFD00280BD1D4E901020E2104F0B4
:10BC900067FA284600F022FD002801D16068286379
:10BCA00070BD78B12B6B53B1A26888B110211846D2
:10BCB00004F056FA284600F011FD0028F0D1002EBD
:10BCC000E2D0D2E7286B0028F9D00F21A268EFE775
:10BCD0000F21ECE7A80000202DE9F0470D460446AF
:10BCE000897B40794FF0000801292AD0010708D547
:10BCF00020F0080121F00101C4F84880617184F846
:10BD00000880277AA87B20726868E060D4F8549095
:10BD10005FEA09007ED004F0ADFEBF4E00287060DF
:10BD200078D0A87B08B1A5F80C80484604F0A2FEA4
:10BD3000706000286ED0A97B012905D000296AD047
:10BD40000EE1000766D4DCE717B1012F36D007E11A
:10BD50000AF0A2FAA06469680A2906D0142917D04B
:10BD6000132918D01B291AD024E0706808F03DFC74
:10BD700020B91021706808F015FA08B1012700E019
:10BD80000027484604F070FE8743D9D101216AE0BC
:10BD9000A889401E01E0A889401CA881E0E01B2181
:10BDA000484604F0D1FE201D00F098FC002831D157
:10BDB000202158E0484604F0C7FE58E06079C007EB
:10BDC0003ED1A06C0AF061FA2168898B88426079C3
:10BDD00034D940F0010060710AF05EFAE0646868EE
:10BDE0000A281CD1706808F000FC20B91021706886
:10BDF00008F0D8F9B8B1484604F043FE01280ED93E
:10BE0000484604F031FE80F00101484604F0ADFEE2
:10BE1000202101E090E030E0706806F0DDFD6079FF
:10BE200040F001009BE0D6E90102052104F098F9F9
:10BE3000201D00F053FC00287ED1F0E7C0071BD086
:10BE4000E06C0AF022FA2168C98B884214D90AF002
:10BE500023FAE06469680A2904D0142998D01329C8
:10BE6000A8D198E70621D6E9010204F079F9201D4E
:10BE700000F034FC00285FD172E0012F70D16968B6
:10BE80000A2967D108F0B1FB20B91021706808F0C9
:10BE900089F9A8B3484604F0E7FD002860794FEA25
:10BEA000C07052D020B1484604F0EBFD012847D8BD
:10BEB000D6E90102082104F053F9201D00F00EFC20
:10BEC00000286FD1D6E90102042104F049F9201DB0
:10BED00000F004FC002865D1D6E90102072104F036
:10BEE0003FF9201D00F0FAFB00285BD10A214846EB
:10BEF00004F02AFE201D00F0F1FB002852D129E0B9
:10BF0000FFE7D6E90102082104F02AF9201D00F01C
:10BF1000E5FB002846D16079C00704D1D6E90102CB
:10BF2000042104F01DF9201D00F0D8FB002839D1B0
:10BF3000D6E90102072100E034E004F011F9D9E765
:10BF40002021706806F048FD04E018B90121484638
:10BF500004F00BFEC4F84880607920F001006071A5
:10BF6000C6F80480A88900281CD0484604F07CFD4F
:10BF70000028B5F90C0029D0002815DA4FF000068A
:10BF80000BE000BF4FF01401484604F0DDFD201D1A
:10BF900000F0A4FB002805D1761CB5F90C00404246
:10BFA000B042EFDCBDE8F087FCDD002609E013219C
:10BFB000484604F0C9FD201D00F090FB0028F1D197
:10BFC000761CB5F90C00B042F1DCEBE7002811DA81
:10BFD0004FF0000608E0484604F02AFD201D00F05E
:10BFE0007DFB0028DED1761CB5F90C004042B04242
:10BFF000F1DCD7E7D6DD002608E0484604F0BAFCBD
:10C00000201D00F06BFB0028CCD1761CB5F90C008C
:10C01000B042F2DCC6E70000A800002070B504467C
:10C02000C06A002870D194F84100C0076CD14FF469
:10C030000046656A03E0284607F07AF90546002DB8
:10C0400062D03146284608F0ADF80028F3D1B4F9A3
:10C050001400002801DD014600E041422B4A9268AD
:10C0600013689B7E994209DAB4F91610002900DCA6
:10C070004942994202DA0021A187E187A18F084451
:10C0800000B2A087E18FE38A0028194409B2E18752
:10C0900001DD034600E043421668F67EB34206DC4B
:10C0A000002901DD0B4600E04B42B3422CDD0123A9
:10C0B00084F84130002801DD034600E043420029B6
:10C0C00001DD0E4600E04E42B34209DD002894F83F
:10C0D000400020F0F00001DD20300AE0103008E0E0
:10C0E00094F84000002920F0F00001DD803000E0ED
:10C0F000403084F840000C21284604F031F82046F6
:10C10000BDE8704000F0EABA70BD0000A800002051
:10C110002DE9F0470E460446897B40794FF0000830
:10C12000012923D0010708D520F0080121F00101E1
:10C13000C4F84880617184F80880D4F854905FEAAC
:10C1400009007CD004F096FC664D0028686076D02B
:10C15000802108F033F80746E1687068E060207AD3
:10C16000B27B2272B27B012A03D003E0000766D4BF
:10C17000E3E708B1AFB3B0E00AF08EF8A0647168ED
:10C18000092903D00B2909D087B1A6E00021484630
:10C1900004F0EBFC484604F0EDFB56E00021484675
:10C1A00004F0E3FC484604F043FC4EE00A2902D0C8
:10C1B0001B290BD016E00A21484604F0C5FC201DBF
:10C1C00000F08CFA00283AD1012137E01B214846C3
:10C1D00004F0BAFC201D00F081FA00287FD1202154
:10C1E0002CE003E0484604F0AFFC2EE0012A01D029
:10C1F00032B372E0012870D170680A2809D1D5E9FC
:10C200000102022103F0ACFF201D00F067FA0028B4
:10C2100065D16079C00720D1A06C0AF036F821689A
:10C22000898B8842607916D940F00100607170688E
:10C230000A2852D10AF030F80521E06401E04EE00E
:10C240001FE0D5E9010203F08BFF201D00F046FA44
:10C25000002844D141E0C0073FD0E06C0AF015F857
:10C260002168C98B884238D90AF016F8E0647168F1
:10C270000A2904D0092989D00B29B3D18EE70621D8
:10C28000DCE7012829D171600A2920D1D5E9010212
:10C29000082103F065FF201D00F020FA00281ED1C0
:10C2A0006079C00709D1D5E90102042103F058FFE4
:10C2B000201D00F013FA002811D1D5E90102072151
:10C2C00003F04EFF201D00F009FA002807D1C4F842
:10C2D0004880607920F001006071C5F80480BDE8F5
:10C2E000F0870000A800002070B5044600680D46E5
:10C2F00009880069A1826988E1820268117CC1F322
:10C300000111022901D003290AD111882A88891A2A
:10C31000491E298001686A884988891A491E6980EE
:10C320000168097CC1F30111012901D0032907D15A
:10C3300069882A886A8000684088401A401E2880E0
:10C340002068006901F080FB2068006901F0C2FBF1
:10C35000206D78B1B4F91020B5F900108A4205D1EA
:10C36000B4F91220B5F902309A4203D0B5F902208F
:10C3700009F05BF82888208168886081207901288D
:10C3800004F1040006D000F0FBF8208920826089C7
:10C39000608270BD00F002F8F7E700002DE9F0417F
:10C3A000764D0446406A6860617809077DD4A968C3
:10C3B000002609680F6930B1E16A39BB4FF40051BA
:10C3C00007F0F0FE10BB384601F054FB211D05F0CC
:10C3D000CFF8686070B9384601F054FB211D05F0B4
:10C3E000C7F8686030B9384601F05EFB211D05F0E2
:10C3F000BFF86860A06A48B1A683E6832046F8F7D4
:10C40000BDFB204600F06AF900284ED1606A6968D9
:10C4100088423CD0A188A181E188E18140B103211B
:10C42000AA6803F09DFE204600F058F900283CD190
:10C4300068686062A06250B309F02EFF60646078A3
:10C44000012120F0010060702683668394F840008B
:10C4500020F0FF0084F8400084F84160A687E6875A
:10C46000A682E682D5E9010203F07AFE204600F0BA
:10C4700035F900287FD1A868417909077BD4001DD0
:10C48000FFF7DCFB204600F029F9002873D1A088D3
:10C49000A189401A00B2A082E188E289891A09B212
:10C4A000E182B4F91C20104400E064E000EBD0709D
:10C4B0004010A083B4F91E00084400EBD070401077
:10C4C000E083E06920626868002854D00221AA68ED
:10C4D00003F046FE204600F001F900284BD1A86881
:10C4E0004079000747D42046F8F792FA204600F03A
:10C4F000F5F800283FD12046FFF790FD204600F0D8
:10C50000EDF8002837D1E06A002834D16078C00700
:10C510001DD1606C09F0B9FEAA681168898B884248
:10C520000FD90521686803F01BFE204600F0D6F8FD
:10C53000002820D1607840F00100607009F0ACFE66
:10C54000A064E06A002816D16078C00713D0A06C00
:10C5500009F09BFEAA681168C98B88420BD9062195
:10C56000686803F0FDFD204600F0B8F8002802D10D
:10C5700009F092FEA064BDE8F0810000A800002050
:10C580002DE9F84304464078434E00074FF000057C
:10C5900011D5606A0321B26803F0E2FD204600F085
:10C5A0009DF8002876D16562A5626564A56460780F
:10C5B00020F008006070606A7060D4F82C80002859
:10C5C0005DD00821B26803F0CBFD204600F086F86C
:10C5D00000285FD1B8F1000F16D16078C00709D1EB
:10C5E000D6E90102042103F0BBFD204600F076F8F5
:10C5F00000284FD1D6E90102072103F0B1FD204602
:10C6000000F06CF8002845D165626564A564B8F156
:10C6100000003FD04FF48079009500274E46054634
:10C6200000216E2207F03CFC384407B22846002166
:10C630006D2207F035FC00B2C11700EB116000124B
:10C64000704306B2284606F073FE0500E8D10FB924
:10C650004E4514D0784205B24FF4803090FBF6F08E
:10C6600006B26B463246294604F11C0009F0CCF8AC
:10C670006B463246294604F1200009F0C5F8B8F1AE
:10C68000000F07D02046F8F779FA2046BDE8F843B6
:10C6900000F024B8BDE8F883A80000204279910793
:10C6A00018D500218162C16201638164C164818304
:10C6B000C18390F8443022F0030223F00F0380F886
:10C6C000443001844184A0F84010A0F84210427127
:10C6D0000148416070470000A800002040788107B1
:10C6E00002D5034A00215160C0F3400070470000AA
:10C6F000A80000202DE9F843C56A04468021284699
:10C7000007F050FD4D4FFE0CC8B1284606F03BFF28
:10C7100001281DD0022828D0032837D0E786668755
:10C72000284606F029FF012847D0022850D00328C8
:10C730005AD0A7862687A08E002872D072E0334692
:10C7400039463A4604F13400009600F006FEF2E75E
:10C75000E88A0023401C01B232462846FEF784FADC
:10C76000E086E88A401E02B209E0B5F91A100023FB
:10C7700032462846FEF778FAE086B5F91A200023FB
:10C7800039462846FEF770FA6087C9E7688BE98A60
:10C790000023401A401C00B200EBD07001EB60088F
:10C7A00008F1010001B232462846FEF75DFAE08644
:10C7B000A8F10100002302B2E2E7B5F9141000234A
:10C7C00032462846FEF7C8F9A086B5F9142009E0DC
:10C7D000B5F91810002332462846FEF7BDF9A086A9
:10C7E000B5F91820002315E0288BA98A0023401AE8
:10C7F000401C00B200EBD07001EB600808F10100B2
:10C8000001B232462846FEF7A7F9A086A8F101003A
:10C81000002302B239462846FEF79EF920878AE7B0
:10C82000FFE7A786208F00B92687E08E00B9E7864C
:10C83000608F002800D16687BDE8F88301E0FFFF24
:10C840002DE9F74F0D4682B00446B04907F0B1FC20
:10C8500000287DD12046FEF7A9FD82462046FFF73D
:10C860002DF85FEA000973D0BAF1000F70D02046AE
:10C87000FEF792FD07462046FFF716F8DFF890B264
:10C88000064620460021BBF80E2007F009FB00F009
:10C89000FF0820460021BBF8142007F001FBC0B2BE
:10C8A00001902B6807EB0A006FF00102D5F808C071
:10C8B00033F8171002EB40001B5A3CF800001844F4
:10C8C000401A00B200906B6806EB090002EB4000D2
:10C8D00033F816101A5AEB68185A1044401A0FFA17
:10C8E00080FB0021204607F0D6F901280AD1B8F1D3
:10C8F000000F03D0B8F1020F02D003E0022000E0E5
:10C9000000208046208BA18A401A401C0FFA80FA32
:10C91000608BE18A401A401C0FFA80F94046B8F15A
:10C92000010F1BD0022824D02868B8F1030F30F97A
:10C93000170028D18046608CDDF800A040F400602C
:10C940006084019801287BD0022877D0032800E07A
:10C95000D8E0686830F9167071D119E0296800983C
:10C96000A0EB0A0031F8171000EBD07001EB60006B
:10C9700008E0204607F010FC296831F817200099DC
:10C980001144081A00B28046608C20F40060D7E79A
:10C99000608CD94640F480606084204607F0FCFB40
:10C9A000504504D1204606F09CFC484527D0A08A7B
:10C9B000ADF80000E08AADF80200208BADF804006D
:10C9C000608BADF80600204607F0D2FD04F114009C
:10C9D0005146054600F0CDFC4946284600F0C4FC0F
:10C9E000204607F0C5FD6A462921204603F0B8FB22
:10C9F000204606F09DFC2246222103F0B1FB204692
:10CA000000216B2207F04CFA06B2204600216C226E
:10CA100007F046FA05B2204607F0BEFB81462046E5
:10CA200006F05FFC0146C6F3413064224FF4FA631E
:10CA30004FF47A7C01281BD027E001E00AE013E0E4
:10CA40006968ABEB090000EBD07031F8161001EB10
:10CA5000600008E0204606F044FC696831F81620C2
:10CA600002EB0B01081A07B2608C20F4806093E798
:10CA700026F4C040984208DC604501DDC0F57A70BC
:10CA800000FB09F090FBF2F006B2C5F3413001283B
:10CA90000BD125F4C040984207DC604501DDC0F5AC
:10CAA0007A70484390FBF2F005B2049A08EB060056
:10CAB000791912891044A28A801A05B20498408913
:10CAC0000844E18A401A06B255EA06001AD0204608
:10CAD00007F04EFDA08A2844A082208B28442083A2
:10CAE000E08A3044E082608B30446083204607F067
:10CAF0003FFD05B0324629462046BDE8F04F0023F1
:10CB000007F0BABD05B0BDE8F08F000001000600D7
:10CB1000F00000202DE9F041064615460F460020A2
:10CB200005E039462046B04701280AD020460AF0E1
:10CB3000C1FA040002D060688000F2D10020BDE894
:10CB4000F08105B12C600120F9E703880A8893423F
:10CB500001D0981A704740884988401A7047037876
:10CB60000A78934201D0981A704740784978401A61
:10CB7000704700002DE9F0414268096822F0404208
:10CB80008A4227D10446FEF7F6FBDFF84C800546C3
:10CB9000D8F80820131BA2EB05005E1BC8F808009C
:10CBA00015D0274661193246384605F03DFB06E0B0
:10CBB000A068401BA0602046FEF7DDFB0444D8F8C7
:10CBC00008008442F4D1B819294605F0F3FB01208E
:10CBD000BDE8F0810020FBE7D00000202DE9FC41FA
:10CBE000064614468846D80729D004F108000125D6
:10CBF000002206F114010746F7F7C6FB58B10020E2
:10CC00008DF800006A4612213046019703F0A8FA19
:10CC10009DF8000098B16089218A0844401EE08197
:10CC2000B4F90E10B4F90600814200DDE08102B0D3
:10CC30002A4621464046BDE8F04101F083BA00256E
:10CC4000EEE72DE9F041074688B01D4616468846B6
:10CC50000846F8F7F4F9044602A9404606F008FB36
:10CC60002246114602A800F05EFB022E05D0012EDE
:10CC700029D0002008B0BDE8F081DDE90201CDE94E
:10CC8000040100231A4604A9404607F0D2F904AA79
:10CC90006846B968F7F750FB0028EBD0DDE90001E2
:10CCA000CDE906010123002206A9404607F0C1F99B
:10CCB00006A902AA0846F7F73FFB0028DAD0069833
:10CCC0002860079809E002AA6846B968F7F734FBBC
:10CCD0000028CFD000982860019868600120C9E73B
:10CCE00070B5044606F03EFA0646002506E0A06848
:10CCF000006850F82500FFF7F3FF6D1CB542F6D32E
:10CD0000608CC1071AD020F001006084204607F033
:10CD10000DFF204607F02CFE86B10021204607F0CB
:10CD200017F858B10C494968884207D80B49096877
:10CD300001EBC00050E9022120469047608C81073A
:10CD400008D520F0020060842046BDE87040002134
:10CD500007F052BD70BD0000BC0000206001002043
:10CD60002DE9F0478046089D1F46E86900FB01F366
:10CD70009B12002807DD934207DD00BF95F82800CD
:10CD800080070DD48BE09342F8DBCB1943439B1211
:10CD9000002808DD934239DA95F8280080077ED410
:10CDA0000120BDE8F0879342F6DCA869521C50438D
:10CDB00040F395000312C0B2FF22002828D000BF24
:10CDC0006E6AC0F1FF0404FB06F4A2EB242600BF48
:10CDD000A3EB0104A14636D0002C15DBBC4213DACC
:10CDE000C0F1FF00C6F1FF014843A2EB6020C1B2D1
:10CDF00095F82800800701D5C1F1FF0118F804005B
:10CE00000AF04AF908F80400641C1CE0A869CEE79F
:10CE10004FF0FF06DCE7002C10DBBC420EDAA6EB7D
:10CE20006000C1B295F82800800701D5C1F1FF016B
:10CE300018F804000AF030F908F80400686A641C65
:10CE4000361ABC4202DA686AB042E4DBBC4218DA45
:10CE5000002C16DBA869704380127043C0F3472191
:10CE6000E869002801DAC1F1FF0195F82800800780
:10CE700001D5C1F1FF0118F804000AF00DF908F816
:10CE8000040095F82800800707D54946B94506DC17
:10CE900000290DDB404609E001E0641C01D50020BB
:10CEA0007FE7BC4204DC391B08EB040005F082FA82
:10CEB000022076E72DE9F05F06460A9F8A461D4666
:10CEC000B86900FB02F18C12002800DD641C97F8A1
:10CED0002830544502DA980707D4D5E08C120AEBC3
:10CEE000050CA44502DA98077ED483E0521C424325
:10CEF00041F3950142F395044FEA2129221204F0EF
:10CF0000FF08C9B2A9EB0A04914505D0002803DA4D
:10CF100011B9FF219146641E914528D1002C0CDBEC
:10CF2000AC420ADA01EB08004108980701D5C1F1CB
:10CF3000FF01305D0AF0B0F8305597F82800641C06
:10CF4000800706D5A9EB0A01A9424DDA8EE03046EA
:10CF50000AE0AC4200DD2C46002C45D006DD00BFC7
:10CF6000A5EB040106EB040005F024FA89E04FF07C
:10CF7000FF0B002844DAF869404248434FEAA028F2
:10CF8000002C0DDBAC420BDA08FB01F0C0F34721AB
:10CF9000980701D5C1F1FF01305D0AF07DF83055E9
:10CFA000B969A8F1FF0041438812641E11D4AC4254
:10CFB0000FDAC8F1FF014143ABEB6120C1B297F832
:10CFC0002800800701D5C1F1FF01305D0AF064F847
:10CFD000305597F82800A41C800709D5A9EB0A0151
:10CFE000491EA9424DDC00E04EE00029AFDC48E0DC
:10CFF000AC4202DD0120BDE8F09F002CB0DA40E039
:10D00000C1F1FF00F96941434FEAA128002C0EDB72
:10D01000AC420CDA00FB08F0ABEB6020C1B2980721
:10D0200001D5C1F1FF01305D0AF036F83055B9691C
:10D03000C8F1FF0041438912641C0ED4AC420CDAE3
:10D040004843C0F3472197F82800800701D5C1F174
:10D05000FF01305D0AF020F8305597F82800641C75
:10D06000800707D5A9EB0A01A9420DDC0029BFF60C
:10D070006EAF06E0AC4200DD2C46002C04D03FF73A
:10D080006FAF4FF00200B6E74FF00000B3E70000CB
:10D090002DE9F0410746884600261448F7F700FFBF
:10D0A00004461DE021461148F7F70CFF05462068AD
:10D0B000B84200D09FB96168414502D0B8F1000F75
:10D0C0000DD121460948F7F786FF216909B12046AD
:10D0D0008847204605F06CF8F8F73CFB01262C4603
:10D0E000002CDFD13046BDE8F08100000453002061
:10D0F00070B505460C460948F7F7D2FE0BE001680B
:10D10000A94204D14168A14207D0002C05D00146B4
:10D110000248F7F7D7FE0028F1D170BD0453002074
:10D1200010B50446442105F045F94FF4FA70E06269
:10D13000002020626420A0620120A4F8400004487E
:10D14000E06194F8420040F0010084F8420010BD14
:10D1500089D1000838B504464FF480650095D4E9BC
:10D160000B200023194604F079FF40F2B6334FF448
:10D1700061720021009500F001F9226AA16A891A02
:10D18000414302EBA12038BD38B504464FF480601E
:10D190000090D4E90B200023194604F05FFF226AB7
:10D1A000A16A891A414302EBA12038BD8B1A002BDA
:10D1B00000DC531A4FF47A714B43B3FBF0F00028B4
:10D1C00000D101207047000070B54168054611B1DB
:10D1D0002868FFF75DFF1948F7F7F4FE184E10B105
:10D1E00009F05AF870601548F7F77FFE040024D064
:10D1F0004422294605F018F82868A84200D1246086
:10D20000717894F8420061F3820084F84200C0070C
:10D210000FD0616939B120468847216A01442162F3
:10D22000A16A0844A06262681AB1206808B1216A44
:10D230009047F8F78FFA204670BDFEE704530020B0
:10D24000480100200A8802804A8842808A888280B9
:10D25000C988C18070470A8802804A8842808A88CB
:10D260008280C988C18070470A8802804A884280CB
:10D270008A888280C988C18070470A8802804A886B
:10D2800042808A888280C988C18070470A8802806B
:10D290004A8842808A888280C988C18070470A880B
:10D2A00002804A8842808A888280C988C18070470B
:10D2B0000A8802804A8842808A888280C988C18020
:10D2C0007047C1884088081A401C00B27047C18866
:10D2D0004088081A401C00B27047B0F90410B0F939
:10D2E0000020891AB0F90620B0F90200101A401C7B
:10D2F000491C4843704781880088081A401C00B2C6
:10D30000704781880088081A401C00B270478188E5
:10D310000088081A401C00B2704781880088081AEB
:10D32000401C00B2704703885B1A0380838819444D
:10D3300081804188891A4180C1881144C180704729
:10D3400003880B44038083881944818041881144F9
:10D350004180C1881144C180704710B5029C018092
:10D3600042808380C48010BD4288491E1144C18020
:10D3700070470288491E114481807047F0B5C0F59E
:10D38000806404FB04F5AD0A05FB04F64FEA962C15
:10D3900000FB00F6B60A06FB00F745435543BF0AFB
:10D3A0000CFB01FC74434FEA9C2105EB45005C43F8
:10D3B000DDF814E004EB440201EB105007FB0EF71C
:10D3C00000EB125000EB9720F0BD10B50C46102179
:10D3D000204605F0C7FA2046BDE810404FF48061B2
:10D3E00005F046B810B50146034805F00DFA0446AD
:10D3F00005F07EFA204610BDCCE80108F0B50446E1
:10D400004FF4FA66C1F341307710642501280BD13F
:10D4100021F4C040B04207DCB84201DDC0F57A70AB
:10D42000584390FBF5F001B2C2F3413001280BD113
:10D4300022F4C040B04207DCB84201DDC0F57A708A
:10D44000584390FBF5F002B2944201DA204600E026
:10D450001046884201DA0846F0BD944201DA2046BF
:10D46000F0BD1046F0BDF0B504464FF4FA66C1F3C6
:10D4700041307710642501280BD121F4C040B0421F
:10D4800007DCB84201DDC0F57A70584390FBF5F037
:10D4900001B2C2F3413001280BD122F4C040B042A6
:10D4A00007DCB84201DDC0F57A70584390FBF5F017
:10D4B00002B2944201DA204600E01046884201DAC6
:10D4C0000846F0BD944201DA2046F0BD1046F0BD9A
:10D4D000002208B51146104600F075F80090BDF81E
:10D4E000000008BD002208B51146104600F083F880
:10D4F0000090BDF8000008BD002208B51146104696
:10D5000000F0A9F80090BDF8000008BD38B50C4641
:10D510000546FFF7F1FF2246294600F01BF900906F
:10D52000BDF8000038BD000007B58107BDF8043024
:10D5300002D020F8023B521EBDF8041001EB01415D
:10D540000EE002C0103A02C040F8081B40F8041C6C
:10D5500040F8101B40F80C1C40F8081C40F8041C54
:10D56000102AEED803E000BF20F8023B521E002A2A
:10D57000FAD10EBD4FF478414FF4FC6201EA10215C
:10D5800002EA501208B51143C0F3C4000143ADF8DC
:10D59000001088B208BD08B5D308BDF8002063F3B9
:10D5A0000402ADF800208A08BDF8001062F34A11A9
:10D5B000ADF80010C108BDF8000061F3CF20ADF850
:10D5C000000080B208BD08B5D308BDF8002063F3A1
:10D5D0000402ADF800208A08BDF8001062F34A1179
:10D5E000ADF80010C108BDF8000061F3CF20ADF820
:10D5F000000080B208BD08B5D308BDF8002063F371
:10D600000402ADF800208A08BDF8001062F34A1148
:10D61000ADF80010C108BDF8000061F3CF20ADF8EF
:10D62000000080B208BD08B5D308BDF8002063F340
:10D630000402ADF800208A08BDF8001062F34A1118
:10D64000ADF80010C108BDF8000061F3CF20ADF8BF
:10D65000000080B208BD08B5D308BDF8002063F310
:10D660000402ADF800208A08BDF8001062F34A11E8
:10D67000ADF80010C108BDF8000061F3CF20ADF88F
:10D68000000080B208BD08B5D308BDF8002063F3E0
:10D690000402ADF800208A08BDF8001062F34A11B8
:10D6A000ADF80010C108BDF8000061F3CF20ADF85F
:10D6B000000080B208BD000008B5121DD3080A4A58
:10D6C00089B280B241EA014140EA00401140104075
:10D6D000401A584301EB5010104040EA1040ADF89A
:10D6E000000080B208BD00001FF8E00708B5121D59
:10D6F000D3080A4A89B280B241EA014140EA0040B7
:10D7000011401040401A584301EB5010104040EABD
:10D710001040ADF8000080B208BD00001FF8E0071F
:10D7200008B5121DD3080A4A89B280B241EA014104
:10D7300040EA004011401040401A584301EB50109D
:10D74000104040EA1040ADF8000080B208BD000073
:10D750001FF8E00708B5121DD3080A4A89B280B243
:10D7600041EA014140EA004011401040401A58434C
:10D7700001EB5010104040EA1040ADF8000080B2BC
:10D7800008BD00001FF8E00782B2D00AC0EBC0035A
:10D7900003EB0020C01D400960F317410846C2F3A7
:10D7A000451101EB410303EB0121C91C890961F318
:10D7B0000F2002F01F01C1EBC10202EB0121C91DC4
:10D7C000490961F30700FF2161F31F607047FF22E1
:10D7D00008B511461046FFF70EFF0090BDF8000097
:10D7E00008BD08B51F20BDF800103F2260F30401FA
:10D7F00089B262F34A1189B260F3CF21ADF800100B
:10D8000088B20090BDF8000008BD70B50C00054658
:10D810000FD000F007F960435030B0F5A07F0ADB6D
:10D82000284600F0FFF86043A021503090FBF1F053
:10D8300002E0002000E0012000B270BD2DE9F041BF
:10D840000D461E46174604461C2104F0B3FDC4E9EC
:10D850000057C4E90256BDE8F081000038B504461F
:10D86000502104F0A7FD4FF4A0702080F0206080CC
:10D870004FF0FF30A080E08000202081608120698F
:10D88000822120F0400040F0080061F3D0102061B8
:10D890004FF4FC60ADF800000090BDF80000208758
:10D8A0000248206460645820A06438BD2DF600084A
:10D8B000F8B505465048F7F718FB040002D0E86BAE
:10D8C00008B10AE0FEE7A86C04F0E6FB06007AD097
:10D8D00001462A6C28469047EE634FF4B471204607
:10D8E00004F068FD01202560C4F85401082104F506
:10D8F000AC70F7F7F2FA414E22461E21F768404815
:10D90000F46008F0DDFC606000285DD028698107C4
:10D910000BD5B5F90010B5F902205143EA68D26879
:10D92000914202D920F002002861BDF800101F20AA
:10D9300060F304013F2289B262F34A1189B260F3B5
:10D94000CF21ADF8001088B20090BDF80000009023
:10D95000BDF800006085FF2084F8290008F082FCF3
:10D9600080B308F023FCA060002005F08BF8206154
:10D97000002005F087F8E061002005F083F8214DD4
:10D9800020622A460021E06907F012FB2A460021A6
:10D99000206A07F00DFB0221E06904F0E3FF022199
:10D9A000206A04F0DFFF0021E06907F049FD002153
:10D9B000206A07F045FD206906F0DAFDF760A7B19F
:10D9C00014E000E001E0FEE7FEE7002007F00CFFB6
:10D9D0000546052007F008FF01460B48009000238C
:10D9E0002A46204608F0ECFBBDE7F460606808F0CA
:10D9F00038FD2046F8BD0000E05200203001002034
:10DA000075460008FFFF0F0004E60108C268002108
:10DA10001161C068416170470148C06870470000EB
:10DA20003001002010B90548C06820B100680069C5
:10DA3000C0F3C910704782207047000030010020F9
:10DA40000068C0687047000018B90948C06800281D
:10DA500009D00068017CC1F30111012904D0032918
:10DA600002D0B0F900007047B0F902007047000022
:10DA70003001002010B518B9FFF7CEFF002800D004
:10DA8000006A10BD10B518B9FFF7C6FF002800D016
:10DA9000C06910BD18B101460248F7F713BA014832
:10DAA000F7F7FEB9E052002010B518B9FFF7B4FF40
:10DAB000002800D0006910BD10B518B9FFF7ACFF01
:10DAC000002800D0406910BD10B508B9FFF7A4FFC9
:10DAD000806810BD18B90948C068002809D00068DE
:10DAE000017CC1F30111012904D0032902D0B0F94E
:10DAF00002007047B0F900007047000030010020BC
:10DB000010B518B9FFF788FF002804D0D0F85401E9
:10DB1000002801DD012010BD002010BD2DE9F041DD
:10DB20001D0017460E4604461AD0F07A02281AD96C
:10DB3000D4F81CC0BCF1000F03D02046E0470128F8
:10DB400011D02B463A4631462046F9F7EFF9012825
:10DB500009D006A239462046BDE8F0410BF0B3B823
:10DB600002A23946F8E7BDE8F08100004E6F0A6472
:10DB70006174610038B58469049D002C01D0009562
:10DB8000A04738BD38B50446182104F013FC002224
:10DB900011461046FFF7FFFC0090BDF80000009012
:10DBA000BDF800002081FF20E072401C6080012051
:10DBB000207538BD704700002DE9FF4FB5B0887E55
:10DBC000429F1E4692460C4602287DD920680028B6
:10DBD0007AD03598006A002876D0202212A8F2F771
:10DBE00079FD20680390002E6ED0307800286BD02D
:10DBF0003598514682682EA8F6F79EFB002863D020
:10DC0000207FB0F1000B01D14FF0010B607F800746
:10DC100007D4BAF80410BAF80000081A401C03B27E
:10DC20000FE0B4F91200627F41F6FF718DE8070042
:10DC3000B4F91430314606A8226808F0EFFDBDF9AA
:10DC400018300398B4F912100025B0F908906A1E34
:10DC500001EB09000B90BAF80000ADF81000BAF81B
:10DC60000210ADF81210B4F916000990B4F91800BA
:10DC70000144ADF81210FFB1F0B9BAF90210002951
:10DC80001ADAD7F808C0ACEB0100002801DCA1EBE0
:10DC90000C000B994FF4806C49420CEB4101884217
:10DCA00000DD3A603868002806DB0546BDF8121032
:10DCB000B8880844ADF81200617F0020CDE900016A
:10DCC000B4F91420701900E0A1E02D930399F7F73F
:10DCD000F3FB00EB050829E0617F0020CDE900019E
:10DCE000B4F9142006EB08002D9B0399F7F7E4FB29
:10DCF000454600EB0508BDF812100B98084400B229
:10DD0000ADF812007FB110F5806F0CDB3868002889
:10DD100009DA3D60BDF91210BAF90200081A7860FC
:10DD2000BAF90200B860705D002870D0BDF9121019
:10DD300001EB090035998968B1F902108842CBDB03
:10DD40005846CDF8C0B0BBF1020F02D0032816D060
:10DD500029E0607F0090B4F91430A8EB0501701938
:10DD6000039A08F0B9FD07465046FFF7CAFAC01BF0
:10DD7000BDF8101000EBD07001EB600011E0607F87
:10DD80000090B4F91430A8EB05017019039A08F05B
:10DD9000A3FD07465046FFF7B4FABDF81010C01BAC
:10DDA0000844ADF81000D4E9019BD94502D9484692
:10DDB000D9468346A07F800717D02AA800F02DFA05
:10DDC000A089ADF8A800039890F90E0000B90120D1
:10DDD000ADF8AA00A07E8DF8B000A07F9DF8B1102C
:10DDE000C00860F301018DF8B11000200E90FFF71C
:10DDF0006FFB3390FFF76CFB31901AA800F048FFDF
:10DE0000208AADF86C00BDF9100032906BE16EE134
:10DE1000BDF81010099800270844ADF810007019DB
:10DE20000F900797A8EB05001190BCE00020A9F522
:10DE30007F410A90FF390AD0ABF57F40FF3806D00A
:10DE4000AC4A079829181268304690470A9007ABE9
:10DE50006A4601A90F98F7F717FB607FC0070AD041
:10DE60000198232802D0012F13D004E047B1012FDD
:10DE70000AD0022F0BD0E0683190022F4FD050E033
:10DE800007980E90012048E00027E06848E0002055
:10DE900043E0202842D107990E98081A072801D09C
:10DEA000A08938E0DDE90E210A4428A85FF00601C8
:10DEB00012F8013B00F8013B491EF9D100208DF812
:10DEC000A6009DF8A100FDF761FE07469DF8A000A1
:10DED000FDF75CFE07EB00100A909DF8A300FDF72C
:10DEE00055FE07469DF8A200FDF750FE07EB001017
:10DEF0000C909DF8A500FDF749FE07469DF8A4008B
:10DF0000FDF744FE07EB0010C2B20C98C1B20A98AC
:10DF1000C0B2FFF758FB33900220074643E0339826
:10DF20003190DDE90021039802F02EFA29904FF696
:10DF3000FF70814522D0834520D00A9848451DD3E3
:10DF400058451BD2BDF81000ADF83000BDF81210D6
:10DF5000ADF83210A28A02442998401E1044ADF850
:10DF600034000B980CAA401E0844ADF836001AA9DC
:10DF7000359800F079FEE089ADF8C400BDF8C40022
:10DF8000ADF8540004AA12A9019B359800F033F9AA
:10DF90002998002807DDBDF81010A08A08442999A7
:10DFA0000844ADF810000799119888423FF63EAF3B
:10DFB000A07F800723D53298ADF800002068BDF916
:10DFC000AA1002ABB0F9080001EBD17100EBD070E0
:10DFD000401000EB6100BDF812106A460844BDF81D
:10DFE0001010ADF80810ADF80200ADF80A00BDF849
:10DFF000C400ADF8A8002AA9359800F001F9A07F67
:10E00000C0071FD03298ADF800002068BDF812108C
:10E0100002AB028940891144091A03986A4690F9B3
:10E020000D00081ABDF81010ADF80810ADF8020088
:10E03000ADF80A00BDF8C400ADF8A8002AA93598CB
:10E0400000F0DEF8617F0020CDE9000106EB08005A
:10E05000B4F9142007462D9B0399F7F72DFA45468E
:10E0600000EB0508BAF80000ADF81000309802285F
:10E0700002D0032816D029E0607F0090B4F9143054
:10E08000A8EB05013846039A08F026FC07465046DF
:10E09000FFF737F9C01BBDF8101000EBD07001EB93
:10E0A000600011E0607F0090B4F91430A8EB050126
:10E0B0003846039A08F010FC07465046FFF721F94E
:10E0C000BDF81010C01B0844ADF81000BDF81210C8
:10E0D0000B980844359900B2ADF812008968B1F97F
:10E0E0000610884203DC705D00287FF491AE39B0E1
:10E0F000BDE8F08FB401002038B50446202104F0BB
:10E1000059F9FF20A076FFF7E3F90090BDF8000071
:10E11000A0810B4820604FF6FF706060A060FFF7A1
:10E12000D7F90090BDF80000E081052007F05CFB06
:10E130000090BDF8000020820020E07638BD00008D
:10E1400004E60108036C002B00D018477047436CAD
:10E15000002B00D0184770472DE9F0410546C06BF1
:10E1600017460E46002826D0E86C03F095FF040001
:10E170001CD0E96C04F01EF9F7F74AF9296821620E
:10E180006968E161A968A16100683A462146007C9E
:10E19000C0F3801084F824003068206070686060EC
:10E1A000EB6B28469847050001D003E0FEE72046C8
:10E1B00003F0FEFF2846BDE8F08170B50C46054629
:10E1C00001F089FF206A2860E0696860A069A860A2
:10E1D000F7F71EF9006894F82420016962F38611AC
:10E1E0000161AA6C12B12146284690472046BDE83D
:10E1F000704003F0DDBF30B4046AA44630BC604711
:10E2000030B44C88002C06D00C7A022C03D9446A16
:10E21000A44630BC604730BC704738B504460A217C
:10E2200004F0C8F801206080FF202072BDF80010C3
:10E23000002060F3040189B260F34A1189B260F3EF
:10E24000CF21ADF8001088B20090BDF8000000901A
:10E25000BDF80000208038BD10B503460A4A0020F2
:10E2600052F8304024B1401CC0B21028F8D301E06D
:10E27000102802D34FF0FF3010BD42F8303002EBCF
:10E28000C002516010BD0000505400202DE9FF4F26
:10E2900081B08B460E9D16461C46B5F90A10B5F99D
:10E2A0000C00571AB5F9082005F11009ABEB020371
:10E2B00005F13C0AB4285DDAB5F90E20B42A7DDAFE
:10E2C00000287BD0002A79D0904277DDB1425ADC19
:10E2D000696D79434FEAA12CA96A7F1C79438912A1
:10E2E000A0F20F15582D01D8002909DB451E592D24
:10E2F00001D8002904DB5B38B32802D2002900DDF5
:10E300000021A2F20F10582801D8002909DB501E65
:10E31000592801D8002904DB5B3AB32A02D200292C
:10E3200000DD0021ACEB010001EB60000125C71A04
:10E33000A74200DD2746002F0DDD3BB2324659468D
:10E34000CDF80090019800F091F9050003D139460D
:10E35000019804F02FF8A74200DD2746002F00DACD
:10E360000027CDF800A05DE0B54276D1284605B083
:10E37000BDE8F08F68DDB5F90E20B42A64DD904267
:10E3800062DDB14201DA0120F1E7696D79434FEABC
:10E39000A12CA96A7F1C79438912A0F20F15582D70
:10E3A00001D8002909DB451E592D01D8002904DBBD
:10E3B0005B38B32804D2002902DD00E044E00021EC
:10E3C000A2F20F10582801D8002909DB501E592845
:10E3D00001D8002904DB5B3AB32A02D2002900DD10
:10E3E0000021ACEB010001EB60000125C71AA74238
:10E3F00000DD2746002F0DDD3BB232465946CDF8F1
:10E4000000A0019800F032F9050003D139460198C7
:10E4100003F0D0FFA74200DD2746002F00DA0027D7
:10E42000CDF800900BEB070001B20198E41B3844D3
:10E4300023B20746324600F019F9060094D121466E
:10E44000384603F0B7FF8FE70127B846B42805D058
:10E4500038B109DAB14209DC0AE047E0B14210DC28
:10E4600004E0B14202DC0CE0B14201DC032708E029
:10E47000234632465946CDF80090019800F0F6F850
:10E480000746B5F90E00B42806D060B1B5F90A0008
:10E490000FDAB04204DC0EE0B5F90A00B04206DD46
:10E4A0004FF0030803E0B5F90A00B042F8DDBFB150
:10E4B0000EE0B042F4DD234632465946CDF800A0C6
:10E4C000019800F0D3F8804657B1B8F1000F07D09B
:10E4D000032F02D0012F05D008E0B8F1030F05D1BA
:10E4E000002044E74046B8F1010FFAD002203EE791
:10E4F0002DE9F8430546884640F26710411C089C08
:10E500001746002B01DA002302E08B4200DB0346B2
:10E51000002C01DA002402E08C4200DB04469C421D
:10E5200003DAC3F5B470204403E0E01A002800DCED
:10E53000181BA5F86800AB81EC81A5F808806F81F5
:10E5400015482860012028718B4200D9FEE7B42BC2
:10E5500001D2002000E00120002C01DB8B4200DD15
:10E56000FEE7B42C05D3A4F1B401B42901D20026EE
:10E5700000E0012600903A46414605F1100000F007
:10E58000CBF823463A46414605F13C00009600F0A0
:10E59000C3F8BDE8F88300008DE200082DE9F843D8
:10E5A0001E4617468846814600250C4C0DE000901B
:10E5B000D0F800C033463A4641464846E047002876
:10E5C00008D0022800D10125083420680028EED1A7
:10E5D00015B10220BDE8F8830120FBE7505400206C
:10E5E00010B50179022906D0052913D18068BDE84C
:10E5F000104003F0DDBD0446406900280AD00169DF
:10E60000002904DA406803F0D3FD6069EFE741694F
:10E61000491E416110BD000070B5134D060008D0C1
:10E620005FF0000455F83410B9B10879022805D01C
:10E6300002E02868002800D0012070BD887CB1F974
:10E640001020C007304601F1080102D0F5F70CFF99
:10E6500001E0F5F799FE0028EED0641CE4B2102C1E
:10E66000E0D3002070BD000050540020F8B5069C97
:10E67000A58A266A521B658A12B2491B94F8285053
:10E6800009B24FEAC57526B1009485B3FEF768FB61
:10E69000F8BD85B1207C810727D000F00301012956
:10E6A00023D0022901D1511C1FD4C043800728D197
:10E6B000002A1ADC25E0227C02F00304022C14D08C
:10E6C000D543AD0711D0012C01D100290DDC9207F3
:10E6D00001EB030207D0002A13DB49420FD50021CA
:10E6E000002B0EDD0FE0002A02DA0120F8BD10E059
:10E6F0004A4206D49A420ADA991A104405E099422D
:10E7000001DB0020F2E7994201DA03F053FE022018
:10E71000ECE7FEF7CFFBE9E72DE9FC471C46DDF807
:10E72000288016460F468146B42B01DDB43C24B246
:10E7300004F15A0000B207F0ADFF07EB6015204668
:10E7400007F0A8FF06EB601000B2CDE900082BB27D
:10E7500032463946484600F003F8BDE8FC87000021
:10E760002DE9F0470F46DDE908699846154604464D
:10E770002C2103F01FFEB54206D1B9F1030F03D1DE
:10E780006D1E761E2DB236B2B54205DD4046B84646
:10E79000074630462E46054627816581A4F80C8041
:10E7A000E68184F810906782A8EB07004B46A582AB
:10E7B000002801DD014601E0A7EB0801721B002AD9
:10E7C00001DD154600E0AD1BA94294F8281002DDDA
:10E7D00041F0010101E021F0010184F82810002539
:10E7E000E561244E2660A5612571CE074FF48015A2
:10E7F0000DD020B195FBF0F65643B612E66122B17A
:10E8000095FBF2F242439012A061E0690CE022B164
:10E8100095FBF2F64643B612A66120B195FBF0F0E7
:10E8200050438012E061A0692062980709D003F08C
:10E830000300012808D0022813D0D843800714D041
:10E8400006E021F0020001E041F0020084F8280017
:10E85000216A88106062002901DA40426062BDE8E6
:10E86000F087206A0028EFDCEBE7206A0028EBDD68
:10E87000E7E700006DE600082DE9FE4F8046DDF871
:10E8800030900E461C4699F81200174600F0010A17
:10E89000B9F91050684609F10801FEF7F7FCBDF917
:10E8A0000200BAF1000F2FD0B84250DCBDF90600CB
:10E8B000B8424CDBBDF900004119B14205DCBDF99D
:10E8C00004203119521B914209DDBDF902104A1989
:10E8D000BA4240DCBDF90620521BBA423BDBBAF11A
:10E8E000000F18D0801B00D50020A04231DCBDF9FC
:10E8F0000410891B091A491C4218A24200DD211A82
:10E90000002926DB4044EFE0B84213DCBDF90600E5
:10E91000B8420FDBCEE7871BA7420BDC002F03DBDF
:10E920003946404603F046FDBDF90400851B6D1CC9
:10E93000002D02DC0020BDE8FE8FA54204DA611B39
:10E9400008EB050003F036FD1FB9A54201D10120F7
:10E95000F1E70220EFE7BDF80430821B181A401CD3
:10E960000FFA80FCBDF80600401A401C03B2781A6A
:10E9700000B2A84202DA281A401E01E0591B401AD0
:10E98000D9F8141000B20223CF6803EB4003FB5AFE
:10E9900037F810609B1B1EB28B68496833F8103043
:10E9A00037F810004FF0000700EB010B02EB0C00F2
:10E9B000401B18440FFA80F95019C01A401E05B2C6
:10E9C000BAF1000F22D06BE0F11B01EB0B0010F845
:10E9D000010C029009EB07005FEA000A08D4A24587
:10E9E00006DA18F80A10029808F056FB08F80A0030
:10E9F000B5EB070A08D4A24506DA18F80A100298FF
:10EA000008F04AFB08F80A007F1C3FB2B742DBDB84
:10EA100009EB0700A04201DA014600E02146002987
:10EA200001DA002002E0A04200DB204600B2211AF9
:10EA3000404403F0BFFCA81B411CA14201DA0A4676
:10EA400000E02246002A01DA002402E0A14200DAB6
:10EA50000C4621B2404647E0F11B01EB0B0010F8D9
:10EA6000010CC0F1FF00029009EB07005FEA000A09
:10EA700008D4A24506DA18F80A10029808F00CFB30
:10EA800008F80A00B5EB070A08D4A24506DA18F818
:10EA90000A10029808F000FB08F80A007F1C3FB239
:10EAA000B742D9DB681CA04201DA691C00E02146AC
:10EAB000002901DA002504E0A04201DA6D1C00E023
:10EAC00025462AB2A9EB0200A11A884201DA0346C0
:10EAD00000E00B46002B01DA002002E0884200DB58
:10EAE000084601B208EB020003F064FC31E70000C5
:10EAF0002DE9F0411546064688880A881C46801A8A
:10EB0000401C02B2C8884B88C01A401C00B2824226
:10EB100000DA1046B5EB600F00DD4510002D00DA7D
:10EB2000002506F10800FEF7B1FB3582B4743848C1
:10EB30003060022030710023C5B1364800214FF407
:10EB40007A7200BFC1EBC10400EB8404B4F9184031
:10EB5000AC421BD1C1EBC10100EB81004169491CF2
:10EB600041610169102D04DA012303E07361BDE8FE
:10EB7000F0812B110B44934205DA102D01DA0122AA
:10EB800000E02A110A4402617061F0E7491C04297F
:10EB9000D8D300244FEA0401C1EBC10700EB87077B
:10EBA000D7F814C0BCF1000F07D12CB1D7F810C0B2
:10EBB000D4F810E0F44500DA3C46491C0429EBD3B4
:10EBC0003CB16069401CC4E90430102D0EDA01200C
:10EBD0000DE01C2003F060FA040006D01C2103F0B5
:10EBE000E9FB4FF0FF3020610BE0FEE728111844ED
:10EBF000904205DA102D01DA012000E028111A18E0
:10EC00002261204629467461BDE8F041F7F7A6BEAF
:10EC100079E80008E0530020F0B50025094E0746CA
:10EC20002C4600BF06EBC4004068B84204D156F839
:10EC30003450204600F008F8641CE4B2102CF1D3E4
:10EC40002846F0BD505400200021421C08D0054A3F
:10EC5000002352F8301042F8303002EBC00043601D
:10EC6000084670475054002030B4D38854881B1B8A
:10EC70005B1C1BB2012B09DB938814881B1B5B1CDC
:10EC80001BB2012B02DB036930BC184730BC704754
:10EC900038B50446382103F08DFBFEF798FD00904F
:10ECA000BDF8000024F8040FFEF791FD0090BDF8B8
:10ECB00000006080FEF716FC0090BDF80000E080C8
:10ECC000FF2525720220A072FEF70CFC0090BDF813
:10ECD00000006083FEF706FC0090BDF80000208570
:10ECE0000748206104F8015CA57584F82650A577D3
:10ECF00084F83250E07F20F03E001E30E07738BDCF
:10ED000004E601082DE9F04FCBB08346DDE95465F8
:10ED1000087B984614460F4602287DD9B7F90200B1
:10ED2000002879D0AE4277D01AB28146924640454B
:10ED300000DD914601A8FFF7ABFF787B00F00300F0
:10ED40008DF80600B86840B100208DF80700B8685B
:10ED50000590387B8DF81E0005E0387B8DF80700A4
:10ED60003888ADF808002188A8F10103A1EB08025A
:10ED7000ADF840206188A1EB0801ADF84210208871
:10ED80001844ADF84400B4F802C0ADF8D4006344B0
:10ED9000ADF84630ADF8D020ADF8D210ADF8D63091
:10EDA000B7F802C06244ADF8D020B7F802C06144A1
:10EDB00009B2ADF8D210B7F802C0A0EB0C00ADF864
:10EDC000D400B7F802C0801AA3EB0C034FF0FF3C4D
:10EDD0001BB2CDF80CC1401CADF8D6304FF0000C82
:10EDE00000B2CDF810C1002812DD581A401C00B244
:10EDF00000280DDD012347F6FF7234A937A8FFF77D
:10EE000077FE01204490002137A8FFF725FA4390B0
:10EE1000002347F6FF7200E02DE010A93DA8FFF7A0
:10EE200067FE00213DA8FFF717FA459006F5B4707C
:10EE3000A84205D005F5B4714FF4B4708E4220D1CC
:10EE400047F6FF70ADF8040010AA01A95846FFF775
:10EE50000BFF4598FFF7F8FE4398401C02D04398FB
:10EE6000FFF7F2FE3DA8FFF7BBFB4498002802D055
:10EE700037A8FFF7B5FB4BB0BDE8F08FA6F5B47629
:10EE8000B6B28642FAD202E0A5F5B475ADB28542BB
:10EE9000FAD228B249900090B4F90220B4F90010D7
:10EEA00033B219A84A93FFF723FB002119A8FFF7F3
:10EEB000D3F94690B54203D9A81BC0F5B47000E061
:10EEC000701BDBF8081000913C282ADDB8F10A0F0E
:10EED00027D95A20B6FBF0F1B5FBF0F000F00300A3
:10EEE000ADF8540001A8ADF84CA0ADF8505001F0B9
:10EEF000030116901294ADF84E60ADF85210ADF8C3
:10EF0000569010A8CDE9170B12A8F9F755FF12A8D3
:10EF1000FAF71AF812A8FAF7E6F812A8FAF7D1F9F0
:10EF200004E010AA01A95846FFF79EFE19A8FFF7B2
:10EF300057FB3DA8FFF754FB449810B137A8FFF7E3
:10EF40004FFB4698FFF780FE4598FFF77DFE4398FC
:10EF5000401C02D04398FFF777FE787B40078AD5A4
:10EF600009F0FF0212AB51464A98FCF75AFCBDF873
:10EF70004800218812AA0844ADF84800BDF84C00AA
:10EF800021880844ADF84C00BDF84A006188084467
:10EF9000ADF84A00BDF84E0061880844ADF84E0057
:10EFA00015A80099F5F7C8F915AEC0B1002347F6CA
:10EFB000FF7212A943A8FFF79BFD002143A8FFF7AA
:10EFC0004BF90546584610AA01A9CBF80860FFF78F
:10EFD0004BFE2846FFF738FE43A8FFF701FB09F078
:10EFE000FF0212AB51464998FCF71BFCBDF84800E4
:10EFF000218812AA0844ADF84800BDF84C002188C9
:10F000000844ADF84C00BDF84A0061880844ADF8EA
:10F010004A00BDF84E0061880844ADF84E0015A8BE
:10F020000099F5F789F9C0B1002347F6FF7212A9DC
:10F0300043A8FFF75DFD002143A8FFF70DF9044643
:10F04000584610AA01A9CBF80860FFF70DFE20462C
:10F05000FFF7FAFD43A8FFF7C3FA0098CBF80800C2
:10F0600009E770B514460D460646F8F781F82246C2
:10F0700029463046BDE87040F8F74FBA7CB50446E3
:10F08000087E0D4602280ED9A26868462968F5F761
:10F0900053F9002807D0616B09B120468847626D9B
:10F0A0002946204690477CBD2DE9F04FCD6889B0B8
:10F0B0000C46074615B1207C00287DD0207C012815
:10F0C00000D10025786881880088081A401C00B2A9
:10F0D0000790BA6805A82168F5F72EF900286BD0CB
:10F0E000F6F796F983460068D7F80090C16941BBEE
:10F0F000017C490610D47968BDF91420B1F90030BB
:10F10000B1F90210D21ABDF916305B1A079901FB4A
:10F11000032209EB420113E07A68BDF91630B2F917
:10F120000260B2F900209B1B079E734303EB43036D
:10F1300003EB0901BDF914309A1A02EB42021144A3
:10F140008946D4F804A05FEA0A0114D021688B88AC
:10F15000B1F90020B1F902109B1A5B1C0FFA83F879
:10F16000BDF914309A1ABDF91630591A08FB01225C
:10F170000AEB420A01E04FF000083DB3007C0007B3
:10F180000FD46069FEF7A9F80146002007E02A5C69
:10F19000802A01D9FF2200E000222A54401C884224
:10F1A000F5DB60698288B0F90010521A521C16B261
:10F1B000BDF91420511A00E026E0BDF91620B0F97F
:10F1C00002002944101A06FB001500E000267868AA
:10F1D0004188008849420AB2404201B205A8FEF7C0
:10F1E000AFF8DBF80000C069D0B160680028207E6D
:10F1F0000DD001A9CDF8008081E86100534605A932
:10F200004846079A07F0C8FE09B0BDE8F08F8DE8C0
:10F210006100A36805A94846079AFBF71DFBF3E7C1
:10F22000607E80B161680029217E25D0CDF8008004
:10F23000CDE90360CDE90115534605A94846079A73
:10F2400007F06AFCE0E760680028207E0BD001A987
:10F25000CDF8008081E86100534605A94846079A29
:10F2600007F018FDD0E78DE86100A36805A94846BE
:10F27000079AFBF751F9C7E7CDE90260CDE9001520
:10F28000A36805A94846079AFBF7A0F8BCE72DE953
:10F29000F0479046B3F902401D4604FB08F301EB2A
:10F2A0004303B5F900100A9ADDE9080903EB4106AA
:10F2B000B2F90230B2F9002003FB09F300EB43007E
:10F2C00000EB4207A888401A401C00B24FEA400AEF
:10F2D0000AE052463946304602F0A6FF641C06EBAF
:10F2E000480607EB490724B2B5F90600A042F0DA58
:10F2F000BDE8F0872DE9FF4F9FB00D46824681683B
:10F300001446DDF8B0901BA8FDF7C9FF1BA8FFF756
:10F3100083F91890288818B96888B0F5807F01D0E3
:10F32000012100E0002117911C210CA803F042F8F4
:10F33000E87A8DF84800287B4FF0000600F00F00B7
:10F340008DF8490006A80C90DDE9171008432CD170
:10F35000B9F1040F06D0B9F10E0F0AD0B9F1140FAC
:10F3600021D022E0A87A00BB22980CA9CDE90C405C
:10F3700013E021466846DAF80820F4F7DDFF00289C
:10F380000ED022980D9611940F902889ADF8380070
:10F3900002208DF840000C946FE05046FFF76EFE9F
:10F3A00023B0BDE8F08FA87AF0B3DAF8080001883E
:10F3B000ADF818108288ADF81C20DAF808004088F3
:10F3C000ADF81A00DAF80830DE88ADF81E60A388C0
:10F3D0002788301ADB1B5B1C1BB21393E3886788FA
:10F3E000401CDB1B07B25B1C501A1BB2401C0FFAFF
:10F3F00080FB1493F6F70CF8FEF726FB804606A870
:10F40000FDF76BFF5E46404501D9B8FBFBF77E4335
:10F41000700002F06FFE1590304602F06BFE09900E
:10F420000F9006A8119000E012E002208DF8400035
:10F4300015980D90BDF91E0016907F1EBDF81A009C
:10F440001A973844ADF81E00B9F1040F1DD116E02B
:10F45000A08821886288401AE188401C891A491CCA
:10F460000AB2229900B2400000FB0210CDE90C4123
:10F470000F90022011948DF840000CA98DE7288888
:10F4800018B96888B0F5807F01D0022000E0012023
:10F490008DF84000BCE006A91DA8FDF700FF6088BC
:10F4A000404202B22088404201B21DA8FDF748FF49
:10F4B00017981599002809980ED0CDE90410CDE9C8
:10F4C0000259DDE91310CDE900011DA95046139B37
:10F4D000229A00F0E5FD0BE0CDE90310CDE90159DA
:10F4E00013980090DDE913231DA82299F7F737FC44
:10F4F000A87A022858D92A89C1B292B2D70A4F43B2
:10F5000067F30F00C2F345174F4302F01F024A434F
:10F5100062F30F03C1F1FF01CDE9041367F31F404C
:10F5200000223FE01599049B01EB420E521CBEF8ED
:10F530000010ADF82810BDF8287081B24FEAD72C22
:10F540000CFB031101EBC11C0CEBC131C1F3C45C1A
:10F55000BDF82C10C7F345186CF3CF214FEA104CBF
:10F5600008FB03CC0CEBCC1808EBCC3CCCF3C55C13
:10F570006CF34A11DDF814C007F01F071FFA8CFC6A
:10F5800007FB03C303EBC31707EBC333C3F3C45336
:10F5900063F30401ADF82C1089B20191BDF8043079
:10F5A000AEF80030B242BDD31898F0B1BDF91A7070
:10F5B000DDF8248015E000BFBDF918105B463A461F
:10F5C0004046FEF7EBFF10B1022804D006E0594692
:10F5D000404602F0EFFE02208DF840007F1CD84428
:10F5E0003FB2BDF91E00B842E6DA0CA95046FFF75B
:10F5F00045FDBDF81E00401CADF81A001A990844DC
:10F6000000B2ADF81E001699884201DDADF81E105B
:10F61000BDF91A00169988427FF73DAF099802F0AC
:10F62000B5FD159802F0B2FDBAE6000010B50C4623
:10F630005821204602F0BEFE10486061104820614B
:10F6400010482063104820621048A0611048606292
:10F650001048A0621048E062104860631048A06340
:10F660001048E06310482064104860641048A064AB
:10F67000104860652C20E06410BD000005ED000816
:10F68000C5FD000863F0000887F80008F5F20008DF
:10F690009DF9000841FB0008FDFD00089F000108DE
:10F6A0008FF200088BF70008B9F6000805F700088C
:10F6B00081F80008A9F000082DE9F04117460C4632
:10F6C0000646F5F7A5FE0546F807A06A20F00041BA
:10F6D0000BD0606902F06EFEA06A40F00041A162AA
:10F6E0002868016941F0400104E0A16228680169CD
:10F6F00021F04001016160690834C6E90004B4608A
:10F70000BDE8F081FEB505460068029000980C4601
:10F7100020F0E00000906868164681880088081A8A
:10F720000099401C60F3942100916868C18840886A
:10F73000081A0099401C60F35F510091A06A0028EC
:10F7400001DA052100E00421009861F30400009033
:10F75000206A2860E0696860A069A860F5F758FE33
:10F76000006894F824206B46016962F386110161F8
:10F7700004F1080231462846FEF7D0F9284600F089
:10F78000AAFC684601F012FAFEBD70B506461546A1
:10F790000C46D00701D0002070BDA80743D5A06A51
:10F7A00000F0004000F5C040A0622046FDF795FD46
:10F7B000A16A400021F00042824202D960F31E019A
:10F7C000A162A06A20F0004002F066FC2146606160
:10F7D00068B9A06A00F0004000F54060A06220F027
:10F7E000004002F059FC214660610028D4D0084650
:10F7F000D0E900128160E2606188E181A1892089FD
:10F80000081A401CA16A00B221F0004100EB40023E
:10F8100091FBF2F12182A16A21F0004191FBF0F00D
:10F82000411061822AE00846D0E900128160E2605E
:10F83000FDF753FD4100A06A61F31E00A06220F0B5
:10F84000004002F029FC6061A16A21F0004102F051
:10F85000B1FDA06A05F0010565F3DF70A062606983
:10F86000002899D0306004F108007060B060F5F7AE
:10F87000CFFD0068016965F386110161204670BD06
:10F88000486902F095BCF0B51C46074697B015468E
:10F890000E4608680023224601A900F0CEFCF0B312
:10F8A000BDF80C20002A3FD0BDF80A1000293BD03B
:10F8B0002888BDF80E30184400B2ADF84C0033680B
:10F8C0006D88B3F808C05B89ACEB03032B44BDF82B
:10F8D00010509B1A5B1B1BB2ADF84E304518B9682F
:10F8E000B1F900C065451FDBB1F90450A8421BDC2B
:10F8F0009818B1F90220904216DBB1F90600834254
:10F9000012DC2146019800F094FC00280CD00199EB
:10F91000097B890708D101AB13AA314600E005E055
:10F9200000903846F8F72CFC17B0F0BD202CFBD324
:10F93000A4F57840FF38F7D0A4F500500C38F3D088
:10F940002888BDF80E10BDF81020084401B2688860
:10F95000104402B2BDF80C00104400B20090BDF893
:10F960000A00084403B214A8FDF7F7FC05A8FFF746
:10F970008FF902208DF817008DF83E008DF84A00AF
:10F980008DF82E00B089ADF832000120ADF83400BA
:10F990003B6914AA05A938469847C5E72DE9F04701
:10F9A0000E46B1F9021096B01C4615468146002954
:10F9B0007ED0307A02287BD9B5F90000B4F9002056
:10F9C000904205D1B5F90230B4F90270BB426FD054
:10F9D000904200DB104601EBD171A0EB6100ADF865
:10F9E0004400B5F90010B4F90000B6F902208142D4
:10F9F00000DD084602EBD27100EB6100ADF8480073
:10FA0000B5F90210B4F90200B6F90220814200DA19
:10FA1000084602EBD271A0EB6100ADF84600B5F9E3
:10FA20000210B4F90200B6F90220814200DD084656
:10FA300002EBD27100EB6100ADF84A0011A9084653
:10FA4000D9F80820F4F778FC002875D011A9D9F866
:10FA500008A0C9F80810B5F90200B4F902108842EC
:10FA600006D123462A4631464846F8F7EBFC0EE01D
:10FA7000B5F90000B4F90010234688422A46314601
:10FA8000484602D1F8F744FF01E0F8F795FD707A97
:10FA9000010701D440074DD502A8FFF7F9F83088D7
:10FAA000ADF80C0047F6FF70ADF80800307A00E0C2
:10FAB00042E08DF80B00B6F90200471040F3000059
:10FAC00000F10108707A400718D528886A46C01BE3
:10FAD000ADF800006888C01BADF802002888C11985
:10FAE000A1EB0800ADF804006888C119A1EB08007B
:10FAF000ADF8060002A94846FFF7B6F8707A00078D
:10FB000018D520886A46C01BADF800006088C01B6D
:10FB1000ADF802002088C119A1EB0800ADF804007F
:10FB20006088C119A1EB0800ADF8060002A948469B
:10FB3000FFF79AF8C9F808A016B0BDE8F0870000F2
:10FB40002DE9FF4F8BB01F461646032B7ED3002EA8
:10FB50007CD0B80002F0CEFA05007BD000243068DB
:10FB6000286020467A1E15E006EB800136F9203029
:10FB7000B1F904C0634505D1B1F90230B1F906C04D
:10FB8000634505D005EB84030968641C1960A4B2C1
:10FB9000401C80B29042E7DB06EB8700B6F900100C
:10FBA00030F9042C914205D1B6F9021030F9022C3B
:10FBB000914206D005EB840150F8040C641C0860E7
:10FBC000A4B2032C43D37E49D1E90001CDE902015F
:10FBD000002027E0BDF9082035F920108A4200DA1C
:10FBE0001146ADF8081005EB8003BDF90A20B3F902
:10FBF00002108A4200DA1146ADF80A10BDF90C2055
:10FC000035F920108A4200DD1146ADF80C10BDF91F
:10FC10000E10B3F90220914200DC1146401CADF8F1
:10FC20000E1080B2A042D5D30B9802A9826805A815
:10FC3000F4F782FB58B10B9805A90026806809905B
:10FC40000B988160B5F90210012011E002E028460E
:10FC500002F09CFA0FB0BDE8F08F00BF05EB800208
:10FC6000B2F902208A4201DA114606B2401C80B283
:10FC7000A042F3D32C2104FB01F002F03BFA8346AF
:10FC8000B2460490D1464FF00008701E00D52044C3
:10FC9000621E09F101010892914200DD002135F850
:10FCA000203035F8262005EB80009B1A1FB235F86E
:10FCB000213005EB81019A1A05EB860340885B88A9
:10FCC0004988C01AC91A12B200B209B200235043BF
:10FCD00079430793884267DA0120079001E007988B
:10FCE000F0B308980AF10106864200DD0026B9F15A
:10FCF000010700D5274405EB860005EB8A01B0F922
:10FD00000200B1F90220904216DB12D035F92630FC
:10FD100035F92A108B420CD04FF0010CCDE9000CC4
:10FD20005846FEF71DFD58460499FEF795FA0BF16B
:10FD30002C0B08F10108B246A04523D005EB870043
:10FD400005EB8901B0F90200B1F90220904217DBFE
:10FD500013D035F9273035F929108B420DD000E04A
:10FD600022E00026CDE900065846FEF7F9FC584689
:10FD70000499FEF771FA0BF12C0B08F10108B94652
:10FD8000A045ACD3DDE90B0102AAFEF76DFF049894
:10FD9000FEF742FF049802F0F9F9284602F0F6F95E
:10FDA0000B990998886055E7BAF1010600D52644F9
:10FDB000089809F1010787429DDD00279BE70000B5
:10FDC000BCB0010870B514460D460646F9F79AFB1B
:10FDD000224629463046F7F7CBF9224629463046D7
:10FDE000F7F79BFB224629463046F7F788FC224668
:10FDF00029463046BDE87040F8F774BF2DE9FF4F43
:10FE0000A1B00D46309FDDF8CCB04FF48031B7F98A
:10FE100000004FF00A0940421A907888B1FBF0F0D8
:10FE20001A99199091FBF9F478681D90604200EBE3
:10FE3000800001EB400604F1010820B206F02AFC24
:10FE400005900FFA88F006F025FC82465A3420B25D
:10FE500006F020FC044608F15A0000B206F01AFC35
:10FE600002460598C6F10A0101FB00F30AFB0633BE
:10FE700093FBF9F0614302FB0611179091FBF9F037
:10FE80001890179840111790189840111890BDF9C4
:10FE9000740000021B90BDF9760000021C90A88837
:10FEA0002988401A401C04B2E8886988401A401C1E
:10FEB0000FFA80FA002648E00CA80090B5F902007D
:10FEC000B5F9001082190BAB13A809F036FE0EA885
:10FED0000090B5F90200B5F9041082190DAB13A812
:10FEE00009F02BFE0B9B0D980E99A0EB03080C98C4
:10FEF0000022A1EB000C1146012C08DD4FEA08227C
:10FF0000611E92FBF1F24FEA0C2C9CFBF1F103F124
:10FF100080093B7D8030DB071CD0DDE9318CCDF8DA
:10FF20000090CDE9010203AB83E81210CDE906B8D9
:10FF3000DDE92301DDE92E23F5F7DCFC3298761CA0
:10FF400000EB4400A34436B232905645B4DB25B0F2
:10FF5000BDE8F08F319B042B54D0052B13D0062B1A
:10FF600050D0142BEAD1239B1E93249B12932E9BDB
:10FF7000079305912F9B3299864609920020CDF870
:10FF80008090109188E0239B1293249B1093DDE9CD
:10FF90002E3C0491CE4632998146E04601920020E3
:10FFA00009912CE0049A0199424341430EEB21212F
:10FFB00009EB222209124FEA222207D4DDF840C0C1
:10FFC000614503DA002A01DB9A4203DB00210BF8CA
:10FFD000001012E002FB0811DDF848C001EB4101FE
:10FFE00061440A7891F801C002EB0C22DDF824C0CC
:10FFF0002CF810208A780BF80020401C00B2A04298
:020000040801F1
:10000000D0DB9BE7DDF8C8C0CDF80090CDE9010258
:100010000DF10C0888E81210CDE906B3DDE92301E3
:10002000DDE92E2308F096FA88E70999209A4143E2
:1000300002EB2121059A42430EEB222209124FEADC
:10004000222209D4DDF848C0614505DA002A03DB25
:10005000DDF81CC0624501DB002219E002FB031938
:10006000DDF87880DDF840C008EB49080CEB40096A
:10007000B8F80080A9F80080DDF81C8003FB08FCBC
:10008000DDF8788008EB4C0C614402FB03110A7820
:100090000BF80020401C00B2A042C6DB4EE77047C0
:1000A0002DE9F04387B08946DDE91251DDE910768C
:1000B000DDE90E8C70B1C46A002C08D0CDF8008048
:1000C000CDE904510396CDE901C74946A04707B0E1
:1000D000BDE8F083FEE7416B002900D00847704778
:1000E000007A20F08000704740687047017A152937
:1000F0000BD0142909D0162907D0182905D01729A3
:1001000003D0192901D00020704700697047017A97
:1001100001291FD002291DD003291BD0042919D081
:10012000052917D0062915D0072913D0082911D081
:1001300009290FD00A290DD00B290BD00C2909D081
:100140000D2907D00E2905D00F2903D0102901D081
:100150000020704700697047006970470068704769
:1001600010B588B0C0B1009001908DF80810002043
:10017000CDE903029DF81800084C20F007008DF827
:10018000180060680590C4F804D06846FAF78EF845
:100190000599616008B010BD0120FBE79C000020BC
:1001A000027A132A06D10069B0F900208A4200DDE4
:1001B00011460180704710B500F004F8BDE810400A
:1001C00000F06ABB10B500210C4801F02BFF0C4C6D
:1001D0002080002005F0D2FD6080042005F0CEFDD7
:1001E000A080042005F0CAFDE080042005F0C6FDD3
:1001F0002081042005F0C2FD608110BDB9AF000868
:10020000E400002010B5092900D120210469FBF782
:10021000D7F8002806D0616801EBC000618A890B1D
:1002200001D0002010BD00682168C0F3130008440D
:1002300010BD08B142681047FEE72DE9F0479A4625
:1002400090460C46070011D08CB100260546B146F9
:100250002660D5F800C05346424621462846E0476E
:1002600040B1A07BC00603D425600EE0FEE7FEE7A8
:1002700006B92E466D69002DEBD14EB13568534657
:10028000424621463046A84726600120BDE8F08757
:10029000B8F1200F20D3A8F57841FF391CD0A8F57C
:1002A00000510C3918D0B7F9080000EBD0704008A5
:1002B000E080801CA080C4F8009039892181A4F8D6
:1002C0000A90A4F80C90A07B20F00F00401C40F096
:1002D0001000A0730020D9E74846A4F80690E9E78B
:1002E0002DE9F0479A460C468146092A47D0002658
:1002F0001146D9F81050FBF763F8071E3DD0E868A7
:100300004FF0000850B151464846FBF759F802003B
:1003100004D039464846FBF70DF980466868298ABB
:1003200000EBC70001FB08F10A110168090D002E5E
:1003300002D000BF4FEA4101114401F108014FEA28
:100340001111A180417921810179E18090F9062084
:10035000628190F90700A081688A4FEA5022A07B51
:1003600062F3030020F01000A07304D04FF6FF707A
:1003700000EA4100E0804FF00100BDE8F0874FF057
:1003800001064FF02002B3E71FB540B113460A46FD
:100390006946FFF752FFBDF8040004B010BDFEE748
:1003A00070B504464068B0B1C268B2B121689047E8
:1003B00005466068408840B1A06830B1C06808B1A7
:1003C00001F0F6FEA06801F0F3FE002020606060FE
:1003D000A060284670BD0B2070BD092070BD0000D4
:1003E00010B504460748F4F75BFD08E0086800789C
:1003F000A04201D1086810BD0248F4F763FD010076
:10040000F4D110BDF852002010B50446F0F7FEF804
:1004100040B1215C2E2907D02F2903D05C2901D0BF
:10042000401EF6D102A010BD2044401C10BD0000AB
:100430000000000010F8011F3A2900D1401C70474D
:100440002DE9F04117460E0005462BD03078FFF716
:10045000C7FF040028D0616809B1884730B3A0689D
:1004600030B33046FFF7E6FF0146A3683A46204620
:100470009847F8B1411C1DD0C5E90004608870B1EF
:10048000102001F009FEA860B0B1102101F092FF28
:10049000A9684FF0FF300860A9684000486000205C
:1004A000BDE8F0810B20FBE70320F9E70120F7E727
:1004B0000920F5E70C20F3E7FEE77CB51C004FF0C0
:1004C000000500D02560436853B11B6953B1019505
:1004D00045686B88002B01AB06D000F012F80BE0EA
:1004E0000B207CBD09207CBD0093006813460A46A2
:1004F00001462E692846B047002CF4D001992160AE
:100500007CBD2DE9FF4F0546806814460027D0E9E1
:100510000021D0E902808146686883B09A46B0F82D
:1005200002B0424549D8884547D2A8EB020080B2C4
:10053000ABEB0006A1EB08018E4200D30E46B4429D
:1005400009EB000106D82246049801F06DFECAF8B6
:10055000004066E03246049801F066FE00200190FB
:1005600001A85C45009008D90498A31B8219D5E91D
:1005700000100769B847074617E0D5E900105B4649
:1005800007694A46B8470746A86842680260A968F2
:10059000019802444A60A11B814200D2084682B2FF
:1005A00004984946304401F03FFE01983044A0428F
:1005B00000D20446CAF8004030E05C4508D9CDF8C6
:1005C00000A0066929682346049AB047074625E03B
:1005D000B9F1000F06D1584601F05EFDA968C86068
:1005E000F0B181460020019001A80090D5E90010EB
:1005F0005B4606694A46B0470746A868C0F80080CF
:10060000019AA86808EB02019442416000D2224698
:10061000CAF800204946049801F006FE0FB106E032
:10062000FEE7A868DAF8001082681144816007B01C
:100630003846BDE8F08FF8B545680446E5B1AE69C7
:10064000E6B16B880020C3B3D2B1012A21D0022ABF
:1006500011D1134620680A4601462846B0470028B3
:1006600009D1D4E900106A46C3699847002802D12D
:10067000A26800999160F8BD0B20F8BD0920F8BD73
:10068000A2689160A3680A461D68A9420CD3596804
:1006900008E0A3689A680A449A60A1680B689A42C5
:1006A00002D349688A42EAD9D4E900100023846958
:1006B00001B0A446BDE8F0406047FFE7134620685C
:1006C0000A46014601B02846B446BDE8F0406047FE
:1006D0002DE9FC410C4681781546614309128A4296
:1006E00002DC0088BDE8FC81027A00EB820111F88F
:1006F000023C63431B129D4202DB31F8040CF1E71C
:10070000012358E000EB83018978614309128D428F
:100710004FDC00EB830737F8040DADF804000198B7
:10072000FDF732F80646B888ADF804000198FDF7E9
:100730002BF80146B878BA79604300126243D0EBD7
:1007400022223AD0281A00B2C0EB002090FBF2F02F
:10075000C2B2C8B2C2F1FF035043F4B204FB0300BB
:1007600000EBC01404EBC030840EBDF80000C6F3EB
:10077000072564F30400C1F307245443C1F3074180
:1007800005FB03445143C6F3074204EBC41502FBC7
:10079000031105EBC434640E01EBC11202EBC1314D
:1007A00064F34A10890E61F3CF20ADF8000080B2E7
:1007B00098E75B1CDBB29A42A4D8FEE741680029A7
:1007C00001DA01F0F5BC7047FEB50546407A1646E1
:1007D0000C4640072FD0224F387820B9002000F077
:1007E00043F801203870687A00F00700022818D01A
:1007F0004FEA060080EA6400684001900020009003
:100800006A4601A91748FCF785F901280BD0324642
:1008100021462846F4F730FF009000280BD0002432
:1008200018E02046E6E700980422416802EBB17127
:100830004FEAB1014160FEBD22462846FFF748FF5E
:1008400002900098BDF80810806800EB4400641C1A
:10085000018024B20098B0F90E10A142ECDCFEBD7C
:10086000D000002019A9000870B5094D0446286879
:1008700001F09EFC204601F00FFC2860054DA860A9
:1008800020B1214601F096FD6C6070BDFEE70000CE
:1008900070010020D000002010B50021164801F0A2
:1008A000C1FB164C2080042005F068FA608004200B
:1008B00005F064FAE080042005F060FAA0800420CE
:1008C00005F05CFA2081042005F058FA60820420CB
:1008D00005F054FA2082042005F050FAA08104208B
:1008E00005F04CFA6081042005F048FAE08104200C
:1008F00005F044FAA08210BDB9BA0008F00000204B
:1009000070B506000C4633D0084600F0D1F83046EA
:10091000F4F7C6FA05E00868A04229D03046F4F79B
:10092000D1FA0100F7D1204602F0D6FC40B1A1680F
:10093000896829B1C9680968A14201D100F0A3F80A
:10094000A06810B9204601F043FEA06886603046DA
:10095000F4F71AFB05000AD030462C60F4F7A0FA31
:10096000A84205D13046BDE8704000F08CB8FEE7E3
:1009700070BD000010B50446074A0849FAF784FC28
:100980006269002A06D0002804D12046BDE8104044
:100990000121104710BD0000C54E0008A14E0008FF
:1009A00070B5060043D002F097FC04003FD0207FD2
:1009B000C0073CD10021204600F0D7F82046F4F7CC
:1009C0006FFA32E02868B0422BD1E06888B1006845
:1009D000B0420ED02046FAF785FD0246E0680F21AE
:1009E0000068FFF7BDFB012821D1E068006803F033
:1009F000BFFDE560002D1AD0216909B12046884766
:100A00002046FAF76FFD0246E0680E210068FFF706
:100A1000A7FB01280BD1E0680068BDE8704003F037
:100A2000A7BD29462046F4F74DFA0500CAD170BD8E
:100A300010B50446074A0849FAF726FC6269002AFD
:100A400006D0002804D12046BDE810400021104700
:100A500010BD0000CD4E0008D34E000801480068CC
:100A600070470000A4000020002802D0007FC0F3DF
:100A700040007047002803D0C068002800D00068FC
:100A80007047F4F711BA70B50446007FC0F3C00593
:100A900040F0080020774007204602D4FFF76AFFA5
:100AA00001E0FFF7C5FF207F65F3C300207770BD2D
:100AB0002DE9F041064602F00FFC04003DD0E0684D
:100AC000002740B30068B04220D1207FC10702D088
:100AD00020F0010020772046F4F7E2F9E16888422F
:100AE0000FD12046F4F7F5F9E168884209D1204694
:100AF000FAF7F8FC0246E0680F210068FFF730FBC8
:100B000002E02046FFF7BFFFE06820B1E068006820
:100B1000B04200D1E7602046F4F7C2F911E028683E
:100B20002946B04220460AD1F4F755FA284601F08A
:100B30003FFBB068002800D08760BDE8F081F4F783
:100B4000C1F90500EBD1F8E713B5FFF793FF0400F7
:100B500003D0802103F032FB08B101201CBD01AAA3
:100B60000D212046FFF7FCFA1CBD70B504001CD017
:100B7000207FC0F340028A4217D061F34100207702
:100B80002046FFF777FF05000FD02046FAF7AAFCB2
:100B90000246E0680E210068FFF7E2FA012804D15E
:100BA0002846BDE8704003F0E3BC70BD70470146C5
:100BB00000200F290AD2DFE801F009090909080A13
:100BC000080C0E10120C0E10120010207047182086
:100BD00070470120704702207047042070470820AA
:100BE000704701460020891E0D2909D2DFE801F077
:100BF0000708080708070707070707070700012076
:100C0000704701460020032901D0062900D10120A8
:100C1000704770B54C6A0D46002C12D0287C012814
:100C200002D12046FFF7BCFBE06808B101F0C0FA32
:100C3000206908B101F0BCFA204601F0B9FA0020A1
:100C4000686270BD7FB514460D46084600F0B9FBDA
:100C500020B1012817D0022839D035E0296801F0E9
:100C60001F00001F11282FD2880A216860F39421E9
:100C700021602868400D60F35F512160287860F39F
:100C8000040121602FE02846FFF7BEFB17A1EFF714
:100C9000A5FDC8B9022229466846FFF7D1FB68B90D
:100CA00003AB042221466846FFF707FC0546684669
:100CB000FFF776FB45B90398042805D1207800F0AA
:100CC0001F00001F11280ED3002004B070BD206843
:100CD000012161F39420C0F3140000F5001020F00E
:100CE0001F000B3020600120EFE7000062696E00FA
:100CF0002DE9FF4F80465CA087B0006804905BA0A0
:100D00005BA3006893460F4605900FCB8DE80F005C
:100D1000B8F80810002089B2CAB2090A09E000BF79
:100D2000149C00EB4003401CE254149C00B223448A
:100D300059700A9B9842F3DB98F814004FF00009B1
:100D400000F01F00FFF733FF8246012101FA0AF18C
:100D5000491E88B206900025D8F814002C4600F0F1
:100D60001F012E460B2906D00C2912D00D2920D0A8
:100D70000E2931D12CE0C0F38A20C01DC50804EB38
:100D8000E70107F0070005FB0B14C0F1070604A8F4
:100D90000DE0C0F38A20C01C850804EBA70105FB09
:100DA0000B1407F003000621A1EB400605A88146BD
:100DB00012E0C0F38A20401C450804EB670105FBE4
:100DC0000B1407F001000421A1EB80066846EEE752
:100DD000C0F38A2505FB0B742846D8F8247001F06F
:100DE00089F95FEA000B13D098F81000A0B1002237
:100DF000211D3846FFF71FFC00232A465946384676
:100E0000FFF75BFB5946CAF10802002053B222E00B
:100E100000200BB0BDE8F08FD8F8040080680119FD
:100E2000F1E70A78069CF240224098F8144004F05A
:100E30001F040E2C01D019F80220149C00EB400571
:100E40002C44A270A6EB0A0256B2002E01DA1E460E
:100E5000491C401C00B20A9A9042E2DB584601F05D
:100E600095F90120D5E7000000FF00000055AAFF1A
:100E700000112233445566778899AABBCCDDEEFF7A
:100E80002DE9FF4F8046007D81B091460E4600F06F
:100E90001F00FFF78CFE8246012101FA0AF1491E6C
:100EA0000025D8F814001FFA81FB00F01F012F461F
:100EB0002C46072906D0082912D009291FD00A2953
:100EC00032D12BE0C0F38A20C01DC50804EBE60137
:100ED00005FB091406F00700C0F10707083423E0FA
:100EE000C0F38A20C01C850804EBA60105FB091489
:100EF000062106F00300A1EB4007103414E0C0F314
:100F00008A20401C450804EB660105FB09140421F6
:100F100006F00100A1EB8007403405E0C0F38A250C
:100F200005FB096404F580642846D8F8249001F094
:100F3000E1F8061E40D098F8100068B10022211D8B
:100F40004846FFF778FB00232A4631464846FFF71C
:100F5000B4FA3146002028E0D8F80400806801196E
:100F6000F8E70A78D9F80C30FA4002EA0B0203EBF2
:100F700042030E9D1B8800EB4004ADF800302B555A
:100F8000BDF800301D0A0E9B23445D70D9F8104057
:100F9000A25C9A70A7EB0A0257B2002F03DACAF1DB
:100FA000080257B2491C401C00B2049A9042D8DB98
:100FB000304601F0EBF8012005B0BDE8F08F0000ED
:100FC0002DE9FE430646087C0C46012801D028B3D3
:100FD00028E06068FFF718FA6BA1EFF7FFFB002825
:100FE0005BD1022268466168FFF72AFA0028F7D130
:100FF000606A38B9142001F04FF8606268B11421BA
:1010000001F0D8F9D4F8240069460C2211F8013B0C
:1010100000F8013B521EF9D104E0FEE760688068E9
:10102000002874D0616901F01F000E2816D0142822
:1010300014D004283AD0052838D0062836D00728FE
:1010400038D0082836D0092834D00A2832D00B28C6
:1010500027D00C2825D00D2823D08FE0227CEAB1A0
:10106000C1F38A22490D4A4314281BD00126564356
:10107000304601F011F805000FD0676A0022042104
:101080003846FFF7D8FA0023324629463846FFF79C
:1010900014FA48B1284601F08BF873E06068806864
:1010A000A06168E00326E2E7A56164E0207C0028F7
:1010B000F4D060E0FFF77BFD01278740606A38B914
:1010C000142000F0E9FF6062B8B1142101F072F958
:1010D0007800656A00F0E0FFE86078B1384600F01B
:1010E000DBFF286158B1E86878B3207C012807D07D
:1010F00060680024D0F808803BE0FEE7FEE7FEE7EA
:10110000002204212846FFF796FA00241AE033E073
:101110000023042269462846FFF7CFF99DF80020F6
:101120009DF801109DF80200FCF77DFA0190E86837
:10113000BDF8041000EB4400018029699DF803000C
:101140000855641CBC42E3D315E017E008EB8406A5
:1011500018F824207178B078FCF765FA0090E868F8
:10116000BDF8001000EB440001802969F0780855B3
:10117000641CBC42EAD30120BDE8FE832146304610
:10118000FFF747FD0020F7E762696E002DE9F84F91
:101190000C461D461646207DDDE90A32002100F08E
:1011A0001F00042816D0052814D0062812D00B28BA
:1011B00039D00C2837D00D2835D00E2833D0072849
:1011C00038D0082836D0092834D00A2832D0002058
:1011D000BDE8F88F277C012F33D198469146D4F88B
:1011E00024A0FFF7E4FC074660690022C0F38A20D0
:1011F00005FB00607843C1105046091DFFF71BFA3C
:10120000002470B9FD0805FB08F56B462A464946DF
:1012100050460094FFF751F918B90098854200D163
:10122000012421460DE000922A4631462046FFF770
:101230005FFD05E000922A4631462046FFF720FE7A
:1012400001460846C4E710B50446006800280BD0E4
:10125000C2680AB121469047207C012804D1606809
:1012600000F0A6FF0020606010BD000010B505482A
:10127000F3F73BFE040004D0142101F09BF8204654
:1012800010BDFEE71C5300202DE9F0410F46054636
:101290000421384601F08EF825B1284600F091F877
:1012A00018B105E00020BDE8F081A8680028FAD058
:1012B00000260A48F3F7F4FD0BE023682BB13A4609
:1012C000294698470646012805D021460348F3F7EA
:1012D000F9FD0400F1D13046E5E700001C53002081
:1012E0002DE9FF410E461D460446282101F062F813
:1012F000AEB1304600F065F808B9B16879B1BDF813
:10130000081021812074E56001280CD06660002758
:101310002148F3F7C5FD054604F1140831E000202B
:1013200004B0BDE8F0813046EFF770F9401C00F0E2
:10133000B3FE606018B13146EFF744F9E7E7FEE726
:101340002B68CBB16868B8B1424631462846984709
:101350000746012810D125606A6821462846904733
:1013600007460128DCD00421404601F023F8002084
:101370002062A0616062E06129460748F3F7A2FDA0
:101380000546002DDCD1207C012802D1606800F0E8
:101390000FFF3846C4E700001C5300202DE9FC4134
:1013A00005680E46089FAC6800213CB1CDE90037C6
:1013B0001346014632462846A04701460846BDE886
:1013C000FC81032130B10078A0F120015F2903D80E
:1013D0000120704708467047802801D302207047DB
:1013E0000020704710B50446202100F0E3FF0020E4
:1013F00020700A20207660764FF4C870A0836420A5
:10140000E0833220E0760320A07610BD70B505465B
:10141000006920B9FCF700FB2861002814D00B48B4
:10142000F3F763FD040010D05C2100F0C3FF2560DA
:101430006079224640F0020060711E21044804F0E9
:101440003FFF21684861204670BDFEE7EC52002056
:10145000C11401080148806870470000A8000020FE
:1014600018B101460248F3F72DBD0148F3F718BD46
:10147000EC5200200148406870470000A80000209E
:10148000002806D001680978012903D0032901D07A
:101490000020704790F8440000F00F0070470028CB
:1014A00006D001680978012903D0032901D0002062
:1014B0007047006B7047002801D0006800787047C3
:1014C0007FB52A4CC068A0600168096900294CD02A
:1014D000FBF7E4F8A0684179490746D40068006941
:1014E0004069002841D100256946A068F3F76EFAEB
:1014F0009DF80F60A068FBF7D1F86560A1689DF8C2
:101500000E000871012806D008680078042809D167
:10151000BDF80C00D0B104F0BFFEA16809680969EC
:10152000C1F86401A06801680978012906D0022980
:1015300008D004290AD003290DD00FE06946FAF734
:10154000D3FE0BE06946FAF7E3FD07E06946A068C1
:10155000FAF7C2FB02E06946FAF738FBA068FBF72E
:101560009DF8002EC0D1A56065607FBDA800002059
:10157000F8B50C460546012102F014FE68BB206850
:101580000090012300226946284604F0B1F869461C
:10159000284602F018FE06460022694605F11400AE
:1015A000F2F7B2FF28B94FF40021284602F0FAFD05
:1015B00080B1284601F0D6FD401E04000AD4A86878
:1015C0006946006850F82400FFF7D2FF002803D1D5
:1015D000641EF4D50EB12846F8BD0020F8BD02689F
:1015E0001278032A00D181657047000010B5144CB1
:1015F0002078002821D100F0F1FDF3F737FFF3F751
:10160000DDF8F2F7E3FDF3F7DFF8FCF7D3FAF3F7D1
:1016100001FE4FF4B4710B48F3F75FFC5C210A48FC
:10162000F3F75BFCF3F7FAFEF3F7B4F94420112863
:1016300004D0FEF7C0FD0120207010BDFEE70000C1
:10164000B4000020E0520020EC52002010B50C46FF
:101650000020486214F8481F21F0180104F81C19F2
:10166000411E2160227F22F00702227720836083BF
:10167000E060C4E90110090C2161616144F8040CC7
:1016800014F81C0F022120F0400004F848092046FD
:1016900001F068F90021204600F050FC2046BDE82A
:1016A000104001A100F086BC546578740000000071
:1016B00010B50146034801F0A7F8044601F018F9F7
:1016C000204610BDE8E8010810B508460C4600F0B9
:1016D0000AF894F84800000702D4606A00F068FD38
:1016E0000020606210BD10B5044690F84800400626
:1016F00003D5A06A08B100F05BFD94F8480020F023
:10170000400084F848000020A06210BD2DE9FF478A
:101710000E463F4801F0FEFC012876D13046FEF728
:10172000DFFC04463046FEF719FD05462A2C1CD086
:10173000132C0BD0292C18D02C2C1ED0152C64D196
:1017400004B03046BDE8F047F7F791B9002102F048
:1017500025FCB0F9080004B0C11700EB91708110AE
:101760003046BDE8F047FEF71BBD00F0B5FB04B006
:101770002846BDE8F04700F04BB9002102F00EFC0E
:1017800081460021284602F00CFC804600212846B4
:1017900002F00DFC074695F848000024C10600D56C
:1017A0000124800601D544F00204284601F046FDDC
:1017B0000021284602F02BFCA0F51C51D13905D19F
:1017C000688C000502D441F6FF7002E0284601F063
:1017D00035FD0097CDE9010443464A4603A8696AEE
:1017E00005F01CF83046FEF7B7FCB0F90020BDF953
:1017F0000C108A4200DD11460180B0F90220BDF9CB
:101800000E108A4200DD11464180BDE8FF870000CE
:10181000E8E801082DE9F04F8BB00D00804659D063
:101820000021122202F03CFB29881022081A60F3E2
:101830000F044046002102F033FB6988081A60F368
:101840001F44A14608A9404601F0B0FCBDF82400A1
:10185000BDF820100025401A401C00B2D8F82470B2
:1018600005902C462946404602F098FB0290002144
:10187000404602F09CFB00900021404602F091FBA4
:1018800003900298AB465E46B0F90800079098F8BE
:101890004800C10600D50126800601D546F00206A3
:1018A0000021404602F0B3FBA0F51C51D13905D10F
:1018B000B8F82200000501D446F004064046002195
:1018C000D8F8242000F086FF82460099079800EBA4
:1018D000010821E0FEE70020CDE90006DDE9021263
:1018E0007819059BF3F7E8FD044407984FEA29426D
:1018F000584482420BDC444A0094694612683846D8
:1019000090470A280BD0385D48B9641C07E008EB03
:101910000B000FFA80FB2546785D0028DBD107EB32
:10192000050B4FF00008BAF1020F03D0BAF1030F14
:1019300016D025E0DDE90223611B5846009604F02D
:10194000CBFFBDF82410BDF8202000EBD070891A21
:10195000491C09B201EBD1714910A1EB60000DE007
:10196000DDE90223611B5846009604F0B5FFBDF87F
:101970002410BDF82020891A491C081A0FFA80F893
:1019800000208DF818008246049044BB2BE004AB85
:101990006A4601A95846F3F777FDF00706D0049888
:1019A0001BF8001006A8F3F707FEC0B9DDE9011027
:1019B000009AFEF7E9FC01B20FFA89F208EB010088
:1019C00082421EDB04994A19A2421AD00AEB050290
:1019D000BA5CB2B1039A8A4610440FFA80F80498B0
:1019E0002844A042D3D3094C584604992268904712
:1019F000064622682946384690470BB03044BDE879
:101A0000F08FCDF810A0EEE7B0010020B401002067
:101A10002DE9F04F0446406A97B000287ED04FF081
:101A2000FF3903A92046C4F8309001F0BFFBBDF890
:101A30001000BDF80C10401A401C0FFA80F800216D
:101A4000204602F0ABFA05460021204602F0AFFA2C
:101A500007460021204602F0A4FA824694F8480086
:101A60000026C10600D50126800601D546F00206F3
:101A70000021204602F0CBFAA0F51C51D13904D147
:101A8000608C000501D446F004060097CDE901867C
:101A900053462A4616A8616A04F0C0FE204603F0A9
:101AA000C7F994F848004FF6FF7B00F007004FF0AD
:101AB0000008022804D003287ED001287DD0F6E15A
:101AC0000021204602F0D2F80604360C08D1204648
:101AD00001F0D4FBFBF7A6FF032190FBF1F086B2E7
:101AE00005A8FBF71DFB4FF4967005941290149017
:101AF000BDF81000BDF80C10BDF95820401A401C6C
:101B0000002700B2ADF854B0904233DA0021801AB9
:101B1000CDE90E10E9480D91014600E0CAE10690BA
:101B20002046FBF7E5FA00210A4620B1016B90F848
:101B30004200C0F34002109888420FDD9DF8560025
:101B4000119120F001008DF856003AB140F00200EA
:101B50008DF856000F990D980D910F9030460F9A01
:101B60000D99FBF723FB1090139005A8FBF72CFBB6
:101B7000012705E0D1492046FBF78AFAA4F8448002
:101B8000BDF81200BDF80E10BDF95A20401A401CD5
:101B900000B290427EDA002F7CD1821AB5F908009B
:101BA0000021101ACDE90E10C5480D91014606908E
:101BB0002046FBF79DFA01E023E0C5E000210A463C
:101BC00020B1016B90F84200C0F3400210988842A7
:101BD0000FDD9DF85600119120F001008DF85600A0
:101BE0003AB140F002008DF856000F990D980D9112
:101BF0000F9030460F9A0D99FBF7D8FA109013907A
